:020000040800F2
:10800000008001204D8C02083D4902083F490208CA
:10801000414902084349020845490208000000009E
:1080200000000000000000000000000047490208B6
:1080300049490208000000004B49020881CA0108B2
:10804000918C0208918C0208918C0208918C020894
:10805000918C0208918C020865EB0108C5EB0108C0
:10806000918C0208918C0208918C0208918C020874
:10807000918C0208918C0208918C0208918C020864
:10808000918C0208918C0208918C0208918C020854
:10809000918C0208918C0208918C0208918C020844
:1080A000918C0208918C0208918C0208918C020834
:1080B00051F70108918C0208918C0208918C0208FA
:1080C000918C0208918C0208918C0208918C020814
:1080D000918C0208918C0208C9DF010859DC010863
:1080E000918C0208918C0208918C0208918C0208F4
:1080F000918C0208918C0208918C0208918C0208E4
:10810000918C0208918C020825EC0108918C0208E0
:10811000918C0208918C0208918C0208918C0208C3
:10812000918C0208918C0208918C0208918C0208B3
:10813000918C0208918C0208918C0208918C0208A3
:10814000918C0208918C0208918C02089FD501083D
:10815000918C0208918C0208918C0208D9D90108EF
:10816000918C0208918C0208918C0208918C020873
:10817000918C0208918C0208918C0208918C020863
:04818000918C0208D4
:1081880010B5054C237833B9044B13B10448AFF349
:1081980000800123237010BDD00E002000000000D5
:1081A80048B802080C4B43B10C4810B50C49AFF362
:1081B80000800C48036823B910BD0A48036833B926
:1081C8007047094B002BF7D0BDE810401847064B05
:1081D800002BF5D0184700BF0000000048B802087F
:1081E800D40E0020CC0E002000000000000000008B
:1081F80010B516F03BFD0022054B1A70054B1B68A5
:108208009847BDE81040044B9B695B69184700BF5D
:10821800C0090020A0000020649E0208431E2DE92A
:10822800F0471446052B00F22281DFE813F0060020
:108238000C000C004F007A00D000FFF7D9FF47F67A
:10824800A85323603FE0904B904D022816BFA946E3
:1082580099461D464FF0FF364FF000084FF0010ACF
:108268008B4BA9F10409DF68043D3B68D9F8040089
:108278001B6998473B686868DB6898473B6868688B
:108288005B6998473B68D9F804001B6A984718B996
:108298000AFA08F326EA03063B6855F8040F9B69B7
:1082A80098473B6859F8040F1B6A984718B10AFAAF
:1082B80008F326EA030608F10108B8F1110FD4D132
:1082C800C6F3100626600020BDE8F0872160032968
:1082D8002DD8DFE801F0021B1F236D4BDB691B68FB
:1082E800188880B21FF0ECFC63A3D3E900231FF0C9
:1082F80077FE63A3D3E900231FF048FD0022654BF6
:108308001FF044FD1FF054FF2060DCE7604BDB6981
:108318005B68E5E75E4BDB699B68E1E75E4B1B69E1
:108328008FE70129216021D004D3022934D002200B
:10833800BDE8F087564BDC686068236820309B688E
:108348009847606823683C30DB6898476068236812
:108358005830DB689847236860685B693C30984709
:10836800236860685B6958309847ACE7484BDC681D
:10837800606823683C309B689847606823682030B1
:10838800DB689847606823685830DB6898476068FE
:10839800236820305B69E2E73D4BDC68606823684E
:1083A80058309B689847606823682030DB68984796
:1083B800606823683C30DB68984760682368203031
:1083C8005B699847236860685B693C30CCE70129A2
:1083D800216036D01BD30229A9D12D4BDC686068F7
:1083E800236858309B689847606823682030DB68AA
:1083F8009847606823683C30DB6898476068236862
:1084080020305B699847236860689B69DDE7204BEB
:10841800DC686068236820309B6898476068236838
:108428003C30DB689847606823685830DB689847B9
:10843800236860685B693C309847236860689B697B
:1084480091E7134BDC68606823683C309B68984769
:10845800606823682030DB68984760682368583074
:10846800DB6898476068236820305B69E4E704208C
:10847800BDE8F087AFF300800000000000FEAF40C9
:10848800AAF1D24D62101440FC3E0020DC3D0020D1
:10849800649E020800002440C009002038B5064C3C
:1084A80005462368C31AB3F5FA7F04D3034B9B69C7
:1084B8009B699847256038BDEC0E0020649E020831
:1084C8003B4B3C4ADB685B6803F5B871116003F10C
:1084D800AC01516003F1E401916003F58E71D16044
:1084E80003F5AA71116103F5D471516103F5F071B7
:1084F800916103F50671D16103F51471116203F5F9
:108508002271516203F53071916203F53E71D162B7
:1085180003F54C71116303F55A71516303F56871E2
:10852800916303F57671D16303F582611164224A80
:1085380003F17401116003F19001516003F1C80166
:10854800916003F58071D16003F59C71116103F5A9
:10855800C671516103F5E271916103F5FE71D16154
:1085680003F50D71116203F51B71516203F5297151
:10857800916203F53771D16203F54571116303F513
:108588005371516303F56171916303F56F7103F5DD
:108598007D731364D1630122084B1A70084B094A92
:1085A8001A65094A9A65094A5A651CF039B800BF24
:1085B800649E0208DC3D0020FC3E0020C00900202B
:1085C800203E002025820008F9810008A5840008C3
:1085D800704702207047022070477047704702209A
:1085E800704702207047022070470120704770478B
:1085F80070474369124A10B5C3F80422C3F8082229
:10860800104B11498365114B114A836183620363DF
:10861800C361104B104C4364104B41628364104B90
:1086280010494363C36303640F4B42650366002329
:10863800C16284630465C164C265836610BD00BFFE
:10864800F3850008D9850008DB850008DF85000868
:10865800F9850008E3850008EF850008E58500082E
:10866800EB850008E7850008F7850008704700BF1C
:108678000022012110B44FF0FF340848084B80F85D
:108688007C205A7083F810124467C0F880308167E4
:1086980002671A706C3010BCFFF7ABBF203E002099
:1086A800FC0E0020012108480023C1604FF0FF3173
:1086B800064A81601370537082F810324261037465
:1086C8004360FFF796BF00BF203E00201C1100202A
:1086D8000023184610B5064C1A5D590002F0030233
:1086E80001338A40072B40EA0200F5D110BD00BFD4
:1086F8003C130020002304495A5C02F00302C254D0
:108708000133072BF8D170473C130020074B1A7828
:1087180002705A7842709A788270DA78C2701A7940
:1087280002715A7942719B79837170473C1300201A
:10873800F8B50024084B094F094DDE68E15D336840
:108748006A6CDB6952F8240001F003010134984790
:10875800072CF3D1F8BD00BF649E02083C1300202B
:10876800000000200023054A00F00301995401335A
:10877800072B4FEA9000F7D1DAE700BF3C1300203F
:10878800014B586AEEE700BF0000002000230449AF
:10879800C25C02F003025A540133072BF8D1C7E731
:1087A8003C1300200278074B1A7042785A7082787E
:1087B8009A70C278DA7002791A7142795A7182799C
:1087C8009A71B5E73C1300200022014B1A677047E5
:1087D800203E002070B504460A4E0B4D33682A46E9
:1087E8000146002017F0CAFC002017F097F83368FC
:1087F8002A462146012017F0C1FCBDE8704001203F
:1088080017F08CB8C0410020403F0020012808B56F
:1088180003D817F077F8002008BD082008BD012804
:1088280008B503D817F062F8002008BD082008BD75
:108838000021F4E74942F2E7F1E7024B186817F024
:10884800ADBC00BFC041002038B5002017F044F986
:1088580008B1002038BD012017F03EF90546002870
:10886800F7D10A4B0A4C186817F08FFC17F07AF901
:108878002B46A2682168284617F0C4F82B46E26800
:108888006168012017F0BEF8012038BDC041002002
:108898006C130020022804BF0B4B93F8D80030B9A2
:1088A8000A4BDB681B685B69094A1069184701288D
:1088B80009D1054B93F8D830012B04D1034BDB6861
:1088C8001B689B69F0E77047203E0020649E020801
:1088D8006C13002070B50020FFF7DCFF0A4B0B4C2F
:1088E800DD6820692B689B6898472B68206A9B681D
:1088F80098472B68606A9B68984717F087F9BDE826
:108908007040034B5B681847649E02086C13002094
:1089180070090020012838B504460D4605D820B94D
:1089280017F0DAF82860204638BD082038BD02283C
:1089380010B5144610D0032815D0012817D10D4BB7
:108948000D4ADB68106A1B681B6A9847003018BF1D
:1089580001202060002010BD064B074ADB68506AE2
:108968001B681B6AF1E7084617F02CF8F1E70420AA
:1089780010BD00BF649E02086C130020012838B5A2
:1089880004460D4608D817F08DF82B68C1182960E1
:108998002046BDE8384039E7082038BD2DE9F843BE
:1089A8000F4691469846174C0021236847F08000EF
:1089B8009B689DF820609DF8245098472368002103
:1089C8009B6848469847236800219B68404698471B
:1089D800236800219B6830469847236828469B688F
:1089E80001219847084B48EA09281B6846EA0826E7
:1089F80007F07F0703EB870745EA06257D60BDE89A
:108A0800F88300BFC4410020C041002007B5D3B29D
:108A18000193C2F307230093C2F30743120EFFF733
:108A2800BDFF03B05DF804FB0020FFF7EFBF38B5CA
:108A3800234B01F07F04234493F80032DB0705D46D
:108A4800204B1B6803EB8404606838BD1E4D002171
:108A58002B6820469B68984700212B6808469B682E
:108A6800984700212B6808469B68984700212B6887
:108A780008469B6898472B6801219B680020984707
:108A88002B6800219B682046984700212B680846E0
:108A98009B68984700212B6804029B680846984702
:108AA80000212B6804439B68084698472B682402DA
:108AB80004439B680121002098472402204338BDC5
:108AC800403F0020C0410020C441002010B50020D4
:108AD8001446FFF7ACFF206010BDA42A2DE9F04131
:108AE80004460D461E4600F0C18149D8062A00F00A
:108AF800E38017D8022A00F0B78007D8002A00F0D0
:108B08009680012A00F0A480042499E0042A00F049
:108B1800BD8040F2B580002840F0C780084616F0B6
:108B2800F7FF88E01D2A00F01D8114D8082A00F0FC
:108B38000081C0F0E1801C2AE6D1002840F00081C5
:108B4800090141F06C0101F0FC012846FFF76FFFB5
:108B5800C0F380406FE0A22A00F04C8100F26881E7
:108B68008C2AD1D1002840F00381090141F06C0121
:108B780001F0FC012846FFF75AFFC0F303605AE0F2
:108B8800AC2A00F0878229D8A82A00F0188212D8C7
:108B9800A62A00F0D98140F28781002840F0FE81A2
:108BA800090141F06C0101F0FC012846FFF73FFF85
:108BB80000F00F003FE0AA2A00F03C8240F21C823D
:108BC800002840F05582090141F06D0101F0FD01D6
:108BD8002846FFF72CFFC0F341102CE0B42A00F020
:108BE800BC8214D8AE2A00F08182C0F06182B32A18
:108BF8008AD1002840F09F82090141F06C0101F000
:108C0800FC012846FFF713FFC0F3404013E0B82AE1
:108C180000F0B882CE2A00F0D382B52A7FF474AF70
:108C2800002840F0A782084616F08EFF03E020B91E
:108C3800084616F043FF306002E0012803D0002404
:108C48002046BDE8F0811968284616F05BFEF6E775
:108C580018B9084616F026FFEDE70128EFD1196884
:108C6800284616F0F9FEEAE718B9084616F042FF5A
:108C7800E1E70128E3D11968284616F037FEDEE758
:108C8800002871D1084616F027FFD4E718B908461E
:108C980016F04CFFCFE70128D1D1196828460029E2
:108CA800B8BF494216F0E6FEC9E70128C7D11968DE
:108CB800284616F0D2FFC2E750B92021A94041F05A
:108CC8001001C9B22846FFF7B2FEC0F30420B2E78C
:108CD8000128B4D120248C4044F01004E4B2214689
:108CE8002846FFF7A4FE336820F4F8521B0203F469
:108CF800F8531A43214623E150B92021A94041F0F5
:108D08001001C9B22846FFF792FE00F01F0092E753
:108D1800012894D120248C4044F01004E4B2214668
:108D28002846FFF784FE336820F01F0203F01F0374
:108D3800DFE7C8B9084616F045FEC0F300107AE729
:108D480001287FF47CAF0C0144F06C04E4B22146A6
:108D58002846FFF76CFE336820F480229B0403F456
:108D68008023C6E700288ED0012C3FF4CDAE66E7FD
:108D780001287FF464AF1B68102B23D00DDC022B75
:108D88001CD004DC012B16D04FF0FF3314E0042B69
:108D980016D0082BF8D105230EE0402B14D003DCA5
:108DA800202BF1D1032307E0802B0FD0B3F5807F70
:108DB800EAD1002300E00823336008E00723FBE73B
:108DC8000623F9E70423F7E70223F5E73060336861
:108DD80001333FF434AF2C0144F06C04E4B2214673
:108DE8002846FFF724FE336820F070621B0603F064
:108DF80070637EE750B9090141F06C0101F0FC0194
:108E08002846FFF714FEC0F3C13014E701287FF4A9
:108E180016AF0C0144F06C04E4B221462846FFF773
:108E280006FE336820F4C032DB0303F4C03360E786
:108E380050B9090141F06C0101F0FC012846FFF727
:108E4800F6FDC0F38030F6E601287FF4F8AE0C0199
:108E580044F06C04E4B221462846FFF7E8FD336885
:108E680020F480429B0303F4804342E750B9090190
:108E780041F06C0101F0FC012846FFF7D8FDC0F372
:108E88000030D8E601287FF4DAAE0C0144F06C0417
:108E9800E4B221462846FFF7CAFD336820F4805221
:108EA8001B0303F4805324E70F0147F06C07FFB25C
:108EB80039462846FFF7BBFD8046A4B918F4804F11
:108EC8003946284604D0FFF7B2FDC0F3C310B2E616
:108ED800FFF7ADFD18F4006FC0F3021018BF40F0A3
:108EE80008003060ABE6012C7FF4A9AE18F4804886
:108EF8003946284608D0FFF79AFD336820F4F06217
:108F0800DB0103F4F06347E0FFF791FD326820F0DE
:108F18007000120102F07002024339462846FFF73A
:108F280075FD39462846FFF782FD336820F4006254
:108F380013F0080F18BF4FF4006842EA08023946D8
:108F48002846FFF763FD7AE60F0147F06C07FFB28A
:108F580039462846FFF76BFD74B910F48048394646
:108F6800284604D0FFF763FDC0F3021063E6FFF75D
:108F78005EFDC0F3C310B4E7012C7FF460AE10F4BB
:108F8800804F39462846B6D0FFF751FD336820F0A8
:108F980070021B0103F070031A43D0E701287FF425
:108FA8004EAE0C0144F06C04E4B221462846FFF7AB
:108FB8003EFD336820F00F0203F00F0399E650B925
:108FC800090141F06D0101F0FD012846FFF72FFD71
:108FD800C0F3C0302FE601287FF431AE0C0144F015
:108FE8006D04E4B221462846FFF721FD336820F4DA
:108FF8000042DB039BB27CE650B9090141F06D01E8
:1090080001F0FD012846FFF712FDC0F3413012E6DA
:1090180001287FF414AE0C0144F06D04E4B221463B
:109028002846FFF704FD336820F4C0425B0303F4CD
:10903800C0435EE650B9090141F06D0101F0FD0140
:109048002846FFF7F4FCC0F30320F4E501287FF479
:10905800F6AD0C0144F06D04E4B221462846FFF752
:10906800E6FC336820F470621B0203F4706340E688
:1090780001287FF4E4AD0C0144F06D04E4B221460C
:109088002846FFF7D4FC336820F060025B0103F048
:1090980060032EE628B9090141F06D0101F0FD01D8
:1090A80083E501287FF4CBAD0C0144F06D047BE728
:1090B80050B9090141F06D0101F0FD012846FFF7A3
:1090C800B6FCC0F30060B6E501287FF4B8AD0C012A
:1090D80044F06D04E4B221462846FFF7A8FC336843
:1090E80020F080721B0603F0807302E688B909013C
:1090F80041F06D0101F0FD012846FFF798FC0014CE
:1091080000F07F0310F0400018BF6FF07F00184395
:1091180091E501287FF493AD0C0144F06D04E4B2AD
:1091280021462846FFF783FC336820F4FE021B041F
:1091380003F4FE03DDE501287FF481AD0C0144F062
:109148006C04E4B221462846FFF771FC336820F42A
:1091580000325B0403F40033CBE500287FF404AE4F
:10916800090141F06F01C9B22846FFF760FCC0F35E
:10917800044060E501287FF462AD1968284616F0BE
:1091880083FC5CE550B9090141F06C0101F0FC0178
:109198002846FFF74CFCC0F340304CE501287FF42B
:1091A8004EAD0C0144F06C04E4B221462846FFF7AA
:1091B8003EFC336820F400525B0303F4005398E547
:1091C80000287FF4D1AD090141F06F01C9B22846EA
:1091D800FFF72DFCC0F309002DE507B50129019221
:1091E80007D8024601AB0120FFF777FC03B05DF812
:1091F80004FB0820FAE70129134602D8024600209A
:109208006BE40820704770B54E4E4F4816F084FF47
:10921800F5684E4C6B6803F1C802226103F59C7235
:10922800626203F5AA72226203F5C672A26003F5B0
:10923800D47203F5B870626003F5E27203F50D733A
:10924800A3622B68E260DB68206098472B68A068FF
:10925800DB6898472B686068DB6898472B68E0688C
:10926800DB6898472B682069DB6898472B68A06AF9
:10927800DB6898473369364A03F114011160A26A22
:10928800344D9A61344A354B1A6016F06BFC002352
:10929800A2682168184616F0B5FBE26861680023E9
:1092A800012016F0AFFB2E4B2E49D3F88020002466
:1092B800C2F804122C495470C2F808120121117026
:1092C8002A4A0220C3F88C20294A83F87C00C3F874
:1092D8008820284AC3F88420274AC3F89020274AC0
:1092E800C3F8A420264AC3F8A020264AC3F894202D
:1092F800254AC3F89820254AC3F8B420244AC3F85D
:10930800B020244AC3F8C020234AC3F8BC20234A0B
:10931800C3F8B820224AC3F8CC20224AC3F8C82090
:1093280032229A674FF48F725A671F4AC3F8C420D3
:10933800FFF7B0FA2B689847AB682046BDE8704045
:10934800184700BF649E0208403F00206C130020AD
:10935800C441002070090020FC0E0020C0410020FC
:10936800203E00205188000843880008278800080C
:10937800418800083D88000839880008FF910008E6
:10938800E39100081588000885890008318A0008DB
:10939800D58A0008DD870008378900081D8900087C
:1093A8009D880008D1870008DD880008014B104619
:1093B800DB6B184700000020034B10B51B6C1446EC
:1093C8009847206010BD00BF0000002007B5034B80
:1093D80068461B6B984703B05DF804FB000000204B
:1093E80070B50020FFF7F2FF1E4B1F4CDD68206BA5
:1093F8002B689B6898472B68E06A9B6898472B689E
:10940800E0689B6898472B68A0689B6898472B681A
:1094180060689B6898472B6820689B6898472B680A
:10942800A0699B6898472B68E0699B6898472B68F8
:10943800A06A9B6898472B6860699B6898472B6867
:10944800206A9B6898472B68606A9B6898472B68D6
:1094580020699B68984716F0D9FBBDE87040034B1C
:109468005B681847649E0208A41300207009002056
:10947800002016F053BA10B5044618B916F042FA8F
:10948800204610BD082010BD10B5044618B916F0C6
:109498002DFA204610BD082010BD0021F4E74942EE
:1094A800F2E7F1E7062873B505460C465DD80229B0
:1094B80003D901285BD10F2959DC2E4E6846336B3E
:1094C80098473346052D06D8DFE805F0030B4346D9
:1094D800494C8DF800406846DB6A9847002002B086
:1094E80070BD082CF7D8DFE804F0050C11161B2016
:1094F800252A2F00F2788DF80120327B8DF8022082
:10950800E9E732798DF80120727BF7E772798DF8F7
:109518000120B27BF2E7B2798DF80120F27BEDE70A
:10952800F2798DF80120327CE8E7727A8DF8012013
:10953800B27CE3E7B27A8DF80120F27CDEE7327A7A
:109548008DF80120727CD9E7F27A8DF80120327DFE
:10955800D4E78DF80340BEE78DF80440BBE78DF8EB
:109568000540B8E78DF80640B5E70420B7E71020B6
:10957800B5E700BF0000002073B504463F4D6846BC
:109588002B6B0E4698472B46062C1DD8DFE804F0B7
:10959800700464676A6D70009DF80120E978914253
:1095A80008D19DF80200297B884203D10020306051
:1095B80002B070BD1979914208D19DF80200597B1B
:1095C800884203D1012333600020F1E759799142A1
:1095D80006D19DF80200997B884201D10223F2E767
:1095E8009979914206D19DF80200D97B884201D130
:1095F8000323E8E7D979914206D19DF80200197C46
:10960800884201D10423DEE7597A914206D19DF8B8
:109618000200997C884201D10523D4E7997A9142C6
:1096280006D19DF80200D97C884201D10623CAE7F9
:10963800197A914206D19DF80200597C884201D1DD
:109648000723C0E7D97A914215D19DF802201B7DE6
:109658009A4210D10823B6E79DF80330B3E79DF886
:109668000430B0E79DF80530ADE79DF80630AAE76D
:109678009DF80030A7E710209AE700BF00000020FF
:1096880038B5154618B1012807D0042038BD08465A
:1096980016F098F92860002038BD094B094DDC68A0
:1096A800094B606800F5B870D8616B6C5861236825
:1096B800DB6898476A6C236850699B699847EAE7B2
:1096C800649E020800000020A413002038B50C4650
:1096D800054640B916F0E6F92368C1182160284606
:1096E800BDE83840C7E6082038BD30B585B0054626
:1096F80001920C46002961D10B2812D8062846D2BF
:10970800022837D004D848B301282CD004242EE0EE
:10971800042834D00528F9D11146204616F09DFAC0
:1097280025E013280ED80E2846D20C2836D00D284E
:10973800ECD142F210739A42E8D8214B90B29B6860
:10974800984714E08C28E1D101A90120FFF714FF04
:109758001C4B04469B6B02A8984708E0114616F07C
:10976800D1F82C4603E01146204616F075F920463C
:1097780005B030BD1146204616F0B8F8F7E782EA82
:10978800E271A1EBE271204616F074F9EFE70638B2
:109798001146C0B2FFF786FE0446E8E715460A4AB6
:1097A8000A4BD26812681DB15269D86A9047DEE741
:1097B8009269D86A9047D4E70E38E9E70824D6E7D3
:1097C8007009002000000020649E0208A4130020F5
:1097D80010B51446002947D1132847D8DFE800F010
:1097E8000A1014181C202424242424242C373E3E38
:1097F8003E3E3E3E002016F061F92060002010BD7C
:10980800002016F04FF9F8E7002016F073F9F4E796
:10981800002016F061F9F0E7002016F087F9ECE770
:10982800002016F075F9E8E708281FD1002016F087
:10983800C9F8C0F30010E0E70D4B0E4ADB68D06AA8
:109848001B681B6A9847003018BF0120D5E7084BF2
:10985800084ADB68106B1B681B6AF3E70E38114671
:10986800C0B2FFF789FEC9E7082010BD042010BD6B
:10987800649E0208A41300206C4B2DE9F041DE68B9
:109888006B4C7068002500F5FE73236300F5F073D8
:10989800E36200F52973E36000F53073A36000F517
:1098A8002273636000F50D73236000F55A73A3619A
:1098B80000F55373E36100F1C803A36200F5C673B2
:1098C800636100F56873236200F56F736362336840
:1098D80000F5B870DB682061984733686069DB6819
:1098E80098473368206BDB6898473368E06ADB6821
:1098F80098473368206A1B69984733684D4F1B693E
:10990800606A98477B6CE2681A60A2685A6062686D
:109918009A602268DA60A2691A61E2695A61A26AE9
:109928009A617A6C33685059DB6898477A6C336867
:1099380050599B69043598471C2DF2D14FF0000807
:109948003D4DD5F8803083F8008016F00BF943467A
:1099580062692169404616F055F844F62061404690
:1099680016F088F846F2A811404616F076F9334BFF
:109978000220C5F88C30324BC5F88830314BC5F819
:109988008430314BC5F89030304BC5F8A430304B9B
:10999800C5F8A0302F4BC5F894302F4BC5F8983038
:1099A8002E4BC5F8B4302E4BC5F8B0302D4BC5F84A
:1099B800BC302D4BC5F8C0302C4BC5F8CC3001233A
:1099C80085F87C302A4BC5F8C430FFF7FFFC4046C9
:1099D80016F082F810B1274B9B789BB1BB6A984769
:1099E80016F0C0F8002362691846216916F00AF8D3
:1099F80044F62061002016F03DF846F2A811002038
:109A080016F02BF90222236B197C5A74186801226C
:109A18001AF07EFF3368206B174C1B689847236841
:109A28009847A3680020BDE8F0411847649E0208E3
:109A3800A413002000000020203E0020919400087C
:109A4800AB940008A7940008A3940008D9970008CD
:109A5800F39600087F940008D5960008B59300088F
:109A6800C19300088996000879940008D5930008E6
:109A7800E9930008C0090020700900201B4B70B54D
:109A8800DD681B4C2B68A0685B6998472B682068C9
:109A98009B6898472B6860689B6898472B68206A82
:109AA8009B6898472B68606A9B6898472B68E068B2
:109AB8009B6898472B6820699B6898472B68606962
:109AC8009B6898472B68A0699B6898472B68E06952
:109AD8009B6898472B68A0689B68984716F096F88B
:109AE800BDE87040034B5B68184700BF649E0208DE
:109AF800E41300207009002010B51446052804D886
:109B0800DFE800F0052321343F44042010BD44F66B
:109B1800206314689C4243D842F21071214B224AB8
:109B2800DB688C421B68106ADB6994BF0021012145
:109B3800984742F21173B4FBF3F003FB10401B4B40
:109B480080B29B689847002010BD164B1468DB68EC
:109B580058681B682CB10021DB6900F5067098472E
:109B6800F1E79B6800F506709847ECE70D4B116824
:109B7800DB680D4A1B680031DB6918BF01211069D9
:109B8800EDE7084615F01EFF2060DCE7054B064AA6
:109B9800DB6858681B6800F5B8701061DB68E3E79C
:109BA800102010BD649E0208E413002070090020F4
:109BB80010B50348144616F03CFB206010BD00BFEA
:109BC800C8410020014816F026BB00BFC84100204C
:109BD80010B5044618B915F095FE204610BD0820AA
:109BE80010BD10B5044618B915F080FE204610BD0A
:109BF800082010BD0021F4E74942F2E7F1E70148E7
:109C080016F079BBC841002008B5002015F064FFA4
:109C180010B1084B987858B1074816F057FB15F063
:109C2800A1FF00230549184606C915F0EBFE0120DF
:109C380008BD00BFC0090020C8410020E41300206F
:109C4800022804BF0B4B93F8D80030B90A4BDB68E5
:109C58001B685B69094A90681847012809D1054BB8
:109C680093F8D830012B04D1034BDB681B689B6940
:109C7800F0E77047203E0020649E0208E4130020AD
:109C880038B50D46044620B915F026FF2860204651
:109C980038BD082038BD10B501460D4816F044FB04
:109CA800002015F03BFE002015F08CFE10F0080493
:109CB8000DD182060BD56F21054816F0BAFAC301FB
:109CC80005D52046BDE81040022115F053BE10BD51
:109CD800C8410020012903D1024A702116F09BBA1D
:109CE800704700BFC804050038B50C46054640B9A2
:109CF80015F0D8FE2368C11821602846BDE8384011
:109D080066E7082038BDA62A70B504460E461D46EB
:109D180000F0BA8200F28180172A00F0768130D8EC
:109D2800042A00F029810CD8012A00F00681C0F02D
:109D3800F480022A00F00D81032A00F01681042421
:109D4800F0E0072A00F045810ED8052A00F02381AB
:109D5800062AF4D1002840F02A811021BC4816F0C8
:109D680068FAC0F30420DCE0082A00F04681152ACE
:109D7800E5D10028E3D0012840F0D8801A681121E5
:109D880023E11D2A00F0AC811CD81A2A00F06A8150
:109D980009D8182AD3D1002840F05E813321AC4875
:109DA80016F047FABDE01B2A00F074811C2AC6D1C0
:109DB800002840F085810146A54816F03AFAC0F31C
:109DC8004000AEE0A32A00F0EA810ED88C2A00F009
:109DD8008E81A22AB3D1002840F0D3816C219C48FF
:109DE80016F027FAC0F3C1309BE0A42A00F0ED81F9
:109DF800A52AA4D1002840F00E826C21944816F0C0
:109E080018FA10F4804F4FF06C01914800F0F3817C
:109E180016F00FFAC0F3C31083E0B52A00F02B83C5
:109E28003CD8AB2A00F0C08214D8A82A00F07E8261
:109E3800C0F06782A92A00F09382AA2A7FF47FAF34
:109E4800002840F0A3826D21814816F0F2F9C0F392
:109E5800032066E0AE2A00F0DB820FD8AC2A00F0BF
:109E6800B982AD2A7FF46BAF002840F0C3826D2120
:109E7800774816F0DEF9C0F3006052E0B32A00F02C
:109E8800E482B42A7FF45BAF002840F02C816F2174
:109E98006F4816F0CEF9C0F3044042E0BB2A00F048
:109EA800498316D8B82A00F0058307D8B62A7FF464
:109EB80046AF002840F0EC821421A8E0B92A00F04F
:109EC8000F83BA2A7FF43BAF002840F02183132187
:109ED8009DE0C02A00F079830FD8BC2A00F04F8398
:109EE800BF2A7FF42CAF002840F05D8370215848CA
:109EF80016F09FF9C0F3014013E0CC2A00F07883F4
:109F0800CE2A7FF41CAF002840F0ED806F21504826
:109F180016F08FF9C0F3090003E028B9084615F0D8
:109F2800CDFD2860204670BD012801D00024F9E746
:109F38001968304615F0E6FCF8E718B9084615F038
:109F4800B1FDEEE70128F1D11968304615F084FD1E
:109F5800ECE718B9084615F0CDFDE2E70128E5D190
:109F68001968304615F0C2FCE0E7002840F0BB80D5
:109F7800084615F0B1FDD4E718B9084615F0D6FD26
:109F8800CFE70128D2D1196830460029B8BF494225
:109F980015F070FDCAE718B9084615F0B9FDC0E715
:109FA8000128C3D11968304615F057FEBEE70128CD
:109FB800BCD11021264816F03CF92B6820F4F85241
:109FC8001B0203F4F85310211A43214816F023F911
:109FD800ACE730B910211E4816F02BF900F01F002D
:109FE8009FE70128A2D11021194816F022F92B6801
:109FF80020F01F0203F01F03E5E7002873D108468D
:10A0080015F0E0FCC0F300108BE778B91521104873
:10A0180016F00FF90F4A002800F078824FF080738D
:10A0280093FBF0F09042A8BF1046EFE001287FF4C0
:10A038007DAF1968074B49B14FF0807292FBF1F27E
:10A048009A42A8BF1A462A601521BEE71A46FAE7BF
:10A05800C8410020FFFF0F0001287FF467AF1A688E
:10A068003321B2E730B96C21BC4816F0E2F8C0F3EE
:10A07800804056E701287FF459AF6C21B74816F0A5
:10A08800D8F82B6820F480229B0403F480231A4319
:10A098006C219AE730B96C21B04816F0CAF8C0F3C1
:10A0A800C0403EE701287FF441AF6C21AB4816F071
:10A0B800C0F82B6820F40022DB0403F40023E6E751
:10A0C80001287FF433AF0021A44816F0B2F82B68BA
:10A0D80020F002025B0003F002031A43002174E738
:10A0E80000283FF446AF012C3FF429AE1EE750B9D3
:10A0F8006C219A4816F09DF84FF48073C0F3036002
:10A1080043FA00F00DE701287FF410AF1B68102B0D
:10A1180023D00DDC022B1CD004DC012B16D04FF011
:10A12800FF3314E0042B16D0082BF8D105230EE0DA
:10A13800402B14D003DC202BF1D1032307E0802B24
:10A148000FD0B3F5807FEAD1002300E008232B600D
:10A1580008E00723FBE70623F9E70423F7E70223D0
:10A16800F5E728602B68013300F058826C217B48A2
:10A1780016F05FF82B6820F070621B0603F070631E
:10A1880085E701287FF4D2AE6C21744816F051F8A7
:10A198002B6820F4C032DB0303F4C03377E730B90F
:10A1A8006C216E4816F045F8C0F38030B9E60128F6
:10A1B8007FF4BCAE6C21694816F03BF82B6820F49C
:10A1C80080429B0303F4804361E730B96C21634804
:10A1D80016F02FF8C0F30030A3E601287FF4A6AEEE
:10A1E8006C215E4816F025F82B6820F480521B037A
:10A1F80003F480534BE716F01CF86C2106465748C9
:10A2080016F017F83205C0F3021001D428608DE665
:10A2180040F0080085E601287FF488AE6C214F489D
:10A2280016F007F810F480444FF06C014B4808D042
:10A2380015F0FFFF2B6820F4F062DB0103F4F063F4
:10A2480025E715F0F6FF6C21444815F0F2FF2B685E
:10A2580020F4006213F0080318BF4FF400636C2168
:10A268001A433E4815F0D7FF6C213C4815F0E1FF32
:10A278002B6820F070021B0103F070031A436C2155
:10A28800364815F0C8FF4DE6E0B96C21334815F0A3
:10A29800D0FF10F480464FF06C01304804D015F020
:10A2A800C8FFC0F302103CE615F0C3FF6C2104465A
:10A2B8002A4815F0BEFF2305C0F3C31048BF40F07D
:10A2C8000800A3E701287FF431AE6C21234815F07C
:10A2D800B0FF10F480444FF06C01204808D015F00E
:10A2E800A8FF2B6820F070021B0103F07003CEE674
:10A2F80015F09FFF2B6820F4F062DB0103F4F06394
:10A30800BCE730B96C21154815F093FF00F00F0039
:10A3180007E601287FF40AAE6C21104815F089FF82
:10A328002B6820F00F0203F00F03B0E630B96D215F
:10A338000A4815F07EFFC0F3C030F2E501287FF42B
:10A34800F5AD6D21054815F074FF2B6820F4004227
:10A35800DB039BB21A436D2137E600BFC8410020DA
:10A3680030B96D21AE4815F064FFC0F34130D8E52F
:10A3780001287FF4DBAD6D21A94815F05AFF2B6841
:10A3880020F4C0425B0303F4C043E3E701287FF4F1
:10A39800CDAD6D21A24815F04CFF2B6820F47062FA
:10A3A8001B0203F47063D5E730B96D219C4815F0A2
:10A3B80040FFC0F34110B4E501287FF4B7AD6D212B
:10A3C800974815F036FF2B6820F060025B0103F018
:10A3D8006003BFE708B96D2195E701287FF4A6ADB2
:10A3E8006D218F4815F025FF2B6820F00F0203F030
:10A3F8000F03AFE701287FF499AD6D21884815F068
:10A4080018FF2B6820F080721B0603F08073A1E709
:10A4180068B96D21824815F00CFF001400F07F0325
:10A4280010F0400018BF6FF07F00184379E501284D
:10A438007FF47CAD6D217A4815F0FBFE2B6820F483
:10A44800FE021B0403F4FE0384E730B96C21744850
:10A4580015F0EFFEC0F3404063E501287FF466ADD8
:10A468006C216F4815F0E5FE2B6820F400325B0480
:10A4780003F400330BE618B9084615F065FB50E500
:10A4880001287FF453AD1968304615F0FDFA4DE503
:10A4980001287FF44BAD1968624B49B14FF08072C7
:10A4A80092FBF1F29A42A8BF1A462A6014218CE561
:10A4B8001A46FAE730B96C21594815F0BAFEC0F3CC
:10A4C80040302EE501287FF431AD6C21544815F059
:10A4D800B0FE2B6820F400525B0303F40053D6E56A
:10A4E80030B96C214E4815F0A4FEC0F3035018E5AE
:10A4F80001287FF41BAD6C21494815F09AFE2B68A2
:10A5080020F470021B0503F47003C0E510467DE6D5
:10A5180001287FF40BAD1968424B49B14FF08072A6
:10A5280092FBF1F29A42A8BF1A462A6013214CE521
:10A538001A46FAE730B97021394815F07AFEC0F3A7
:10A548000720EEE401287FF4F1AC7021344815F0BF
:10A5580070FE2A6820F47F40120292B202437021F2
:10A568002F4815F058FE00212D4815F062FE2B6883
:10A5780020F00402002BCCBF04230023ADE528B94A
:10A588007021274815F055FEC0B2CAE401287FF4AF
:10A59800CDAC7021224815F04CFE2A7820F0FF003F
:10A5A8000243702111E501287FF4C0AC1B68032B1E
:10A5B80034D870211A4815F03CFE2B6820F440323C
:10A5C8001B0403F440331A43EBE708B970214BE549
:10A5D80001287FF4ABAC7021114815F02AFE2B68D6
:10A5E80020F48022002B14BF4FF480230023EAE7D5
:10A5F80030B970210A4815F01CFEC0F3015090E4F0
:10A6080001287FF493AC7021054815F012FE2B68E1
:10A6180020F440121B0503F44013D4E7102481E40E
:10A62800C8410020FFFF0F0007B5019239B9024663
:10A6380001AB0120FFF767FB03B05DF804FB0820BE
:10A64800FAE710B413460446084619B9224610BC66
:10A65800FFF759BB082010BC7047064B08469B6A99
:10A66800114613B1044B9B6E1847044B1B68DB68FB
:10A67800FAE700BFE4130020203E00204C440020ED
:10A688002DE9F041674D684BD5F8802001216748D6
:10A69800674F15F0FFFD6749644815F041FEFE68F5
:10A6A800654C736803F1C802A26003F5B8722260B2
:10A6B80003F5C672626003F5F072226203F5FE725A
:10A6C800626203F55372E26003F55A7203F568702B
:10A6D800226103F5617203F56F73E36133686261A8
:10A6E8001B69A06198473368E0691B69984733681C
:10A6F80060691B69984733682068DB689847336846
:10A708006068DB6898473368A068DB6898473368F7
:10A718002069DB6898473368E068DB6898473368E6
:10A72800606ADB6898473368206ADB689847336853
:10A73800606A9B6998473368206A9B6998473368C1
:10A7480060699B6998473368E0689B6998473A69EC
:10A758003A4B02F114011960736803F50D739361A4
:10A7680015F000FA94E806000023184615F04AF997
:10A77800D5F88030324A0021C3F80422314A597092
:10A78800C3F8082201221A702F4B85F87C20C5F8DF
:10A798008C302E4BC5F888302D4BC5F884302D4BA6
:10A7A800C5F890302C4BC5F8A4302C4BC5F8A03018
:10A7B8002B4BC5F894302B4BC5F898302A4BC5F86D
:10A7C800B4302A4BC5F8B030294BC5F8C030294BF6
:10A7D800C5F8BC30284BC5F8B830284BC5F8CC3084
:10A7E8003223AB674FF4F0736B67254BC5F8C43061
:10A7F800AB6E03B1A2620220FFF722FA0222636A5B
:10A80800197C5A74186801221AF082F83368606A51
:10A818001C4C1B68984723689847A3680020BDE82C
:10A82800F0411847203E00205C8E0208C8410020F5
:10A83800649E0208DD9C0008E41300204C440020BC
:10A84800119C0008079C0008EB9B0008059C000869
:10A85800019C0008FD9B00084BA6000831A60008D3
:10A86800D99B0008F19C0008CD9B0008B99B000803
:10A878009F9C0008019B0008899C0008499C0008CF
:10A88800859A000870090020194B70B5DD68194CCD
:10A898002B6820685B6998472B6860689B689847B5
:10A8A8002B68A0689B6898472B68E0689B68984766
:10A8B8002B6820699B6898472B6860699B68984754
:10A8C8002B68A0699B6898472B68E0699B68984744
:10A8D8002B68206A9B6898472B6820689B68984774
:10A8E80015F094F9BDE87040034B5B68184700BF4A
:10A8F800649E02081C1400207009002010B514463C
:10A90800052804D8DFE800F005161427323704209C
:10A9180010BD136844F62062934236D842F2117291
:10A92800B3FBF2F002FB1030194B80B29B689847DA
:10A93800002010BD174B1468DB6858681B682CB1E1
:10A948000021DB6900F506709847F1E79B6800F580
:10A9580006709847ECE70F4B1168DB680E4A1B68D6
:10A968000031DB6918BF01215069EDE7084615F091
:10A9780029F82060DCE7074B074ADB6858681B6842
:10A9880000F5B8705061DB68E3E7102010BD00BF28
:10A9980070090020649E02081C14002010B50348AA
:10A9A800144615F040FD206010BD00BF544400203F
:10A9B800014815F02ABD00BF5444002010B50446D4
:10A9C80018B914F09FFF204610BD082010BD10B51F
:10A9D800044618B914F08AFF204610BD082010BD9F
:10A9E8000021F4E74942F2E7F1E7014815F07DBD9F
:10A9F8005444002008B5002015F06EF810B1084B3B
:10AA0800987860B1074815F05BFD15F0ABF80023A6
:10AA1800054918468A68496814F0F4FF012008BD02
:10AA2800C0090020544400201C140020022804BF40
:10AA38000B4B93F8D80030B90A4BDB681B685B698D
:10AA4800094A10681847012809D1054B93F8D830EE
:10AA5800012B04D1034BDB681B689B69F0E7704747
:10AA6800203E0020649E02081C14002038B50D46C4
:10AA7800044620B915F030F82860204638BD082073
:10AA880038BD10B501460D4815F048FD002014F0FA
:10AA980045FF002014F096FF10F008040DD182063F
:10AAA8000BD56F21054815F0BEFCC30105D520461E
:10AAB800BDE81040022114F05DBF10BD54440020D1
:10AAC800012903D1024A702115F09FBC704700BFCD
:10AAD8001E000CC438B50C46054640B914F0E2FF18
:10AAE8002368C11821602846BDE8384066E7082079
:10AAF80038BDA62A70B504460E461D4600F0BA8237
:10AB080000F28180172A00F0768130D8042A00F0FC
:10AB180029810CD8012A00F00681C0F0F480022AAD
:10AB280000F00D81032A00F016810424F0E0072AC2
:10AB380000F045810ED8052A00F02381062AF4D1B9
:10AB4800002840F02A811021BC4815F06CFCC0F3A5
:10AB58000420DCE0082A00F04681152AE5D1002807
:10AB6800E3D0012840F0D8801A68112123E11D2A7A
:10AB780000F0AC811CD81A2A00F06A8109D8182A7A
:10AB8800D3D1002840F05E813321AC4815F04BFC4E
:10AB9800BDE01B2A00F074811C2AC6D1002840F0B1
:10ABA80085810146A54815F03EFCC0F34000AEE0A3
:10ABB800A32A00F0EA810ED88C2A00F08E81A22AFE
:10ABC800B3D1002840F0D3816C219C4815F02BFCB0
:10ABD800C0F3C1309BE0A42A00F0ED81A52AA4D1DE
:10ABE800002840F00E826C21944815F01CFC10F4EB
:10ABF800804F4FF06C01914800F0F38115F013FC81
:10AC0800C0F3C31083E0B52A00F02B833CD8AB2AED
:10AC180000F0C08214D8A82A00F07E82C0F06782B3
:10AC2800A92A00F09382AA2A7FF47FAF002840F077
:10AC3800A3826D21814815F0F6FBC0F3032066E07E
:10AC4800AE2A00F0DB820FD8AC2A00F0B982AD2A18
:10AC58007FF46BAF002840F0C3826D21774815F070
:10AC6800E2FBC0F3006052E0B32A00F0E482B42AA9
:10AC78007FF45BAF002840F02C816F216F4815F0FE
:10AC8800D2FBC0F3044042E0BB2A00F0498316D847
:10AC9800B82A00F0058307D8B62A7FF446AF002803
:10ACA80040F0EC821421A8E0B92A00F00F83BA2AF8
:10ACB8007FF43BAF002840F0218313219DE0C02A98
:10ACC80000F079830FD8BC2A00F04F83BF2A7FF4A5
:10ACD8002CAF002840F05D837021584815F0A3FB85
:10ACE800C0F3014013E0CC2A00F07883CE2A7FF429
:10ACF8001CAF002840F0ED806F21504815F093FB01
:10AD0800C0F3090003E028B9084614F0D7FE28600C
:10AD1800204670BD012801D00024F9E719683046A3
:10AD280014F0F0FDF8E718B9084614F0BBFEEEE79A
:10AD38000128F1D11968304614F08EFEECE718B9F5
:10AD4800084614F0D7FEE2E70128E5D11968304635
:10AD580014F0CCFDE0E7002840F0BB80084614F072
:10AD6800BBFED4E718B9084614F0E0FECFE7012887
:10AD7800D2D1196830460029B8BF494214F07AFE8A
:10AD8800CAE718B9084614F0C3FEC0E70128C3D1C2
:10AD98001968304614F061FFBEE70128BCD11021C4
:10ADA800264815F040FB2B6820F4F8521B0203F4E8
:10ADB800F85310211A43214815F027FBACE730B9A6
:10ADC80010211E4815F02FFB00F01F009FE70128F7
:10ADD800A2D11021194815F026FB2B6820F01F027C
:10ADE80003F01F03E5E7002873D1084614F0EAFDD5
:10ADF800C0F300108BE778B91521104815F013FB44
:10AE08000F4A002800F078824FF0807393FBF0F02F
:10AE18009042A8BF1046EFE001287FF47DAF196883
:10AE2800074B49B14FF0807292FBF1F29A42A8BFEA
:10AE38001A462A601521BEE71A46FAE7544400204C
:10AE4800FFFF0F0001287FF467AF1A683321B2E7CC
:10AE580030B96C21BC4815F0E6FAC0F3804056E7DB
:10AE680001287FF459AF6C21B74815F0DCFA2B683C
:10AE780020F480229B0403F480231A436C219AE770
:10AE880030B96C21B04815F0CEFAC0F3C0403EE7A7
:10AE980001287FF441AF6C21AB4815F0C4FA2B6848
:10AEA80020F40022DB0403F40023E6E701287FF402
:10AEB80033AF0021A44815F0B6FA2B6820F002023F
:10AEC8005B0003F002031A43002174E700283FF4F3
:10AED80046AF012C3FF429AE1EE750B96C219A48C1
:10AEE80015F0A1FA4FF48073C0F3036043FA00F041
:10AEF8000DE701287FF410AF1B68102B23D00DDC61
:10AF0800022B1CD004DC012B16D04FF0FF3314E0C9
:10AF1800042B16D0082BF8D105230EE0402B14D0B3
:10AF280003DC202BF1D1032307E0802B0FD0B3F5EE
:10AF3800807FEAD1002300E008232B6008E0072384
:10AF4800FBE70623F9E70423F7E70223F5E7286080
:10AF58002B68013300F058826C217B4815F063FAA6
:10AF68002B6820F070621B0603F0706385E70128E8
:10AF78007FF4D2AE6C21744815F055FA2B6820F492
:10AF8800C032DB0303F4C03377E730B96C216E4875
:10AF980015F049FAC0F38030B9E601287FF4BCAE59
:10AFA8006C21694815F03FFA2B6820F480429B0316
:10AFB80003F4804361E730B96C21634815F033FA34
:10AFC800C0F30030A3E601287FF4A6AE6C215E48EA
:10AFD80015F029FA2B6820F480521B0303F48053E0
:10AFE8004BE715F020FA6C210646574815F01BFA76
:10AFF8003205C0F3021001D428608DE640F0080045
:10B0080085E601287FF488AE6C214F4815F00BFACD
:10B0180010F480444FF06C014B4808D015F003FA47
:10B028002B6820F4F062DB0103F4F06325E715F0E8
:10B03800FAF96C21444815F0F6F92B6820F40062FF
:10B0480013F0080318BF4FF400636C211A433E48FD
:10B0580015F0DBF96C213C4815F0E5F92B6820F078
:10B0680070021B0103F070031A436C21364815F077
:10B07800CCF94DE6E0B96C21334815F0D4F910F459
:10B0880080464FF06C01304804D015F0CCF9C0F37D
:10B0980002103CE615F0C7F96C2104462A4815F061
:10B0A800C2F92305C0F3C31048BF40F00800A3E766
:10B0B80001287FF431AE6C21234815F0B4F910F45F
:10B0C80080444FF06C01204808D015F0ACF92B688B
:10B0D80020F070021B0103F07003CEE615F0A3F90F
:10B0E8002B6820F4F062DB0103F4F063BCE730B9AD
:10B0F8006C21154815F097F900F00F0007E60128B4
:10B108007FF40AAE6C21104815F08DF92B6820F0F9
:10B118000F0203F00F03B0E630B96D210A4815F0AD
:10B1280082F9C0F3C030F2E501287FF4F5AD6D2156
:10B13800054815F078F92B6820F40042DB039BB230
:10B148001A436D2137E600BF5444002030B96D2101
:10B15800AE4815F068F9C0F34130D8E501287FF40E
:10B16800DBAD6D21A94815F05EF92B6820F4C042CB
:10B178005B0303F4C043E3E701287FF4CDAD6D2101
:10B18800A24815F050F92B6820F470621B0203F4F2
:10B198007063D5E730B96D219C4815F044F9C0F3C8
:10B1A8004110B4E501287FF4B7AD6D21974815F03B
:10B1B8003AF92B6820F060025B0103F06003BFE7F7
:10B1C80008B96D2195E701287FF4A6AD6D218F4858
:10B1D80015F029F92B6820F00F0203F00F03AFE7F1
:10B1E80001287FF499AD6D21884815F01CF92B686A
:10B1F80020F080721B0603F08073A1E768B96D2107
:10B20800824815F010F9001400F07F0310F0400098
:10B2180018BF6FF07F00184379E501287FF47CADF3
:10B228006D217A4815F0FFF82B6820F4FE021B0404
:10B2380003F4FE0384E730B96C21744815F0F3F881
:10B24800C0F3404063E501287FF466AD6C216F4888
:10B2580015F0E9F82B6820F400325B0403F400339E
:10B268000BE618B9084614F06FFC50E501287FF486
:10B2780053AD1968304614F007FC4DE501287FF4FA
:10B288004BAD1968624B49B14FF0807292FBF1F2F5
:10B298009A42A8BF1A462A6014218CE51A46FAE792
:10B2A80030B96C21594815F0BEF8C0F340302EE58E
:10B2B80001287FF431AD6C21544815F0B4F82B689F
:10B2C80020F400525B0303F40053D6E530B96C2137
:10B2D8004E4815F0A8F8C0F3035018E501287FF48C
:10B2E8001BAD6C21494815F09EF82B6820F47002BC
:10B2F8001B0503F47003C0E510467DE601287FF4C2
:10B308000BAD1968424B49B14FF0807292FBF1F2D4
:10B318009A42A8BF1A462A6013214CE51A46FAE752
:10B3280030B97021394815F07EF8C0F30720EEE4F3
:10B3380001287FF4F1AC7021344815F074F82A68BC
:10B3480020F47F40120292B2024370212F4815F078
:10B358005CF800212D4815F066F82B6820F00402EF
:10B36800002BCCBF04230023ADE528B97021274862
:10B3780015F059F8C0B2CAE401287FF4CDAC7021A9
:10B38800224815F050F82A7820F0FF000243702177
:10B3980011E501287FF4C0AC1B68032B34D8702159
:10B3A8001A4815F040F82B6820F440321B0403F4C7
:10B3B80040331A43EBE708B970214BE501287FF4C5
:10B3C800ABAC7021114815F02EF82B6820F48022C0
:10B3D800002B14BF4FF480230023EAE730B9702113
:10B3E8000A4815F020F8C0F3015090E401287FF4D2
:10B3F80093AC7021054815F016F82B6820F440121C
:10B408001B0503F44013D4E7102481E454440020BE
:10B41800FFFF0F0007B5019239B9024601AB0120C1
:10B42800FFF767FB03B05DF804FB0820FAE710B4E8
:10B4380013460446084619B9224610BCFFF759BB03
:10B44800082010BC7047064B08465B6A114613B1CA
:10B45800044B9B6E1847044B1B68DB68FAE700BF78
:10B468001C140020203E0020504400202DE9F0410B
:10B47800624D634BD5F8802001216248624F15F078
:10B4880003F862495F4815F045F8FE68604C736838
:10B4980003F1C802226003F5B872626003F5C67250
:10B4A800A26003F5FE72E26003F55372226103F5B0
:10B4B8005A7203F56870626103F5617203F56F7380
:10B4C80023623368A2611B69E06198473368206A88
:10B4D8001B6998473368A0691B69984733682068D7
:10B4E800DB68984733686068DB6898473368A0680A
:10B4F800DB6898473368E068DB68984733686069B9
:10B50800DB68984733682069DB6898473368E068E8
:10B518005B6998473368A0699B69984733682069D5
:10B528009B6998477068336800F50670DB68984730
:10B538007068336800F506709B6998473A69354B1F
:10B5480002F114011960736803F50D73936114F027
:10B5580009FB0023A2686168184614F053FAD5F86D
:10B5680080302D4A0021C3F804222C4A5970C3F8B0
:10B57800082201221A702A4B85F87C20C5F88C30E5
:10B58800284BC5F88830284BC5F88430274BC5F8B8
:10B598009030274BC5F8A430264BC5F8A030264B71
:10B5A800C5F89430254BC5F89830254BC5F8B4300C
:10B5B800244BC5F8B030244BC5F8C030234BC5F830
:10B5C800BC30234BC5F8B830224BC5F8CC303223F9
:10B5D800AB674FF4F0736B671F4BC5F8C430AB6EA5
:10B5E80003B162621D4C0220FFF720FA23689847D6
:10B5F800A3680020BDE8F041184700BF203E0020A6
:10B608005C90020854440020649E0208C9AA0008FD
:10B618001C14002050440020FDA90008F3A90008CC
:10B62800D7A90008F1A90008EDA90008E9A90008B0
:10B6380037B400081DB40008C5A90008DDAA000831
:10B64800B9A90008A5A900088BAA000805A900083F
:10B6580075AA000835AA000891A8000870090020FA
:10B668000022014B1A677047203E00200523F7B5DA
:10B6780000248DF8003061F07F038DF80230131636
:10B688008DF8033013148DF804308DF8062013124A
:10B698000E4615460721012268468DF805308DF8BB
:10B6A800014014F019FC0D4F8DF807003B689B69A9
:10B6B80098473B681DF804009B6801349847082C9C
:10B6C800F7D1022011F002FA054B26F080061B681C
:10B6D80003EB8606756003B0F0BD00BFDC460020B2
:10B6E800D8460020F0B5314B01F07F06334493F87B
:10B6F8000C3285B0DB07154606D42D4B1B6803EBCF
:10B70800860673682B604FE005238DF8043000230C
:10B718000122032101A88DF805308DF8066014F088
:10B72800DBFB244C8DF8070023689B6998470421AC
:10B7380023680DEB01001B69984711F0C1F9074612
:10B748002368DB699847072829D9082123680DEB66
:10B7580001005B6998470122072102A89DF80F4064
:10B7680014F0BAFB84421FD19DF80830052B1BD179
:10B778009DF80930FF2B17D19DF80A30B34213D139
:10B788009DF80C309DF80B201B0443EA02639DF8DA
:10B798000E2013439DF80D2043EA0223B2E73846F2
:10B7A80011F09EF90A28CBD905B0F0BDE04600207B
:10B7B800D8460020DC46002008B5064B01461B6829
:10B7C8000020054A14F01FFFBDE80840002014F0CF
:10B7D800A5B800BFD8460020E046002038B5154679
:10B7E800044628B9084614F0EDF82860204638BD0C
:10B7F800042038BD10B5044618B914F083F8204663
:10B8080010BD082010BD10B5044618B914F06EF824
:10B81800204610BD082010BD0021F4E74942F2E798
:10B82800F1E7024B186814F006BF00BFD8460020A5
:10B8380008B514F097F90023054918468A6849683D
:10B8480014F0E0F8034B1868BDE8084014F0EABEAD
:10B8580050140020D8460020022804BF0B4B93F850
:10B86800D80030B90A4BDB681B685B69094A106865
:10B878001847012809D1054B93F8D830012B04D17A
:10B88800034BDB681B689B69F0E77047203E00208C
:10B89800649E02085014002038B50020FFF7DCFF32
:10B8A800114B124CDD6820682B689B6898472B6801
:10B8B80060689B6898472B68A0689B6898472B68C6
:10B8C800E0689B6898472B6820699B6898472B68B5
:10B8D80060699B6898472B68A0699B689847BDE892
:10B8E800384014F093B900BF649E02085014002039
:10B8F80038B50C46054640B914F0D4F82368C11889
:10B9080021602846BDE8384074E7082038BD08B5EE
:10B9180019BB052823D8DFE800F003090E22131B02
:10B928001146002013F0EEFF002008BD114600204C
:10B9380014F092F8F8E71146002013F0D7FFF3E768
:10B9480082EAE271A1EBE271002014F093F8EBE7D0
:10B958001146002014F081F9E6E7082008BD04200C
:10B9680008BD10B5144601BB052820D8DFE800F053
:10B9780003090D111519002014F0A0F8206000200B
:10B9880010BD002014F08EF8F8E7002014F0B2F88B
:10B99800F4E7002014F0A0F8F0E7002014F0C6F84F
:10B9A800ECE7002014F0B4F8E8E7082010BD042004
:10B9B80010BD5BE696E6012270B511464B4E072096
:10B9C80014F02CFA4A4814F0E7FDF568494C6B6806
:10B9D80003F5B872626003F5C672A26003F58E7251
:10B9E800E26003F59C7203F1C800226103F1E402EE
:10B9F80003F58073A3612B686261DB682060984758
:10BA08002B686068DB6898472B68A068DB689847F4
:10BA18002B68E068DB6898472B682069DB689847E3
:10BA28002B6860691B6998472B68A0691B69984750
:10BA3800F56A01262B6898472F4B30491D60002571
:10BA48002F4BD3F880200A602E491670C2F80412D2
:10BA58002D495570C2F808122C4A83F87C60C3F847
:10BA68008C202B4AC3F888202A4AC3F884202A4A03
:10BA7800C3F89020294AC3F8A420294AC3F8A02073
:10BA8800284AC3F89420284AC3F89820274AC3F8BC
:10BA9800B420274AC3F8B020264AC3F8BC20264A57
:10BAA800C3F8CC20254AC3F8C82032229A674FF43D
:10BAB800C3725A67224AC3F8C420224AC3F8C02076
:10BAC80014F050F82B46A2686168284613F09AFFD4
:10BAD80028464FF4484113F0CDFF28464FF448411B
:10BAE80014F0BBF83046BDE87040B5E6649E020825
:10BAF800E046002050140020DC460020D8460020F4
:10BB0800203E002039B800082BB800080FB80008FC
:10BB180029B8000825B8000821B800086BB9000842
:10BB280017B90008FDB70008F9B8000875B600088D
:10BB3800EDB60008E5B7000861B8000869B6000866
:10BB4800A1B80008C1B700080022014B1A67704766
:10BB5800203E00200523F7B500248DF8003061F061
:10BB68007F038DF8023013168DF8033013148DF807
:10BB780004308DF8062013120E46154607210122BF
:10BB880068468DF805308DF8014014F0A5F90D4F81
:10BB98008DF807003B689B6998473B681DF80400CF
:10BBA8009B6801349847082CF7D1022010F08EFFCB
:10BBB800054B26F080061B6803EB8606756003B00C
:10BBC800F0BD00BFFC4B0020004C0020F0B5314B0D
:10BBD80001F07F06334493F80C3285B0DB07154635
:10BBE80006D42D4B1B6803EB860673682B604FE069
:10BBF80005238DF8043000230122032101A88DF8C4
:10BC080005308DF8066014F067F9244C8DF80700AC
:10BC180023689B699847042123680DEB01001B6981
:10BC2800984710F04DFF07462368DB6998470728B7
:10BC380029D9082123680DEB01005B699847012287
:10BC4800072102A89DF80F4014F046F984421FD13D
:10BC58009DF80830052B1BD19DF80930FF2B17D113
:10BC68009DF80A30B34213D19DF80C309DF80B2093
:10BC78001B0443EA02639DF80E2013439DF80D2030
:10BC880043EA0223B2E7384610F02AFF1428CBD93A
:10BC980005B0F0BD6C490020004C0020FC4B002092
:10BCA80008B5064B01461B680020054A14F005FD3F
:10BCB800BDE80840002013F031BE00BF004C002052
:10BCC8006C49002038B51546044628B9084613F0D3
:10BCD80079FE2860204638BD042038BD10B50446DA
:10BCE80018B913F00FFE204610BD082010BD10B57E
:10BCF800044618B913F0FAFD204610BD082010BDFF
:10BD08000021F4E74942F2E7F1E7024B186814F022
:10BD1800ECBC00BF004C002008B513F023FF002343
:10BD2800054918468A68496813F06CFE034B186881
:10BD3800BDE8084014F0D0BC78140020004C002066
:10BD4800022804BF0B4B93F8D80030B90A4BDB68C4
:10BD58001B685B69094A10681847012809D1054B17
:10BD680093F8D830012B04D1034BDB681B689B691F
:10BD7800F0E77047203E0020649E020878140020F7
:10BD880070B5144E0020FFF7DBFFF568124C2B68E6
:10BD980020689B6898472B6860689B6898472B6861
:10BDA800A0689B6898472B68E0689B6898472B6851
:10BDB80020699B6898472B6860699B6898472B683F
:10BDC800A0699B689847F36A5B689847BDE870402C
:10BDD80013F01CBF649E02087814002038B50C4686
:10BDE800054640B913F05EFE2368C1182160284655
:10BDF800BDE8384072E7082038BD08B519BB0528EA
:10BE080023D8DFE800F003090E22131B1146002097
:10BE180013F078FD002008BD1146002013F01CFE29
:10BE2800F8E71146002013F061FDF3E782EAE271BA
:10BE3800A1EBE271002013F01DFEEBE71146002094
:10BE480013F00BFFE6E7082008BD042008BD10B575
:10BE5800144601BB052820D8DFE800F003090D11BE
:10BE68001519002013F02AFE2060002010BD0020C4
:10BE780013F018FEF8E7002013F03CFEF4E700206A
:10BE880013F02AFEF0E7002013F050FEECE7002044
:10BE980013F03EFEE8E7082010BD042010BD59E667
:10BEA80094E6012270B511464B4E072013F0B6FFF9
:10BEB8004A4814F0C9FBF568494C6B6803F5B87239
:10BEC800626003F5C672A26003F58E72E26003F544
:10BED8009C7203F1C800226103F1E40203F5807348
:10BEE800A3612B686261DB68206098472B686068F3
:10BEF800DB6898472B68A068DB6898472B68E06880
:10BF0800DB6898472B682069DB6898472B6860696D
:10BF18001B6998472B68A0691B699847F56A012631
:10BF28002B6898472F4B30491D6000252F4BD3F8BD
:10BF380080200A602E491670C2F804122D495570E7
:10BF4800C2F808122C4A83F87C60C3F88C202B4A6C
:10BF5800C3F888202A4AC3F884202A4AC3F89020C4
:10BF6800294AC3F8A420294AC3F8A020284AC3F8BC
:10BF78009420284AC3F89820274AC3F8B420274AAF
:10BF8800C3F8B020264AC3F8BC20264AC3F8CC2000
:10BF9800254AC3F8C82032229A674FF4C3725A67F9
:10BFA800224AC3F8C420224AC3F8C02013F0DAFD9D
:10BFB8002B46A2686168284613F024FD28464FF4F2
:10BFC800484113F057FD28464FF4484113F045FE09
:10BFD8003046BDE87040B3E6649E02086C49002014
:10BFE80078140020FC4B0020004C0020203E00204C
:10BFF80021BD000813BD0008F7BC000811BD0008EA
:10C008000DBD000809BD000857BE000803BE0008A2
:10C01800E5BC0008E5BD00085DBB0008D5BB00080D
:10C02800CDBC000849BD000851BB000889BD000807
:10C03800A9BC0008012810B514460CD003D3022867
:10C0480010D0042010BD1368094AB3FA83F35B09C2
:10C058009372002010BD1368064AB3FA83F35B0994
:10C068001360F6E7084613F0ADFC2060F1E700BF67
:10C07800044C00206400002010B5044618B913F0E1
:10C0880041FC204610BD082010BD024B186814F072
:10C09800CABB00BF504C0020022804BF0B4B93F8CA
:10C0A800D80030B90A4BDB681B685B69094AD0685D
:10C0B8001847012809D1054B93F8D830012B04D132
:10C0C800034BDB681B689B69F0E77047203E002044
:10C0D800649E0208A014002038B50020FFF7DCFF9A
:10C0E8000F4B104CDD68E0682B685B6998472B683C
:10C0F80020689B6898472B68A0689B6898472B68BE
:10C10800E0689B6898472B6820699B6898472B686C
:10C1180060689B689847BDE8384013F077BD00BF5A
:10C12800649E0208A014002038B50D46044620B9C4
:10C1380013F0D2FC2860204638BD082038BD38B539
:10C148000C46054640B913F0ADFC2368C1182160C0
:10C158002846BDE838408FE7082038BD10B50446AA
:10C1680030B9044B5872187213F0C0FB204610BD4A
:10C17800082010BD044C00200021EFE74942EDE7FC
:10C18800ECE738B5002013F0A7FC0546A8B9012450
:10C198000B4B0C48196814F029FB0B4B02201C6050
:10C1A800FFF77AFF13F0DEFC084928460B698A6816
:10C1B800496813F027FC204638BD002038BD00BF71
:10C1C800504C0020044C002064000020A0140020E3
:10C1D8002DE9F843830C04460DD0C0F34243062BE7
:10C1E80009D1294B20F01F045A7A002A43D01B7822
:10C1F80003F01F031C43254F254E3B68254D9B68C4
:10C208000021C4F30740D6F8008095F818909847A5
:10C218002A7E336808EB8908C8F8040003EB820318
:10C228005A68002112025A603B68C4F307209B68D1
:10C2380098472B7E3268012102EB8302536818432A
:10C248003B68000250609B68E0B298473268297EDC
:10C2580002EB81014B6818430011A30C4860106180
:10C268000BD0C4F34243072B02D1C4F30111297642
:10C2780043F0080302E0DB7ABAE7082302EB830302
:10C288005C60BDE8F88300BF044C00204C4C0020E3
:10C29800504C0020A01400200D4B00F077021B68C2
:10C2A80030B406280B4D42F00802C1F3130403EB27
:10C2B800820304BF01F01F01E9725C60AB7A23B905
:10C2C80044EA404030BCFFF783BF30BC704700BF32
:10C2D800504C0020044C002008461146DCE738B5D5
:10C2E80004460F2000F014F80323B4FBF3F30546CB
:10C2F80003EB4303E41A240104F0300420F0300077
:10C308002043FFF765FF2846BDE83840FFF760BFC8
:10C3180010B5084B04469B7A1BB9030701D4FFF7F5
:10C32800DEFF054B04F07F041B6803EB84046068A0
:10C3380010BD00BF044C0020504C0020A82A38B57E
:10C3480004461D46084600F0F0815CD81D2A00F01E
:10C35800D68022D8042A00F0DB800CD8012A00F00D
:10C36800BA80C0F0AA80022A00F0BF80032A00F039
:10C37800C6800424A5E0062A00F0E180C0F0D5803C
:10C38800072A00F0F280082AF3D1002C40F0BC8084
:10C3980013F018FBC0F3001092E0A32A00F06981A3
:10C3A8001ED8A02A00F02E810CD88C2AE1D1002CAE
:10C3B80040F0EB800820FFF7ABFF00F00F00C0F162
:10C3C80008007DE0A12A00F03181A22AD1D1002CF9
:10C3D80040F040810C20FFF79BFFC0F3C1306FE0B5
:10C3E800A52A00F06E81C0F05881A62A00F07D8150
:10C3F800A72ABED1002C40F08C810C20FFF788FFC3
:10C4080000F00F005CE0B22A00F0558225D8AD2A72
:10C4180000F0EA810ED8AA2A00F0B281C0F09C810F
:10C42800AB2A00F0C181AC2AA3D1002C40F0D08106
:10C438000520E3E7AF2A00F00882C0F0EB81B02ABC
:10C4480000F01882B12A94D1002C40F027820720EE
:10C45800FFF75EFFC0F3802032E0B72A00F06E825B
:10C4680010D8B42A00F04F82C0F03982B52A00F003
:10C478005382B62A7FF47DAF002C40F05882AE4B31
:10C488001B695FE0CE2A00F08D820AD8B82A00F036
:10C498006882B92A7FF46DAF002C40F076820720BD
:10C4A800A4E1D02A00F09182D62A7FF462AF002C52
:10C4B80040F09382A04B5B6844E024B913F0FEFA85
:10C4C8002860204638BD012C01D00024F9E71968FE
:10C4D80013F018FAF9E714B913F0E4FAF0E7012CAD
:10C4E800F3D1196813F0B8FAEFE714B913F002FBA7
:10C4F800E6E7012CE9D1196813F0F8F9E5E71CB96A
:10C5080013F0EAFA2860E0E7012C3FF432AFDCE7E9
:10C5180014B913F00BFBD3E7012CD6D11968002905
:10C52800B8BF494213F0A6FACFE714B913F0F0FAEE
:10C53800C6E7012CC9D1196813F08FFBC5E71CB9F0
:10C548007D4BDB7A2B60BCE7012CBED11B687A4C93
:10C558000020E372FFF7DCFE0206B6D4E17A06207B
:10C5680001F01F01FFF798FEAFE714B9724B1B7873
:10C57800E8E7012CA9D11B686F4C00202370FFF756
:10C58800C7FE0306A1D52178E9E7012C9DD11B68D8
:10C59800102B23D00DDC022B1CD004DC012B16D071
:10C5A8004FF0FF3314E0042B16D0082BF8D10523E5
:10C5B8000EE0402B14D003DC202BF1D1032307E03D
:10C5C800802B0FD0B3F5807FEAD1002300E0082349
:10C5D8002B6008E00723FBE70623F9E70423F7E7C6
:10C5E8000223F5E72C602B68013300F0FC8108205A
:10C5F800FFF78EFE2B6820F00F0103F00F0319439D
:10C608000820AFE72CB90820FFF782FEC0F34020CE
:10C6180056E7012C7FF459AF0820FFF779FE2B6805
:10C6280020F400715B0203F40073E8E72CB90820DA
:10C63800FFF76EFEC0F3002042E7012C7FF445AF00
:10C648000820FFF765FE2B6820F480711B0203F4B5
:10C658008073D4E7012C7FF438AF0C20FFF758FE25
:10C668002B6820F4C031DB0303F4C03319430C20DA
:10C6780078E72CB90C20FFF74BFEC0F380301FE79A
:10C68800012C7FF422AF0C20FFF742FE2B6820F428
:10C6980080419B0303F48043E8E72CB90C20FFF7A3
:10C6A80037FEC0F3C1200BE7012C7FF40EAF0C203E
:10C6B800FFF72EFE2B6820F4C051DB0203F4C053B1
:10C6C800D4E72CB90C20FFF723FEC0F3C310F7E61C
:10C6D800012C7FF4FAAE0C20FFF71AFE2B6820F429
:10C6E800F061DB0103F4F063C0E72CB90C20FFF71D
:10C6F8000FFEC0F30210E3E6012C7FF4E6AE0C2037
:10C70800FFF706FE2B6820F070011B0103F0700391
:10C71800ACE7012C7FF4D9AE0C20FFF7F9FD2B68AC
:10C7280020F00F0103F00F03A0E73CB90520FFF745
:10C73800EFFDC0F3C030C3E6044C0020012C7FF4A9
:10C74800C4AE0D20FFF7E4FD2B6820F40041DB03A5
:10C758009BB219430D2005E72CB90520FFF7D8FD3A
:10C76800C0F34130ACE6012C7FF4AFAE0D20FFF7EB
:10C77800CFFD2B6820F4C0415B0303F4C043E8E716
:10C788002CB90520FFF7C4FDC0F3032098E6012C5F
:10C798007FF49BAE0D20FFF7BBFD2B6820F4706182
:10C7A8001B0203F47063D4E72CB90520FFF7B0FD32
:10C7B800C0F3411084E6012C7FF487AE0D20FFF70B
:10C7C800A7FD2B6820F060015B0103F06003C0E760
:10C7D800012C7FF47AAE0D20FFF79AFD2B6820F02C
:10C7E8000F0103F00F03B4E72CB90620FFF790FD03
:10C7F800C0F3004064E6012C7FF467AE0E20FFF71B
:10C8080087FD2B6820F480311B0403F4803319431F
:10C818000E20A7E664B90620FFF77AFD000A00F0AB
:10C828007F0310F0400018BF6FF07F00184347E601
:10C83800012C7FF44AAE0E20FFF76AFD2B6820F426
:10C84800FE411B0203F4FE43E1E72CB90720FFF782
:10C858005FFDC0F3813033E6012C7FF436AE0F2044
:10C86800FFF756FD2B6820F440419B039BB2194308
:10C878000F2077E62CB90720FFF74AFDC0F30130F7
:10C888001EE6012C7FF421AE0F20FFF741FD2B6837
:10C8980020F440511B0303F44053E8E7012C7FF4D4
:10C8A80014AE0F20FFF734FD2B6820F480619B0243
:10C8B80003F48063DBE72CB90720FFF729FDC0F3F9
:10C8C8000120FDE5012C7FF400AE0F20FFF720FDCD
:10C8D8002B6820F440711B0203F44073C7E72CB99E
:10C8E8000720FFF715FDC0F38010E9E5012C7FF460
:10C8F800ECAD0F20FFF70CFD2B6820F040019B01E9
:10C9080003F04003B3E7002C7FF4FEAD0220FFF7ED
:10C91800FFFCC0F38420D3E514B913F015F9CFE573
:10C92800012C7FF4D2AD196813F0AEF8CDE5012CD7
:10C938007FF4CBAD1A682D4B1A61C6E52CB90720D8
:10C94800FFF7E6FCC0F3C010BAE5012C7FF4BDADDB
:10C958000F20FFF7DDFC2B6820F08001DB01DBB244
:10C9680085E72CB90420FFF7D3FCC0F34030A7E5D6
:10C97800012C7FF4AAAD0C20FFF7CAFC2B6820F429
:10C9880000515B0303F4005370E6012C7FF49DAD66
:10C998000F20FFF7BDFC2B6820F480311B0403F443
:10C9A800803364E7002C7FF4AFAD114B1B6833B1C3
:10C9B8000220FFF7ADFC800A00F47870A2E50120A0
:10C9C800FFF7A6FCC0F389209CE5002C7FF49CAD02
:10C9D8000320FFF79DFCC0B272E5012C02BF1A6864
:10C9E800024B5A6071E510246BE500BF044C00202F
:10C9F8006400002007B5019239B9024601AB012055
:10CA0800FFF79CFC03B05DF804FB0820FAE710B4BC
:10CA180013460446084611B9224610BC8EE4082085
:10CA280010BC704710B508461446FFF771FC20602B
:10CA380010BDF8B506460020FFF76AFC284DC0F384
:10CA4800C0176B7E274CBB4208D0002F3ED0217800
:10CA580001F01F010620FFF71FFC6F76237A224A98
:10CA6800002B35D0136F43F00103617A002933D0CE
:10CA780043F002030020136713F02EF823690028FF
:10CA8800B8BF4042984234BF00270127AA7EBA4265
:10CA980010D098424FF00D002CBF647B247BFFF729
:10CAA80037FC04F00F0420F00F0121430D20FFF79D
:10CAB800F3FBAF760D4B31461B680020094A13F093
:10CAC80040FEBDE8F840002012F028BFE17ABFE739
:10CAD800136F23F00103C8E723F00203CAE700BF7E
:10CAE800A0140020044C0020203E0020504C0020C0
:10CAF80010B406290C4C0D4BC2F3130004BF02F00E
:10CB08001F02E2721B6801F0770242F0080203EB91
:10CB180082035860A37A23B940EA414010BCFFF76A
:10CB280057BB10BC704700BF044C0020504C00207D
:10CB380010B5084B0C469B7A23B90B0702D408465C
:10CB4800FFF7CDFB044B04F07F04196801EB840464
:10CB5800606810BD044C0020504C00202DE9F843BB
:10CB68008B0C0C460DD0C1F34243062B09D1294B3F
:10CB780021F01F045A7A002A43D01B7803F01F03C0
:10CB88001C43254F254E3B68254D9B680021C4F367
:10CB98000740D6F8008095F81B909847EA7E3368DE
:10CBA80008EB8908C8F8040003EB82035A680021DF
:10CBB80012025A603B68C4F307209B689847EB7ED3
:10CBC8003268012102EB8302536818433B68000274
:10CBD80050609B68E0B298473268E97E02EB8101B9
:10CBE8004B6818430011A30C486010610BD0C4F3C4
:10CBF8004243072B02D1C4F30111E97643F008033D
:10CC080002E0DB7ABAE7082302EB83035C60BDE845
:10CC1800F88300BF044C00204C4C0020504C0020EE
:10CC2800A01400202DE9F0410126484F484BDFF8B9
:10CC3800788138461E6013F061FDD8F80C50454CD9
:10CC48006B6803F1C802E26003F1E40203F5B8700F
:10CC5800226103F5C67203F50D7323602B68A26089
:10CC6800DB68606098472B68A068DB6898472B688A
:10CC7800E068DB6898472B6820691B6998472B6830
:10CC88002068DB68984768682B6820309B6860617B
:10CC98009847D8F81030304A03F11401116022681F
:10CCA8009A6105233B704FF47A737B6012F05AFF48
:10CCB8002369A2686168002012F0A4FE274B284966
:10CCC800D3F8802002200A602649C2F808122649B3
:10CCD800C2F80412002151701170244A83F87C6054
:10CCE800C3F88C20224ABDE8F041C3F88820214AC5
:10CCF800C3F88420204AC3F89020204AC3F8A4200F
:10CD08001F4AC3F8A0201F4AC3F894201E4AC3F83C
:10CD180098201E4AC3F8B4201D4AC3F8B0201D4A03
:10CD2800C3F8C0201C4AC3F8BC201C4AC3F8B8206A
:10CD38001B4AC3F8CC2032229A674FF416725A67FE
:10CD4800184AC3F8C420FFF7A7B900BF044C002055
:10CD580064000020A01400204C4C0020203E00203D
:10CD6800504C002093C000088BC1000865C1000822
:10CD780089C1000885C1000881C1000817CA0008D8
:10CD8800FDC9000881C0000847C10008E1C20008C9
:10CD98002DCA00083BCA00083DC0000831C1000880
:10CDA800A1C00008E1C00008649E02082DE9F8430C
:10CDB800830C04460DD0C0F34243062B09D1294BFE
:10CDC80020F01F045A7A002A43D01B7803F01F036F
:10CDD8001C43254F254E3B68254D9B680021C4F315
:10CDE8000740D6F8008095F8009098472A7833686D
:10CDF80008EB8908C8F8040003EB82035A6800218D
:10CE080012025A603B68C4F307209B6898472B7846
:10CE18003268012102EB8302536818433B68000221
:10CE280050609B68E0B298473268297802EB81012C
:10CE38004B6818430011A30C486010610BD0C4F371
:10CE48004243072B02D1C4F30111297043F00803B0
:10CE580002E0DB7ABAE7082302EB83035C60BDE8F3
:10CE6800F88300BF584C0020544C0020A04C0020F0
:10CE7800C8140020012810B514460CD003D302288A
:10CE880010D0042010BD1368094AB3FA83F35B0974
:10CE98009372002010BD1368064AB3FA83F35B0946
:10CEA8001360F6E7084612F08DFD2060F1E700BF39
:10CEB800584C00206800002010B5044618B912F03C
:10CEC80021FD204610BD082010BD024B186813F044
:10CED8005CBD00BFA04C0020022804BF0B4B93F898
:10CEE800D80030B90A4BDB681B685B69094A1069CE
:10CEF8001847012809D1054B93F8D830012B04D1E4
:10CF0800034BDB681B689B69F0E77047203E0020F5
:10CF1800649E0208C814002038B50020FFF7DCFF23
:10CF28000F4B104CDD6820692B685B6998472B68AC
:10CF380060689B6898472B68E0689B6898472B68EF
:10CF480020699B6898472B6860699B6898472B689D
:10CF5800A0689B689847BDE8384012F057BE00BFEC
:10CF6800649E0208C814002038B50D46044620B94E
:10CF780012F0B2FD2860204638BD082038BD38B50B
:10CF88000C46054640B912F08DFD2368C118216092
:10CF98002846BDE838408FE7082038BD10B504465C
:10CFA80030B9044B5872187212F0A0FC204610BD1C
:10CFB800082010BD584C00200021EFE74942EDE75A
:10CFC800ECE738B5002012F087FD0546A8B9012422
:10CFD8000B4B0C48196813F0BBFC0B4B02201C6070
:10CFE800FFF77AFF12F0BEFD084928464B69CA6868
:10CFF800896812F007FD204638BD002038BD00BF03
:10D00800A04C0020584C002068000020C8140020C4
:10D018000346C1F31300820C10B40B4C05D0421424
:10D02800062A04BF01F01F01E172084A03F07703E2
:10D03800126843F0080302EB83035860A37A0BB924
:10D0480010BCB3E610BC7047584C0020A04C002020
:10D0580008461146DCE710B5074B04469B7A1BB916
:10D06800030701D400F0D6FB044B04F07F041B68CF
:10D0780003EB8404606810BD584C0020A04C0020CD
:10D08800A82A38B504461D46084600F0F3815CD846
:10D098001D2A00F0D78022D8042A00F0DC800CD8A2
:10D0A800012A00F0BB80C0F0AB80022A00F0C080EB
:10D0B800032A00F0C7800424A6E0062A00F0E280D4
:10D0C800C0F0D680072A00F0F380082AF3D1002C9C
:10D0D80040F0BD8012F076FCC0F3001093E0A32A64
:10D0E80000F06A811ED8A02A00F02F810CD88C2A63
:10D0F800E1D1002C40F0EC800820FFF7ACFF00F0F5
:10D108000F00C0F108007EE0A12A00F03281A22AB7
:10D11800D1D1002C40F041810C20FFF79CFFC0F3D7
:10D12800C13070E0A52A00F06F81C0F05981A62AAD
:10D1380000F08081A72ABED1002C40F08F810C20FE
:10D14800FFF789FF00F00F005DE0B22A00F051827E
:10D1580026D8AD2A00F0E6810FD8AA2A00F0B381BC
:10D16800C0F09D81AB2A00F0C281AC2AA3D1002C6B
:10D1780040F0D181AE4B5B7B87E0AF2A00F00382A1
:10D18800C0F0E681B02A00F01382B12A93D1002CB6
:10D1980040F022820720FFF75EFFC0F3802032E0D4
:10D1A800B72A00F0698210D8B42A00F04A82C0F089
:10D1B8003482B52A00F04E82B62A7FF47CAF002C68
:10D1C80040F053829A4B1B695FE0CE2A00F08882B8
:10D1D8000AD8B82A00F06382B92A7FF46CAF002C11
:10D1E80040F0718207209FE1D02A00F08C82D62A75
:10D1F8007FF461AF002C40F08E828D4B5B6844E079
:10D2080024B912F05BFC2860204638BD012C01D0FF
:10D218000024F9E7196812F075FBF9E714B912F060
:10D2280041FCF0E7012CF3D1196812F015FCEFE787
:10D2380014B912F05FFCE6E7012CE9D1196812F085
:10D2480055FBE5E71CB912F047FC2860E0E7012C24
:10D258003FF431AFDCE714B912F068FCD3E7012CD6
:10D26800D6D119680029B8BF494212F003FCCFE7AC
:10D2780014B912F04DFCC6E7012CC9D1196812F097
:10D28800ECFCC5E71CB96A4BDB7A2B60BCE7012CC8
:10D29800BED11B68664C0020E372FFF7DCFE020675
:10D2A800B6D4E17A062001F01F01FFF7B1FEAFE71F
:10D2B80014B95F4B1B78E8E7012CA9D11B685C4CBB
:10D2C80000202370FFF7C7FE0306A1D52178E9E700
:10D2D800012C9DD11B68102B23D00DDC022B1CD0F8
:10D2E80004DC012B16D04FF0FF3314E0042B16D0CA
:10D2F800082BF8D105230EE0402B14D003DC202B9B
:10D30800F1D1032307E0802B0FD0B3F5807FEAD15A
:10D31800002300E008232B6008E00723FBE706232F
:10D32800F9E70423F7E70223F5E72C602B680133BC
:10D3380000F0F7810820FFF78EFE2B6820F00F0120
:10D3480003F00F0319430820AFE72CB90820FFF7B3
:10D3580082FEC0F3402056E7012C7FF459AF082025
:10D36800FFF779FE2B6820F400715B0203F4007369
:10D37800E8E72CB90820FFF76EFEC0F3002042E76B
:10D38800012C7FF445AF0820FFF765FE2B6820F4D9
:10D3980080711B0203F48073D4E7012C7FF438AF4B
:10D3A8000C20FFF758FE2B6820F4C031DB0303F490
:10D3B800C03319430C2078E72CB90C20FFF74BFE3B
:10D3C800C0F380301FE7012C7FF422AF0C20FFF759
:10D3D80042FE2B6820F480419B0303F48043E8E776
:10D3E8002CB90C20FFF737FEC0F3C1200BE7012C46
:10D3F8007FF40EAF0C20FFF72EFE2B6820F4C051EF
:10D40800DB0203F4C053D4E72CB90C20FFF723FE4A
:10D41800C0F3C310F7E6012C7FF4FAAE0C20FFF737
:10D428001AFE2B6820F4F061DB0103F4F063C0E717
:10D43800584C00202CB90C20FFF70DFEC0F3021049
:10D44800E1E6012C7FF4E4AE0C20FFF704FE2B6824
:10D4580020F070011B0103F07003AAE7012C7FF490
:10D46800D7AE0C20FFF7F7FD2B6820F00F0103F073
:10D478000F039EE72CB90520FFF7EDFDC0F3C03080
:10D48800C1E6012C7FF4C4AE0D20FFF7E4FD2B6844
:10D4980020F40041DB039BB219430D2005E72CB9AA
:10D4A8000520FFF7D8FDC0F34130ACE6012C7FF42E
:10D4B800AFAE0D20FFF7CFFD2B6820F4C0415B0312
:10D4C80003F4C043E8E72CB90520FFF7C4FDC0F317
:10D4D800032098E6012C7FF49BAE0D20FFF7BBFDDF
:10D4E8002B6820F470611B0203F47063D4E72CB935
:10D4F8000520FFF7B0FDC0F3411084E6012C7FF44E
:10D5080087AE0D20FFF7A7FD2B6820F060015B01B7
:10D5180003F06003C0E7012C7FF47AAE1A68824BEF
:10D528005A7375E62CB90620FFF795FDC0F3004045
:10D5380069E6012C7FF46CAE0E20FFF78CFD2B689A
:10D5480020F480311B0403F4803319430E20ACE629
:10D5580064B90620FFF77FFD000A00F07F0310F092
:10D56800400018BF6FF07F0018434CE6012C7FF491
:10D578004FAE0E20FFF76FFD2B6820F4FE411B0213
:10D5880003F4FE43E1E72CB90720FFF764FDC0F37D
:10D59800813038E6012C7FF43BAE0F20FFF75BFDAE
:10D5A8002B6820F440419B039BB219430F207CE673
:10D5B8002CB90720FFF74FFDC0F3013023E6012CFB
:10D5C8007FF426AE0F20FFF746FD2B6820F440516C
:10D5D8001B0303F44053E8E7012C7FF419AE0F2036
:10D5E800FFF739FD2B6820F480619B0203F4806308
:10D5F800DBE72CB90720FFF72EFDC0F3012002E678
:10D60800012C7FF405AE0F20FFF725FD2B6820F4D1
:10D6180040711B0203F44073C7E72CB90720FFF7DA
:10D628001AFDC0F38010EEE5012C7FF4F1AD0F2058
:10D63800FFF711FD2B6820F040019B0103F0400328
:10D64800B3E7002C7FF403AE0220FFF704FDC0F31C
:10D658008420D8E514B912F077FAD4E5012C7FF4C8
:10D66800D7AD196812F010FAD2E5012C7FF4D0ADCD
:10D678001A682D4B1A61CBE52CB90720FFF7EBFC94
:10D68800C0F3C010BFE5012C7FF4C2AD0F20FFF737
:10D69800E2FC2B6820F08001DB01DBB285E72CB9C6
:10D6A8000420FFF7D8FCC0F34030ACE5012C7FF430
:10D6B800AFAD0C20FFF7CFFC2B6820F400515B03C3
:10D6C80003F4005375E6012C7FF4A2AD0F20FFF799
:10D6D800C2FC2B6820F480311B0403F4803364E718
:10D6E800002C7FF4B4AD114B1B6833B10220FFF757
:10D6F800B2FC800A00F47870A7E50120FFF7ABFCC4
:10D70800C0F38920A1E5002C7FF4A1AD0320FFF729
:10D71800A2FCC0B277E5012C02BF1A68024B5A601E
:10D7280076E5102470E500BF584C00206800002002
:10D7380007B5019239B9024601AB0120FFF7A0FCF9
:10D7480003B05DF804FB0820FAE710B50846144654
:10D75800FFF781FC206010BDF8B506460020FFF7F2
:10D768007AFC284DC0F3C0172B7F274CBB4208D04A
:10D77800002F3ED0217801F01F010620FFF748FC5A
:10D788002F77237A214A002B35D0136F43F00103FA
:10D79800617A002933D043F002030020136712F0A6
:10D7A8009BF923690028B8BF4042984234BF00273C
:10D7B80001276A7FBA4210D098424FF00D002CBF63
:10D7C800647B247BFFF747FC04F00F0420F00F0173
:10D7D80021430D20FFF71CFC6F770D4B31461B686A
:10D7E8000020094A13F05FF8BDE8F840002012F065
:10D7F80095B8E17ABFE7136F23F00103C8E723F078
:10D808000203CAE7C8140020584C0020203E00201C
:10D81800A04C002038B504460F20FFF71CFC03235A
:10D82800B4FBF3F3054603EB4303E41A240104F0C5
:10D83800300420F030002043FFF7B8FA2846BDE84E
:10D848003840FFF7B3BA10B413460446084611B976
:10D85800224610BC14E4082010BC7047C2F3130021
:10D86800830C10B40B4C05D04314062B04BF02F0F4
:10D878001F02E272084B01F077011B6841F00801B2
:10D8880003EB81014860A37A13B910BCFFF78EBA85
:10D8980010BC7047584C0020A04C002010B5084B15
:10D8A8000C469B7A23B90B0702D40846FFF7B2FF50
:10D8B800044B04F07F04196801EB8404606810BD10
:10D8C800584C0020A04C00202DE9F8438B0C0C4646
:10D8D8000DD0C1F34243062B09D1294B21F01F0477
:10D8E8005A7A002A43D01B7803F01F031C43254FA4
:10D8F800254E3B68254D9B680021C4F30740D6F8A8
:10D90800008095F81E909847AA7F336808EB89082D
:10D91800C8F8040003EB82035A68002112025A6017
:10D928003B68C4F307209B689847AB7F32680121A6
:10D9380002EB8302536818433B68000250609B68FF
:10D94800E0B298473268A97F02EB81014B6818431F
:10D958000011A30C486010610BD0C4F34243072B9D
:10D9680002D1C4F30111A97743F0080302E0DB7A7E
:10D97800BAE7082302EB83035C60BDE8F88300BFC5
:10D98800584C0020544C0020A04C0020C814002003
:10D998002DE9F0410126484F484BDFF87881384699
:10D9A8001E6012F05DFFD8F80C50454C6B6803F10F
:10D9B800C802226103F1E40203F5B870626103F55D
:10D9C800C67203F50D7363602B68E260DB68A060C4
:10D9D80098472B68E068DB6898472B682069DB6804
:10D9E80098472B6860691B6998472B686068DB68F3
:10D9F800984768682B6820309B68A0619847D8F8DA
:10DA08001030304A03F11401116062689A610523ED
:10DA18003B704FF47A737B6012F0A4F86369E26894
:10DA2800A168002011F0EEFF274B2849D3F8802089
:10DA380002200A602649C2F808122649C2F80412D0
:10DA4800002151701170244A83F87C60C3F88C203F
:10DA5800224ABDE8F041C3F88820214AC3F884204F
:10DA6800204AC3F89020204AC3F8A4201F4AC3F8CC
:10DA7800A0201F4AC3F894201E4AC3F898201E4AC3
:10DA8800C3F8B4201D4AC3F8B0201D4AC3F8C0200B
:10DA98001C4AC3F8BC201C4AC3F8B8201B4AC3F868
:10DAA800CC2032229A6740F225125A67184AC3F8E6
:10DAB800C420FFF711BA00BF584C002068000020AE
:10DAC800C8140020544C0020203E0020A04C002008
:10DAD800D3CE0008CBCF0008A5CF0008C9CF0008D7
:10DAE800C5CF0008C1CF00084FD8000839D70008B3
:10DAF800C1CE000887CF000859D0000853D70008C6
:10DB080061D700087DCE000871CF0008E1CE00087B
:10DB180021CF0008649E02080022014B5A6070471A
:10DB2800203E002070B5184E184CF56860682B68C8
:10DB38009B6998472B68A0699B6898472B68606920
:10DB48009B6898472B6820699B6898472B68E06812
:10DB58009B6898472B68A0689B6898472B68206A41
:10DB68009B6898472B68E0699B6898472B682068F2
:10DB78009B6898472B6860689B6898473369BDE83D
:10DB880070405B6A184700BF649E0208F4140020C6
:10DB98000228F8B5144653D004D890B101283DD0D6
:10DBA800042439E003285DD0FF28F9D1324CD4F899
:10DBB8008030D3F8043298476369D3F80432984721
:10DBC80003E0136833F0030201D0002424E013F0CB
:10DBD800010F2A4D2A4E0ED0F3681B681B6968692D
:10DBE8009847246814F002040DD0F368A8691B68EC
:10DBF8001B699847E9E7F76868693B68DB689847F5
:10DC08003B689B69EBE7F668A8693368DB68984767
:10DC18003368A8699B6998472046F8BD1468174D72
:10DC2800174B24B1DB6828691B681B69E1E7DE68CC
:10DC380028693368DB689847336828699B69EAE78D
:10DC480014680E4D0E4B24B1DB68A8681B681B696D
:10DC5800CFE7DE68A8683368DB6898473368A86848
:10DC68009B69D8E70121074812F0CEFF2060002801
:10DC7800ABD12024D0E700BF203E0020F4140020C0
:10DC8800649E0208A84C00200146014813F072B8AF
:10DC9800A84C002010B50348144612F0D8FE2060A6
:10DCA80010BD00BFA84C0020014812F0C2BE00BF42
:10DCB800A84C002008B5034B03485A6A12F094FF99
:10DCC800002008BDF4140020A84C002008B5034B20
:10DCD80003485A6A12F06CFF002008BDF4140020B3
:10DCE800A84C002008B50021024812F043FF00208C
:10DCF80008BD00BFA84C002008B54942024812F0F0
:10DD080039FF002008BD00BFA84C002008B5024814
:10DD180012F030FF002008BDA84C002038B5094B90
:10DD2800094CDD6860682B689B69984701200EF0F4
:10DD3800CDFE2B6860685B699847044812F0EFFED7
:10DD4800012038BD649E0208F4140020A84C00206D
:10DD580038B5094B094CDD6860682B689B699847A2
:10DD680001200EF0B3FE2B6860685B699847044891
:10DD780012F0C0FE012038BD649E0208F414002091
:10DD8800A84C00206E2938B50446154600F0E381FA
:10DD98006FD8122900F0708137D8052900F0248146
:10DDA80017D8022900F0FD8007D8002900F0DF808D
:10DDB800012900F0EE800424E3E0032900F000814B
:10DDC8000429F8D1002840F00281B14B5B6A2B602E
:10DDD800D7E00F2900F02F810DD8082900F019810C
:10DDE8000E29E8D1002840F01D812021A94812F011
:10DDF8002EFE4000C0E0102900F025811129DAD15B
:10DE0800002840F02E812921F0E0182900F07381C4
:10DE180017D8152900F0528109D8132900F0358147
:10DE28001429C8D1002840F043812621A1E01629F1
:10DE380000F052811729BED1002840F056812E21CA
:10DE480097E01B2900F06F8109D8192900F05C813F
:10DE58001A29B0D1002840F06081332189E06C296B
:10DE680000F06A816D29A6D1002840F06E816121F9
:10DE78007FE07E2900F013823AD8742900F0C4812B
:10DE880019D871295ED009D86F2900F079817029D5
:10DE980091D1002840F0898159216AE0722900F067
:10DEA8009781732987D1002840F0A881794B1B6896
:10DEB800D3F86C318BE7772900F0D9810DD8752913
:10DEC80000F0AE8176297FF476AF002840F0C1815A
:10DED800704B1B6893F8723179E77C2900F0D08188
:10DEE8007D297FF468AF002840F0D3815F2140E0AE
:10DEF800892900F026821BD8852900F0FD8109D8E0
:10DF0800812900F0E28184297FF455AF00285AD195
:10DF180065212EE0862900F0FC8188297FF44BAF2B
:10DF2800002840F0FF815B4B1B6893F890314EE767
:10DF3800D12900F030820FD88A2900F01882C82928
:10DF48007FF439AF002C40F036810521514812F09A
:10DF58007EFDC0B2286013E0D42900F02582D629BE
:10DF68007FF429AF002840F02A82152101E028B962
:10DF78003721484812F06BFD286002E0012802D0E2
:10DF88000024204638BD37211268424812F051FD5E
:10DF9800F6E708B92121ECE70128F1D1126821211F
:10DFA800F3E728B924213B4812F051FD0012E3E7BA
:10DFB8000128E5D1106812F0CBFD24210246E4E7E0
:10DFC80008B92221D5E7012C3FF4F5AED8E701289E
:10DFD800D6D113682E4C20212E48636212F037FDEB
:10DFE8004207CDD5606AE6E728B92821294812F00A
:10DFF8002EFD8010C0E70128C2D11268940DA40537
:10E00800002C40F0E48128219200224812F011FDF2
:10E01800B7E70028D7D10F211E4812F018FD00F0ED
:10E028000100A9E70128ABD113682021002B0CBF00
:10E0380001220222A9E708B925219AE701289FD1E0
:10E0480012682521A1E708B92A21CFE7012897D12D
:10E058001268940DA405002C40F0B98192002A2181
:10E06800D3E701288CD11268940DA405002C40F048
:10E07800AE8192002921C8E708B9272179E701284C
:10E088007FF47EAF126827217FE728B92B21ADE7FF
:10E09800F4140020A84C002001287FF471AF126806
:10E0A800940DA405002C40F0928192002B21ACE73E
:10E0B80001287FF465AF1268262166E708B92C218C
:10E0C80057E701287FF45CAF1268930D9B05002B7E
:10E0D80040F07D812C2158E708B92D2149E7012816
:10E0E8007FF44EAF12682D214FE701287FF448AF27
:10E0F80012682E2149E708B92F213AE701287FF451
:10E108003FAF12682F2140E708B9302131E70128D5
:10E118007FF436AF1268302137E701287FF430AF3B
:10E128001268332131E708B9342122E701287FF446
:10E1380027AF1268342128E708B9602119E70128B8
:10E148007FF41EAF126860211FE701287FF418AF23
:10E158001268612119E728B91C219E4812F077FC42
:10E16800001409E701287FF40BAF1C21994812F02D
:10E178006EFC2A68C0F3080040EA02421C2104E74A
:10E1880028B91C21934812F062FCC0B2F4E60128B9
:10E198007FF4F6AE1C218F4812F059FC2B6800F46E
:10E1A8007F02C3F308031A43E8E701287FF4E8AEC7
:10E1B80012685921E9E6012C7FF4E2AE0521854871
:10E1C80012F045FC2A7820F0FF0002430521DCE626
:10E1D80030B905217F4812F03AFCC0F30720CBE69E
:10E1E80001287FF4CDAE05217A4812F030FC2B6867
:10E1F80020F47F421B029BB21A43E7E701287FF411
:10E20800BFAE12685A21C0E620B9724B1B68D3F81A
:10E218007031DCE501287FF4B3AE12685B21B4E607
:10E2280030B96C4B1B68D3F87031C3F30E03CEE5DD
:10E2380001287FF4A5AE674812680368C2F30E028E
:10E24800D3F8703123F4FF4323F07F031A435B2193
:10E258009CE601287FF494AE5E480368D3F87021E9
:10E268002B6822F47F021B0403F47F03EEE708B94E
:10E278005E217EE601287FF483AE12685E2184E683
:10E2880008B95C2175E601287FF47AAE12685C2132
:10E298007BE601287FF474AE12685F2175E630B919
:10E2A80005214C4812F0D3FBC0F3074064E601286F
:10E2B8007FF466AE0521474812F0C9FB2B6820F4AD
:10E2C8007F021B0403F47F0396E701287FF458AE0E
:10E2D80014684CB101213F4812F096FC28600028D0
:10E2E8007FF44EAE20244CE607213A4812F0AFFBEB
:10E2F800072120F4800288E600287FF441AE072138
:10E30800344812F0A4FBC0F38150431E58425841D0
:10E3180032E608B952212CE601287FF431AE1268A2
:10E32800522132E601287FF42BAE2A48126803688E
:10E3380002F00F02D3F8903123F0FF031A43632150
:10E3480024E630B9234B1B68D3F89031C3F3032379
:10E358003DE501287FF414AE1E480368D3F89021E8
:10E368002B6822F470621B0203F47063E6E720B99D
:10E37800184B1B6893F8923129E501287FF400AE09
:10E3880014480368D3F890212B6822F47F021B04F9
:10E3980003F47F03D2E708B95021EAE501287FF4A6
:10E3A800EFAD12685021F0E518B90A4B1B689B695C
:10E3B8000DE501287FF4E4AD12685321E5E5012855
:10E3C8007FF4DEAD1368044A15215A43DDE51024B5
:10E3D800D7E500BFA84C0020007102000B4611B918
:10E3E80001461846CEE40820704708B5024812F0E6
:10E3F800C1FB002008BD00BFA84C002007B5019252
:10E4080039B9014601AA0120FFF7BCFC03B05DF849
:10E4180004FB0820FAE7034B08461B681146DB6833
:10E42800184700BFA44C0020F8B5484D484F0021BC
:10E43800484B6A69484812F03FFBFE68474C7368CE
:10E4480003F59C72226203F5AA72E26103F5537226
:10E45800A26103F55A72626103F56172226103F5E4
:10E46800687203F57670E26003F56F7203F57D73E9
:10E4780023603368A260DB68606098473368A069EE
:10E48800DB68984733686069DB68984733682069B8
:10E49800DB6898473368E068DB6898473368A068AA
:10E4A800DB689847336860685B6998473368A06998
:10E4B8005B699847336860695B6998473368206986
:10E4C8005B6998473368E0685B6998473368A06878
:10E4D8005B6998473368206A1B6998473368E06925
:10E4E8001B699847336820681B6998473A691C4B31
:10E4F80000211A60736803F53773536001226B6952
:10E50800597018491A70C3F8041217492A74C3F8C5
:10E518000812164B2B62164BEB61164BAB61164B70
:10E528006B62164BAB63164B6B63164BAB62164BA9
:10E53800EB62164BAB64164B6B64164B6B65164B54
:10E548002B65164BEB65164BAB65F8BD203E0020DE
:10E55800649E02085C920208A84C0020F414002073
:10E56800A44C002059DD000825DD0008F3E300086D
:10E5780015DD000801DD0008EDDC0008E5E3000812
:10E5880005E40008D5DC0008BDDC0008B1DC0008A3
:10E598009DDC000891DC000899DB000821DB0008FD
:10E5A8002DDB00080022014B5A607047203E0020F6
:10E5B8000228F8B514464ED004D890B1012839D0B5
:10E5C8000420F8BD032857D0FF28F9D12B4CD4F8E4
:10E5D8008030D3F8043298476369D3F804329847F7
:10E5E80016E0136833F0030247D113F0010F244DEE
:10E5F800244E0FD0F3681B681B6968699847246824
:10E6080014F002040ED0F3681B681B69A8699847C8
:10E618000020F8BDF76868693B68DB6898473B6885
:10E628009B69EAE7F668A8693368DB689847336846
:10E638009B69EBE71468124D124B24B1DB681B6829
:10E648001B692869E3E7DE6828693368DB6898474F
:10E6580033689B69F5E71468094D0A4B24B1DB68F8
:10E668001B681B69A868D2E7DE68A8683368DB689E
:10E67800984733689B69F5E72020F8BD203E0020C5
:10E6880028150020649E020870B5184E184CF568CD
:10E6980060682B689B6998472B68A0699B689847B6
:10E6A8002B6860699B6898472B6820699B68984726
:10E6B8002B68E0689B6898472B68A0689B68984718
:10E6C8002B68206A9B6898472B68E0699B68984785
:10E6D8002B6820689B6898472B6860689B689847F8
:10E6E8003369BDE870405B6A184700BF649E020842
:10E6F800281500200A460146014812F0FBBB00BF5E
:10E70800404F00200146014812F0A2BC404F0020B3
:10E7180010B50348144612F0B8FB206010BD00BFC6
:10E72800404F0020014812F0A2BB00BF404F00201C
:10E7380008B5034B03485A6A12F018FD002008BDBB
:10E7480028150020404F002008B5034B03485A6A9B
:10E7580012F0F0FC002008BD28150020404F0020D2
:10E7680008B50021024812F0C7FC002008BD00BF10
:10E77800404F002008B54942024812F0BDFC002075
:10E7880008BD00BF404F002008B5024812F0B4FC95
:10E79800002008BD404F002038B5094B094CDD6802
:10E7A80060682B689B69984701200EF08FF92B68E9
:10E7B80060685B699847044812F031FC012038BD55
:10E7C800649E020828150020404F002038B5094BE8
:10E7D800094CDD6860682B689B69984701200EF03A
:10E7E80075F92B6860685B699847044812F002FC69
:10E7F800012038BD649E020828150020404F0020E3
:10E8080070B5114C0D4694F86C30012B19D0032BC0
:10E818000BBF002228220C230F2343F0884343F028
:10E82800401343EA4232042112F021FBD4F880302D
:10E83800012D0CBFD3F80432D3F80832BDE870407C
:10E84800184700220B23E8E7203E0020F8B50027F0
:10E858002F4CA56AE66A2A023302C6B243EA156358
:10E86800324394F83000E66B3B43A76B0130350E1A
:10E87800360246EA1766C0B23F02C4E90A2384F8A2
:10E888003000E663A763002940D0042804D91A465B
:10E898006D21204812F0EBFAA26A6C211D4812F093
:10E8A800E6FA01200EF012F9A26A6C21194812F05A
:10E8B800DEFA00230022C4E90E2394F83030042B3A
:10E8C8000AD96F21134812F0E0FAD4E90E23002682
:10E8D80003433243C4E90E236E210E4812F0D5FAE1
:10E8E800D4E90E67034694F8302047EAE371C2F191
:10E8F8000802D200304319F085F800230022C4E949
:10E908000A230023C4E90E0184F830302846F8BDF4
:10E9180028150020404F002008B5024812F0ECFBF3
:10E92800002008BD404F002038B515460C46002988
:10E938007AD1112868D01FD804284ED008D80128C9
:10E9480040D03AD302283FD0032844D0042447E0DB
:10E958000E284DD00AD8052844D00828F6D10F2112
:10E96800324812F092FA00F0010032E00F2849D044
:10E978001028EBD12A2136E017284DD00ED81428BC
:10E9880046D005D8122841D01328DFD12B212AE000
:10E9980015283FD01628D9D12D210FE01A283FD0AD
:10E9A80005D818283AD01928D0D1302106E01B28DC
:10E9B80038D0D628CAD1152100E037211B4812F0DB
:10E9C80064FA06E02121F9E72421184812F05DFADB
:10E9D8000012286004E02221F0E7154B5B6A1360FF
:10E9E800204638BD2821114812F04FFA8010F0E770
:10E9F80020210E4812F049FA00F00300831E584205
:10EA08005841E6E72521D9E72921ECE72721D5E771
:10EA18002621D3E72C21D1E72E21CFE72F21CDE7DF
:10EA28003321CBE73421C9E70824D9E7404F002038
:10EA38002815002038B514460D46002940F0878077
:10EA480012286DD021D805285CD008D801283FD0DD
:10EA580038D302283ED0042842D0042536E00F28B7
:10EA680056D007D80E28F8D1002A14BF0222012256
:10EA7800202128E010284DD01128EED1930D9B05B8
:10EA8800002B66D19200292137E0172857D008D8E3
:10EA980014284DD046D315284CD01628DDD12D2169
:10EAA80011E01A284FD005D818284AD01928D4D1EF
:10EAB800302108E01B2848D0D628CED1264A152177
:10EAC800624300E03721254812F0D1F9284638BDC5
:10EAD8002121F8E782EAE272A2EBE4722421F2E74C
:10EAE8001F4D20211D486A6212F0CFF9430707D550
:10EAF800686A12F0EFFA24210246184812F0B7F9B2
:10EB08000025E3E7950DAD051DBB92002821DAE746
:10EB18002521D8E7950DAD05DDB992002A21D2E768
:10EB28002721D0E7950DAD059DB992002B21CAE7A5
:10EB38002621C8E7950DAD055DB92C21C3E72E2127
:10EB4800C1E72F21BFE73321BDE73421BBE7082503
:10EB5800BCE71025BAE700BF00710200404F002053
:10EB680028150020024B08461B681146DB68184729
:10EB78003C4F0020F8B54D4D4D4C4E4B6A69204630
:10EB880000214D4F12F019FA4C49204612F05CFA58
:10EB9800FE684B4C736803F59C72226203F5AA72F7
:10EBA800E26103F55372A26103F55A72626103F5DB
:10EBB8006172226103F5687203F57670E26003F50D
:10EBC8006F7203F57D7323603368A260DB68606051
:10EBD80098473368A069DB68984733686069DB68E1
:10EBE800984733682069DB6898473368E068DB68D2
:10EBF80098473368A068DB689847336860685B6942
:10EC080098473368A0695B699847336860695B69AE
:10EC18009847336820695B6998473368E0685B699F
:10EC280098473368A0685B6998473368206A1B690E
:10EC380098473368E0691B699847336820681B69FF
:10EC480098473A691F4B00211A60736803F53773B8
:10EC5800536001226B6959701B491A70C3F804127A
:10EC68001A492A74C3F80812194B6B66194B2B62A0
:10EC7800194BEB61194BAB61194B6B62194BAB63C9
:10EC8800194B6B63194BAB62194BEB62194BAB64B5
:10EC9800194B6B64194B6B65194B2B65194BEB655D
:10ECA800194BAB65194BAB66F8BD00BF203E002081
:10ECB800404F00205C940208649E020809E800089E
:10ECC800281500203C4F0020D5E70008A1E70008E0
:10ECD80055E8000821E9000891E700087DE70008E9
:10ECE80069E7000831E900083DEA000851E7000833
:10ECF80039E700082DE7000819E700080DE70008C4
:10ED0800B9E50008ADE5000891E60008FDE6000851
:10ED18000022014B5A607047203E002070B5184E03
:10ED2800184CF56860682B689B6998472B68A06940
:10ED38009B6898472B6860699B6898472B6820698F
:10ED48009B6898472B68E0689B6898472B68A06881
:10ED58009B6898472B68206A9B6898472B68E069EE
:10ED68009B6898472B6820689B6898472B68606861
:10ED78009B6898473369BDE870405B6A184700BFD5
:10ED8800649E0208781500200A460146014812F0E0
:10ED980077BA00BFD85100200228F8B5144653D0DE
:10EDA80004D890B101283DD0042439E003285DD06F
:10EDB800FF28F9D1324CD4F88030D3F80432984780
:10EDC8006369D3F80432984703E0136833F0030209
:10EDD80001D0002424E013F0010F2A4D2A4E0ED052
:10EDE800F3681B681B6968699847246814F0020473
:10EDF8000DD0F368A8691B681B699847E9E7F768AD
:10EE080068693B68DB6898473B689B69EBE7F6688D
:10EE1800A8693368DB6898473368A8699B6998478D
:10EE28002046F8BD1468174D174B24B1DB682869D4
:10EE38001B681B69E1E7DE6828693368DB68984767
:10EE4800336828699B69EAE714680E4D0E4B24B1B4
:10EE5800DB68A8681B681B69CFE7DE68A8683368A9
:10EE6800DB6898473368A8689B69D8E70121074899
:10EE780012F010FB20600028ABD12024D0E700BF9F
:10EE8800203E002078150020649E0208D8510020FA
:10EE98000146014812F0B4BBD851002010B5034810
:10EEA800144612F0B8F9206010BD00BFD8510020F8
:10EEB800014812F0A2B900BFD851002008B5034B91
:10EEC80003485A6A12F0D6FA002008BD78150020C7
:10EED800D851002008B5034B03485A6A12F0AEFA1D
:10EEE800002008BD78150020D851002008B5002161
:10EEF800024812F085FA002008BD00BFD851002052
:10EF080008B54942024812F07BFA002008BD00BF4C
:10EF1800D851002008B5024812F072FA002008BD46
:10EF2800D851002038B5094B094CDD6860682B685A
:10EF38009B69984701200DF0C9FD2B6860685B69E3
:10EF48009847044812F031FA012038BD649E02083F
:10EF580078150020D851002038B5094B094CDD68D8
:10EF680060682B689B69984701200DF0AFFD2B68FE
:10EF780060685B699847044812F002FA012038BDBE
:10EF8800649E020878150020D851002070B5114CF5
:10EF98000D4694F86C30012B19D0032B0BBF0022BF
:10EFA80028220C230F2343F0884343F0401343EAFD
:10EFB8004232042112F021F9D4F88030012D0CBF1F
:10EFC800D3F80432D3F80832BDE87040184700225D
:10EFD8000B23E8E7203E00206F2970B5044615464C
:10EFE80000F0058271D8122900F07D8137D80529F3
:10EFF80000F0318117D8022900F00A8107D80029CA
:10F0080000F0EC80012900F0FB800424F0E00329E3
:10F0180000F00D810429F8D1002840F00F81B34B8E
:10F028005B6A2B60E4E00F2900F03C810DD80829C9
:10F0380000F026810E29E8D1002840F02A812021FD
:10F04800AB4812F0E8F84000CDE0102900F032811A
:10F058001129DAD1002840F03B812921FDE0182947
:10F0680000F0808117D8152900F05F8109D813298D
:10F0780000F046811429C8D1002840F0508126218B
:10F08800AEE0162900F05F811729BED1002840F0B4
:10F0980063812E21A4E01B2900F07C8109D819295D
:10F0A80000F069811A29B0D1002840F06D81332120
:10F0B80096E06D2900F07D8100F284816C29A4D14D
:10F0C800002840F0708160218AE07D2900F02D82BF
:10F0D8003ED8752900F0DE8120D8722900F0B2816F
:10F0E8000ED8702900F0988171298ED1002C40F03B
:10F0F8009C8106217E4812F08EF8C0B2286076E026
:10F10800732900F0B58174297FF47FAF002840F09F
:10F11800BB81774B1B68D3F8703182E7782900F000
:10F12800EC810AD8762900F0CE8177297FF46DAF7B
:10F13800002840F0DC815E2152E0792900F0E68168
:10F148007C297FF462AF002840F0E9815C2147E028
:10F15800882900F0298222D8842900F00D8213D84A
:10F168007E2900F0EB8181297FF44FAF01283ED141
:10F178001668002E00F0F88101465D4812F08AF901
:10F188002860A0BB202433E0852900F0FA81862975
:10F198007FF43BAF002840F00182522120E0C829CB
:10F1A800A4D00DD8892900F014828A297FF42DAFC4
:10F1B800002840F024824E4B1B6893F8923130E7C8
:10F1C800D42900F03082D62900F03882D1297FF482
:10F1D8001CAF002840F02182502101E028B93721D6
:10F1E800434812F018F8286002E0012802D00024F1
:10F1F800204670BD372112683D4811F0FEFFF6E742
:10F2080008B92121ECE70128F1D112682121F3E79F
:10F2180028B92421364811F0FEFF0012E3E701283F
:10F22800E5D1106812F0DAF824210246E4E708B9BB
:10F238002221D5E7012C3FF4E8AED8E70128D6D142
:10F2480013682A4C20212A48636211F0E4FF420720
:10F25800CDD5606AE6E728B92821254811F0DBFFFB
:10F268008010C0E70128C2D11268940DA405002CB3
:10F2780040F0EF81282192001D4811F0BEFFB7E74A
:10F288000028D7D10F211A4811F0C5FF00F001005E
:10F29800A9E70128ABD113682021002B0CBF01225C
:10F2A8000222A9E708B925219AE701289FD1126807
:10F2B8002521A1E708B92A21CFE7012897D11268AB
:10F2C800940DA405002C40F0C48192002A21D3E7B4
:10F2D80001288CD11268940DA405002C40F0B98146
:10F2E80092002921C8E728B9272179E77815002055
:10F2F800D851002001287FF47AAF126827217BE7D4
:10F3080008B92B21A9E701287FF471AF1268940D81
:10F31800A405002C40F09D8192002B21ACE7012828
:10F328007FF465AF1268262166E708B92C2157E7F4
:10F3380001287FF45CAF1268930D9B05002B40F009
:10F3480088812C2158E708B92D2149E701287FF445
:10F358004EAF12682D214FE701287FF448AF12689D
:10F368002E2149E708B92F213AE701287FF43FAF5A
:10F3780012682F2140E708B9302131E701287FF4CE
:10F3880036AF1268302137E701287FF430AF1268B2
:10F39800332131E708B9342122E701287FF427AF68
:10F3A8001268342128E701287FF421AF1268602110
:10F3B80022E708B9612113E701287FF418AF126822
:10F3C800612119E728B91C21A34811F024FF001472
:10F3D80009E701287FF40BAF1C219F4811F01BFFA0
:10F3E8002A68C0F3080040EA02421C2104E728B951
:10F3F8001C21994811F00FFFC0B2F4E601287FF4F0
:10F40800F6AE1C21944811F006FF2B6800F47F0229
:10F41800C3F308031A43E8E708B95921E0E60128CD
:10F428007FF4E5AE12685921E6E6012C7FF4DFAEE1
:10F438000621894811F0EFFE2A7820F0FF000243E8
:10F448000621D9E630B90621834811F0E4FEC0F35D
:10F458000720C8E601287FF4CAAE06217E4811F0CD
:10F46800DAFE2B6820F47F421B029BB21A43E7E7BF
:10F4780020B9794B1B68D3F86C31D2E501287FF4A9
:10F48800B6AE12685A21B7E601287FF4B0AE12680A
:10F498005B21B1E630B9704B1B68D3F87031C3F308
:10F4A8000E03BEE501287FF4A2AE6B48126803681C
:10F4B800C2F30E02D3F8703123F4FF4323F07F0325
:10F4C8001A435B2199E620B9634B1B6893F87231A4
:10F4D800A7E501287FF48BAE5F480368D3F8702155
:10F4E8002B6822F47F021B0403F47F03E8E701285A
:10F4F8007FF47DAE12685E217EE608B918216FE6BA
:10F5080001287FF474AE1268182175E608B919212C
:10F5180066E601287FF46BAE126819216CE60128B3
:10F528007FF465AE12685C2166E608B95F2157E68C
:10F5380001287FF45CAE12685F215DE630B90621D0
:10F54800454811F068FEC0F307404CE601287FF4F7
:10F558004EAE0621404811F05EFE2B6820F47F0273
:10F568001B0403F47F0381E707213B4811F053FE96
:10F57800072120F480023FE600287FF45BAE652176
:10F588002EE600287FF433AE0721334811F043FEFE
:10F59800C0F38150431E5842584124E601287FF4A5
:10F5A80026AE1268522127E620B92B4B1B6893F828
:10F5B800903136E501287FF41AAE274812680368AF
:10F5C80002F00F02D3F8903123F0FF031A436321AE
:10F5D80013E630B9204B1B68D3F89031C3F30323EB
:10F5E8001FE501287FF403AE1B480368D3F8902178
:10F5F8002B6822F470621B0203F47063E6E70128AB
:10F608007FF4F5AD14480368D3F890212B6822F4F1
:10F618007F021B0403F47F03D8E701287FF4E7ADDA
:10F6280012685021E8E518B90B4B1B68DB69F8E450
:10F6380001287FF4DCAD12685321DDE508B91521F6
:10F64800CEE501287FF4D3AD1368044A15215A4347
:10F65800D2E51024CCE500BFD8510020007102008B
:10F668000B4611B901461846B6E408207047F8B5AC
:10F678000027304CA56AE66A2A023302C6B243EA7A
:10F688001563324394F83000E66B3B43A76B0130B7
:10F69800350E360246EA1766C0B23F02C4E90A23AD
:10F6A80084F83000E663A763002940D0042804D911
:10F6B8001A466D21204811F0A0FDA26A6C211E484F
:10F6C80011F09BFD01200DF001FAA26A6C211A4885
:10F6D80011F093FD00230022C4E90E2394F8303082
:10F6E800042B0AD96F21144811F095FDD4E90E2393
:10F6F800002603433243C4E90E236E210E4811F05D
:10F708008AFDD4E90E67034694F8302047EAE3718E
:10F71800C2F10802D200304318F074F90023002225
:10F72800C4E90A230023C4E90E0184F830302846CE
:10F73800F8BD00BF78150020D851002008B5024850
:10F7480011F05EFE002008BDD851002007B50192D7
:10F7580039B9014601AA0120FFF73EFC03B05DF864
:10F7680004FB0820FAE7034B08461B681146DB68D0
:10F77800184700BFD4510020F8B54D4D4D4C4E4BA5
:10F788006A69204600214D4F11F0DDFD4C492046A5
:10F7980011F020FEFE684B4C736803F59C722262E0
:10F7A80003F5AA72E26103F55372A26103F55A7276
:10F7B800626103F56172226103F5687203F5767080
:10F7C800E26003F56F7203F57D7323603368A2600E
:10F7D800DB68606098473368A069DB6898473368DE
:10F7E8006069DB68984733682069DB689847336845
:10F7F800E068DB6898473368A068DB689847336837
:10F8080060685B6998473368A0695B6998473368A3
:10F8180060695B699847336820695B699847336812
:10F82800E0685B6998473368A0685B699847336804
:10F83800206A1B6998473368E0691B6998473368F1
:10F8480020681B6998473A691F4B00211A60736842
:10F8580003F53773536001226B6959701B491A709D
:10F86800C3F804121A492A74C3F80812194B6B66B4
:10F87800194B2B62194BEB61194BAB61194B6B623E
:10F88800194BAB63194B6B63194BAB62194BEB62AA
:10F89800194BAB64194B6B64194B6B65194B2B6592
:10F8A800194BEB65194BAB65194BAB66F8BD00BF3F
:10F8B800203E0020D85100205C960208649E020871
:10F8C80095EF000878150020D451002061EF00085A
:10F8D8002DEF000877F6000845F700081DEF00082F
:10F8E80009EF0008F5EE000869F6000855F700086A
:10F8F800DDEE0008C5EE0008B9EE0008A5EE000828
:10F9080099EE0008A1ED000819ED000825ED0008A2
:10F9180091ED00080022014B5A607047203E0020FC
:10F9280070B5184E184CF56860682B689B69984745
:10F938002B68A0699B6898472B6860699B68984703
:10F948002B6820699B6898472B68E0689B689847F4
:10F958002B68A0689B6898472B68206A9B68984723
:10F968002B68E0699B6898472B6820689B689847D4
:10F978002B6860689B6898473369BDE870405B6A8C
:10F98800184700BF649E0208C81500200A460146B1
:10F99800014811F0F5BE00BF6C5400200228F8B5EC
:10F9A800144653D004D890B101283DD0042439E03E
:10F9B80003285DD0FF28F9D1324CD4F88030D3F831
:10F9C800043298476369D3F80432984703E0136810
:10F9D80033F0030201D0002424E013F0010F2A4D74
:10F9E8002A4E0ED0F3681B681B696869984724681B
:10F9F80014F002040DD0F368A8691B681B699847C6
:10FA0800E9E7F76868693B68DB6898473B689B6982
:10FA1800EBE7F668A8693368DB6898473368A86934
:10FA28009B6998472046F8BD1468174D174B24B1B9
:10FA3800DB6828691B681B69E1E7DE6828693368A9
:10FA4800DB689847336828699B69EAE714680E4DB4
:10FA58000E4B24B1DB68A8681B681B69CFE7DE681A
:10FA6800A8683368DB6898473368A8689B69D8E753
:10FA78000121074811F08EFF20600028ABD1202417
:10FA8800D0E700BF203E0020C8150020649E020871
:10FA98006C5400200146014812F032B86C54002022
:10FAA80010B50348144611F036FE206010BD00BFA3
:10FAB8006C540020014811F020BE00BF6C54002097
:10FAC80008B5034B03485A6A11F054FF002008BDDB
:10FAD800C81500206C54002008B5034B03485A6A27
:10FAE80011F02CFF002008BDC81500206C54002020
:10FAF80008B50021024811F003FF002008BD00BF2F
:10FB08006C54002008B54942024811F0F9FE002063
:10FB180008BD00BF6C54002008B5024811F0F0FE83
:10FB2800002008BD6C54002038B5094B094CDD682D
:10FB380060682B689B69984701200CF0C7FF2B6809
:10FB480060685B699847044811F0AFFE012038BD32
:10FB5800649E0208C81500206C54002038B5094B73
:10FB6800094CDD6860682B689B69984701200CF098
:10FB7800ADFF2B6860685B699847044811F080FE08
:10FB8800012038BD649E0208C81500206C5400206E
:10FB980070B5114C0D4694F86C30012B19D0032B1D
:10FBA8000BBF002228220C230F2343F0884343F085
:10FBB800401343EA4232042111F09FFDD4F880300B
:10FBC800012D0CBFD3F80432D3F80832BDE87040D9
:10FBD800184700220B23E8E7203E00206F2970B564
:10FBE8000446154600F0058271D8122900F07D817F
:10FBF80037D8052900F0318117D8022900F00A8189
:10FC080007D8002900F0EC80012900F0FB800424CB
:10FC1800F0E0032900F00D810429F8D1002840F014
:10FC28000F81B34B5B6A2B60E4E00F2900F03C8145
:10FC38000DD8082900F026810E29E8D1002840F0C7
:10FC48002A812021AB4811F066FD4000CDE0102943
:10FC580000F032811129DAD1002840F03B812921B6
:10FC6800FDE0182900F0808117D8152900F05F8180
:10FC780009D8132900F046811429C8D1002840F07A
:10FC880050812621AEE0162900F05F811729BED1E8
:10FC9800002840F063812E21A4E01B2900F07C811C
:10FCA80009D8192900F069811A29B0D1002840F033
:10FCB8006D81332196E06D2900F07D8100F2848109
:10FCC8006C29A4D1002840F0708160218AE07D2948
:10FCD80000F02D823ED8752900F0DE8120D87229E7
:10FCE80000F0B2810ED8702900F0988171298ED168
:10FCF800002C40F09C8106217E4811F00CFDC0B21A
:10FD0800286076E0732900F0B58174297FF47FAF0D
:10FD1800002840F0BB81774B1B68D3F8703182E72D
:10FD2800782900F0EC810AD8762900F0CE8177296D
:10FD38007FF46DAF002840F0DC815E2152E0792924
:10FD480000F0E6817C297FF462AF002840F0E98169
:10FD58005C2147E0882900F0298222D8842900F014
:10FD68000D8213D87E2900F0EB8181297FF44FAFF3
:10FD780001283ED11668002E00F0F88101465D4842
:10FD880011F008FE2860A0BB202433E0852900F08C
:10FD9800FA8186297FF43BAF002840F00182522186
:10FDA80020E0C829A4D00DD8892900F014828A2916
:10FDB8007FF42DAF002840F024824E4B1B6893F847
:10FDC800923130E7D42900F03082D62900F0388209
:10FDD800D1297FF41CAF002840F02182502101E096
:10FDE80028B93721434811F096FC286002E0012821
:10FDF80002D00024204670BD372112683D4811F01A
:10FE08007CFCF6E708B92121ECE70128F1D112685A
:10FE18002121F3E728B92421364811F07CFC00128F
:10FE2800E3E70128E5D1106811F058FD24210246C6
:10FE3800E4E708B92221D5E7012C3FF4E8AED8E77A
:10FE48000128D6D113682A4C20212A48636211F070
:10FE580062FC4207CDD5606AE6E728B92821254823
:10FE680011F059FC8010C0E70128C2D11268940D26
:10FE7800A405002C40F0EF81282192001D4811F0C4
:10FE88003CFCB7E70028D7D10F211A4811F043FCF2
:10FE980000F00100A9E70128ABD113682021002B4D
:10FEA8000CBF01220222A9E708B925219AE70128F7
:10FEB8009FD112682521A1E708B92A21CFE7012897
:10FEC80097D11268940DA405002C40F0C4819200CB
:10FED8002A21D3E701288CD11268940DA405002C9F
:10FEE80040F0B98192002921C8E728B9272179E78C
:10FEF800C81500206C54002001287FF47AAF1268DE
:10FF080027217BE708B92B21A9E701287FF471AFE6
:10FF18001268940DA405002C40F09D8192002B21BD
:10FF2800ACE701287FF465AF1268262166E708B9B7
:10FF38002C2157E701287FF45CAF1268930D9B05CD
:10FF4800002B40F088812C2158E708B92D2149E77A
:10FF580001287FF44EAF12682D214FE701287FF466
:10FF680048AF12682E2149E708B92F213AE701283E
:10FF78007FF43FAF12682F2140E708B9302131E7FD
:10FF880001287FF436AF1268302137E701287FF463
:10FF980030AF1268332131E708B9342122E701284C
:10FFA8007FF427AF1268342128E701287FF421AFB6
:10FFB8001268602122E708B9612113E701287FF45C
:10FFC80018AF1268612119E728B91C21A34811F05C
:10FFD800A2FB001409E701287FF40BAF1C219F48FE
:10FFE80011F099FB2A68C0F3080040EA02421C217C
:08FFF80004E728B91C21994817
:020000040801F1
:1000000011F08DFBC0B2F4E601287FF4F6AE1C219E
:10001000944811F084FB2B6800F47F02C3F30803BB
:100020001A43E8E708B95921E0E601287FF4E5AE74
:1000300012685921E6E6012C7FF4DFAE06218948DB
:1000400011F06DFB2A7820F0FF0002430621D9E66B
:1000500030B90621834811F062FBC0F30720C8E6DF
:1000600001287FF4CAAE06217E4811F058FB2B68A8
:1000700020F47F421B029BB21A43E7E720B9794B79
:100080001B68D3F86C31D2E501287FF4B6AE126854
:100090005A21B7E601287FF4B0AE12685B21B1E6C1
:1000A00030B9704B1B68D3F87031C3F30E03BEE553
:1000B00001287FF4A2AE6B4812680368C2F30E02F7
:1000C000D3F8703123F4FF4323F07F031A435B21FD
:1000D00099E620B9634B1B6893F87231A7E50128B4
:1000E0007FF48BAE5F480368D3F870212B6822F44D
:1000F0007F021B0403F47F03E8E701287FF47DAE51
:1001000012685E217EE608B918216FE601287FF4A7
:1001100074AE1268182175E608B9192166E601283F
:100120007FF46BAE126819216CE601287FF465AE8E
:1001300012685C2166E608B95F2157E601287FF462
:100140005CAE12685F215DE630B90621454811F0CA
:10015000E6FAC0F307404CE601287FF44EAE0621D4
:10016000404811F0DCFA2B6820F47F021B0403F4F2
:100170007F0381E707213B4811F0D1FA072120F4E2
:1001800080023FE600287FF45BAE65212EE6002862
:100190007FF433AE0721334811F0C1FAC0F3815028
:1001A000431E5842584124E601287FF426AE1268C7
:1001B000522127E620B92B4B1B6893F8903136E586
:1001C00001287FF41AAE27481268036802F00F0274
:1001D000D3F8903123F0FF031A43632113E630B9BB
:1001E000204B1B68D3F89031C3F303231FE501288C
:1001F0007FF403AE1B480368D3F890212B6822F4E8
:1002000070621B0203F47063E6E701287FF4F5AD2A
:1002100014480368D3F890212B6822F47F021B0452
:1002200003F47F03D8E701287FF4E7AD126850217B
:10023000E8E518B90B4B1B68DB69F8E401287FF48B
:10024000DCAD12685321DDE508B91521CEE50128A2
:100250007FF4D3AD1368044A15215A43D2E5102424
:10026000CCE500BF6C540020007102000B4611B9B0
:1002700001461846B6E408207047F8B50027304C10
:10028000A56AE66A2A023302C6B243EA156332431C
:1002900094F83000E66B3B43A76B0130350E360215
:1002A00046EA1766C0B23F02C4E90A2384F8300068
:1002B000E663A763002940D0042804D91A466D21BB
:1002C000204811F01EFAA26A6C211E4811F019FA9A
:1002D00001200CF0FFFBA26A6C211A4811F011FA00
:1002E00000230022C4E90E2394F83030042B0AD9ED
:1002F0006F21144811F013FAD4E90E2300260343AA
:100300003243C4E90E236E210E4811F008FAD4E9F5
:100310000E67034694F8302047EAE371C2F1080201
:10032000D200304317F072FB00230022C4E90A23F5
:100330000023C4E90E0184F830302846F8BD00BF20
:10034000C81500206C54002008B5024811F0DCFAF2
:10035000002008BD6C54002007B5019239B9014650
:1003600001AA0120FFF73EFC03B05DF804FB082062
:10037000FAE7034B08461B681146DB68184700BFC5
:1003800000570020F8B54D4D4D4C4E4B6A69204644
:1003900000214D4F11F05BFA4C49204611F09EFAB6
:1003A000FE684B4C736803F59C72226203F5AA72D7
:1003B000E26103F55372A26103F55A72626103F5BB
:1003C0006172226103F5687203F57670E26003F5ED
:1003D0006F7203F57D7323603368A260DB68606031
:1003E00098473368A069DB68984733686069DB68C1
:1003F000984733682069DB6898473368E068DB68B2
:1004000098473368A068DB689847336860685B6921
:1004100098473368A0695B699847336860695B698E
:100420009847336820695B6998473368E0685B697F
:1004300098473368A0685B6998473368206A1B69EE
:1004400098473368E0691B699847336820681B69DF
:1004500098473A691F4B00211A60736803F5377398
:10046000536001226B6959701B491A70C3F804125A
:100470001A492A74C3F80812194B6B66194B2B6280
:10048000194BEB61194BAB61194B6B62194BAB63A9
:10049000194B6B63194BAB62194BEB62194BAB6495
:1004A000194B6B64194B6B65194B2B65194BEB653D
:1004B000194BAB65194BAB66F8BD00BF203E002061
:1004C0006C5400205C980208649E020899FB0008A6
:1004D000C81500200057002065FB000831FB00080C
:1004E0007B0201084903010821FB00080DFB0008FD
:1004F000F9FA00086D02010859030108E1FA000841
:10050000C9FA0008BDFA0008A9FA00089DFA000817
:10051000A5F900081DF9000829F9000895F9000857
:1005200000207047012070470022014B5A6070473D
:10053000203E00201FB5084B33F8084C5A7802942F
:100540009C1E019433F8041C00910146002011F018
:1005500053FD04B010BD00BF0C57002010B50020A3
:10056000144611F017FB206010BD002011F034BBC1
:1005700010B5044620B9096811F03BFC204610BDB7
:10058000082010BD10B5044618B911F025FC20460E
:1005900010BD082010BD38B50D46044620B911F035
:1005A00016FC2860204638BD082038BD10B504462A
:1005B00018B911F0F3FB204610BD082010BD002132
:1005C000F4E74942F2E7F1E7022804BF0B4B93F846
:1005D000D80030B90A4BDB681B689B69094A106870
:1005E0001847012809D1054B93F8D830012B04D1C5
:1005F000034BDB681B685B69F0E77047203E002017
:10060000649E02081457002010B50020FFF7DCFF9D
:10061000BDE81040034B044ADB6810681B689B6907
:10062000184700BF649E020814570020043A70B5B2
:1006300004460D461E46FA2A00F2F087DFE812F063
:10064000FB00EE07EE07EE07EE07EE07EE07EE07FC
:10065000EE07EE07EE07EE07EE07EE07EE07EE07F2
:10066000EE07EE07EE07EE07EE07EE07EE07EE07E2
:10067000EE07EE07EE07EE07EE07EE07EE07EE07D2
:10068000EE07EE07EE07EE07EE07EE07EE07EE07C2
:10069000EE07EE07EE07EE07EE07EE070D0121016C
:1006A000EE0735014901EE07EE07EE07EE07EE070C
:1006B000EE07EE07EE07EE07EE07EE07EE07EE0792
:1006C000EE07EE07EE07EE07EE07EE07EE07EE0782
:1006D000EE07EE07EE07EE07EE07EE07EE07EE0772
:1006E000EE07EE07EE07EE07EE07EE07EE07EE0762
:1006F000EE07EE07EE07EE07EE07EE07EE07EE0752
:100700005D016F017D018B019901A701B501C30155
:10071000D101DF01ED01FC010B021A0229023802AE
:10072000470252025D02EE07680273027E028902EE
:100730009402A402B402C402CE02EE07EE07EE0752
:10074000D802E102EA02F5020003EE07EE07EE0727
:10075000090312031B03EE07EE07EE07EE07EE0791
:10076000EE07EE07260331033C034703EE07EE07CF
:10077000EE07EE07EE07EE0752035D03680373030F
:100780007E03EE07EE07EE07EE07EE0789039403FC
:10079000A803BC03C503D503E003EC03F703FF0381
:1007A0000E041C042A043804460454046204700431
:1007B000EE077E048D04A404B204C104CF04DD045A
:1007C000EB04F904080519052A053B054C055D05F0
:1007D000700581059205A305B405C505D605E70595
:1007E000F80509061A062B063C064D065D06EE07BF
:1007F000EE07EE07EE07EE07EE07EE07EE07EE0751
:10080000EE07EE076D067E068F06A006B106C2064D
:10081000D306E406F506050715072507350745073E
:1008200055076507750784079307A207EE07B10709
:10083000C307DA07E40730B96021284611F0AAF9A6
:100840003060204670BD012840F0EB8632686021A0
:10085000284611F0C1F90024F3E738B9024608210F
:10086000284611F0D9F900B23060EAE7012840F0DB
:10087000DB86338800220821284611F0DAF90024AB
:10088000DFE738B902460921284611F0C5F900B260
:100890003060D6E7012840F0CA863388002209215B
:1008A000284611F0C6F90024CBE738B90122082107
:1008B000284611F0B1F900B23060C2E7012840F0DB
:1008C000B986024633880821284611F0B2F900247F
:1008D000B7E738B901220921284611F09DF900B285
:1008E0003060AEE7012840F0A8860246338809212F
:1008F000284611F09EF90024A3E758B901220321EC
:10090000284611F069F922460221284611F084F99F
:10091000306096E7012C14BF0024042491E70028DE
:10092000F8D101220321284611F056F901220221B3
:10093000284611F071F9306083E70028EAD10222DD
:100940000321284611F048F922460221284611F0D9
:1009500063F9306075E70028DCD1024603212846A0
:1009600011F03AF922460221284611F055F930607B
:1009700067E70028CED102460321284611F02CF962
:1009800001220221284611F047F9306059E700287A
:10099000C0D103222846114611F01EF92246022139
:1009A000284611F039F930604BE70028B2D1042213
:1009B0000321284611F010F922460221284611F0A1
:1009C0002BF930603DE70028A4D1042203212846FA
:1009D00011F002F901220221284611F01DF93060C0
:1009E0002FE7002896D105220321284611F0F4F8BC
:1009F00022460221284611F00FF9306021E7002835
:100A000088D105220321284611F0E6F801220221AF
:100A1000284611F001F9306013E700287FF47AAF1F
:100A200006220321284611F0D7F822460221284643
:100A300011F0F2F8306004E700287FF46BAF072272
:100A40000321284611F0C8F822460221284611F059
:100A5000E3F83060F5E600287FF45CAF072203215D
:100A6000284611F0B9F801220221284611F0D4F8E5
:100A70003060E6E600287FF44DAF082203212846C7
:100A800011F0AAF822460221284611F0C5F830607C
:100A9000D7E600287FF43EAF08220321284611F054
:100AA0009BF801220221284611F0B6F83060C8E612
:100AB00000287FF42FAF09220321284611F08CF87B
:100AC00022460221284611F0A7F83060B9E6002836
:100AD0007FF420AF02461221284611F09DF800B2A3
:100AE0003060AEE600287FF415AF012212212846BF
:100AF00011F092F800B23060A3E600287FF40AAF4C
:100B000002461321284611F087F800B2306098E6BB
:100B100000287FF4FFAE02461521284611F07CF82C
:100B200000B230608DE600287FF4F4AE012215217A
:100B3000284611F071F800B2306082E600287FF498
:100B4000E9AE02461621284611F066F800B2306080
:100B500077E600287FF4DEAE01221621284611F048
:100B60005BF800B230606CE600287FF4D3AE0A2256
:100B70000321284611F030F822460221284611F0C0
:100B80004BF800B230605CE600287FF4C3AE0A2266
:100B90000321284611F020F801220221284611F0F5
:100BA0003BF800B230604CE600287FF4B3AE0B2275
:100BB0000321284611F010F822460221284611F0A0
:100BC0002BF800B230603CE600287FF4A3AE02466A
:100BD0000621284611F020F8306032E600287FF424
:100BE00099AE01220621284611F016F8306028E659
:100BF00000287FF48FAE4121284610F0CBFF3060F3
:100C00001FE600287FF486AE4221284610F0C2FF7E
:100C1000306016E600287FF47DAE0122462128468A
:100C200010F0FAFF00B230600BE600287FF472AEDD
:100C300002464621284610F0EFFF00B2306000E681
:100C400000287FF467AE4721284610F0A3FF3060EC
:100C5000F7E500287FF45EAE2121284610F09AFFC8
:100C60003060EEE500287FF455AE2221284610F0D2
:100C700091FF3060E5E500287FF44CAE0246232169
:100C8000284610F0C9FF00B23060DAE500287FF492
:100C900041AE2721284610F07DFF20F07F403060D4
:100CA000CFE500287FF436AE2821284610F072FFE9
:100CB00020F07F403060C4E500287FF42BAE012295
:100CC0002A21284610F0A8FF00B23060B9E50028BC
:100CD0007FF420AE02462A21284610F09DFF00B284
:100CE0003060AEE500287FF415AE02463921284673
:100CF00010F092FF00B23060A3E500287FF40AAE46
:100D000001223921284610F087FF00B2306098E5B3
:100D100000287FF4FFAD02463D21284610F07CFFFD
:100D200000B230608DE500287FF4F4AD02463F212B
:100D3000284610F071FF00B2306082E500287FF491
:100D4000E9AD02463A21284610F066FF00B2306055
:100D500077E500287FF4DEAD02465321284610F0E7
:100D60005BFF00B230606CE538B90122642128468F
:100D700010F052FF00B2306063E5012840F060845B
:100D8000024633886421284610F053FF002458E5BA
:100D900038B902466421284610F03EFF00B23060A8
:100DA0004FE5012840F04F84338800226421284613
:100DB00010F03FFF002444E500287FF4ABAD66212E
:100DC000284610F0E7FE30603BE528B96821284648
:100DD00010F0E0FE306034E5012840F037843168DF
:100DE000284610F0F9FF00242BE500287FF492AD8F
:100DF00001226921284610F00FFF00B2306020E583
:100E000000287FF487ADC54B284603EB01135989B1
:100E100010F074FF306014E500287FF47BAD0246CB
:100E20006921284610F0F8FE00B2306009E500287C
:100E30007FF470AD084610F0CAFF306001E520B9BC
:100E4000084610F0EEFF3060FBE4012840F001841A
:100E50003168284610F0E1FF0024F2E400287FF416
:100E600059AD02466D21284610F0B6FE6C21284689
:100E700010F090FE3060E4E400287FF44BAD0122D6
:100E80006D21284610F0A8FE6C21284610F082FE45
:100E90003060D6E400287FF43DAD02226D21284663
:100EA00010F09AFE6C21284610F074FE3060C8E401
:100EB00000287FF42FAD03226D21284610F08CFE10
:100EC0006C21284610F066FE3060BAE400287FF4FA
:100ED00021AD04226D21284610F07EFE6C212846AB
:100EE00010F058FE3060ACE400287FF413AD05220A
:100EF0006D21284610F070FE6C21284610F04AFE45
:100F000030609EE400287FF405AD06226D2128465E
:100F100010F062FE6C21284610F03CFE306090E438
:100F200000287FF4F7AC07226D21284610F054FE0C
:100F30006C21284610F02EFE306082E420B908466D
:100F400010F0ACFE30607CE4012840F0858331680D
:100F5000284610F095FE002473E440B96F4B2846F4
:100F600003EB0113598910F0BFFE306069E40128DA
:100F700040F07583694B326803EB011359892846A9
:100F800010F0A0FE00245CE400287FF4C3AC012232
:100F90006F21284610F020FE6E21284610F0FAFD41
:100FA00030604EE420B9084610F005FF306048E498
:100FB000012840F057833168284610F0EFFE0024E6
:100FC0003FE400287FF4A6AC03226F21284610F0EE
:100FD00003FE6E21284610F0DDFD306031E400286C
:100FE0007FF498AC04226F21284610F0F5FD6E21A5
:100FF000284610F0CFFD306023E400287FF48AAC4F
:1010000005226F21284610F0E7FD6E21284610F0DA
:10101000C1FD306015E400287FF47CAC06226F210E
:10102000284610F0D9FD6E21284610F0B3FD30603F
:1010300007E400287FF46EAC07226F21284610F0E9
:10104000CBFD6E21284610F0A5FD3060FFF7F9BBFF
:1010500000287FF45FAC08226F21284610F0BCFD09
:1010600022466E21284610F0D7FD00B23060FFF70F
:10107000E8BB00287FF44EAC08226F21284610F010
:10108000ABFD01226E21284610F0C6FD00B2306093
:10109000FFF7D7BB00287FF43DAC09226F2128461B
:1010A00010F09AFD22466E21284610F0B5FD00B2E0
:1010B0003060FFF7C6BB00287FF42CAC0A226F21FA
:1010C000284610F089FD22466E21284610F0A4FD26
:1010D00000B23060FFF7B5BB00287FF41BAC0A22DA
:1010E0006F21284610F078FD01226E21284610F06D
:1010F00093FD00B23060FFF7A4BB00287FF40AAC78
:101100000B226F21284610F067FD22466E212846EB
:1011100010F082FD00B23060FFF793BB045700204F
:1011200000287FF4F7AB0B226F21284610F054FD06
:1011300001226E21284610F06FFD00B23060FFF7EB
:1011400080BB00287FF4E6AB0C226F21284610F00C
:1011500043FD22466E21284610F05EFD00B230604D
:10116000FFF76FBB00287FF4D5AB0C226F21284618
:1011700010F032FD01226E21284610F04DFD00B224
:101180003060FFF75EBB00287FF4C4AB0D226F21F7
:10119000284610F021FD22466E21284610F03CFD25
:1011A00000B23060FFF74DBB00287FF4B3AB0D22D7
:1011B0006F21284610F010FD01226E21284610F004
:1011C0002BFD00B23060FFF73CBB00287FF4A2ABE0
:1011D0000E226F21284610F0FFFC22466E21284681
:1011E00010F01AFD00B23060FFF72BBB00287FF42F
:1011F00091AB0E226F21284610F0EEFC01226E21E9
:10120000284610F009FD00B23060FFF71ABB002835
:101210007FF480AB0F226F21284610F0DDFC2246C0
:101220006E21284610F0F8FC00B23060FFF709BBD1
:1012300000287FF46FAB0F226F21284610F0CCFC02
:1012400001226E21284610F0E7FC00B23060FFF763
:10125000F8BA00287FF45EAB10226F21284610F008
:10126000BBFC22466E21284610F0D6FC00B230604E
:10127000FFF7E7BA00287FF44DAB11226F21284613
:1012800010F0AAFC22466E21284610F0C5FC00B2E0
:101290003060FFF7D6BA00287FF43CAB11226F21F3
:1012A000284610F099FC01226E21284610F0B4FC6B
:1012B00000B23060FFF7C5BA00287FF42BAB1222D2
:1012C0006F21284610F088FC22466E21284610F037
:1012D000A3FC00B23060FFF7B4BA00287FF41AAB69
:1012E00013226F21284610F077FC22466E212846F3
:1012F00010F092FC3060FFF7A4BA00287FF40AAB2C
:1013000013226F21284610F067FC01226E21284627
:1013100010F082FC3060FFF794BA00287FF4FAAA3C
:10132000C0226F21284610F057FC22466E21284625
:1013300010F072FC00B23060FFF783BA00287FF42F
:10134000E9AAC0226F21284610F046FC01226E2136
:10135000284610F061FC00B23060FFF772BA002836
:101360007FF4D8AAC1226F21284610F035FC22460E
:101370006E21284610F050FC00B23060FFF761BAD1
:1013800000287FF4C7AAC1226F21284610F024FC50
:1013900001226E21284610F03FFC00B23060FFF7BA
:1013A00050BA00287FF4B6AAC2226F21284610F056
:1013B00013FC22466E21284610F02EFC00B230604D
:1013C000FFF73FBA00287FF4A5AAC2226F21284662
:1013D00010F002FC01226E21284610F01DFC00B224
:1013E0003060FFF72EBA00287FF494AAC3226F2141
:1013F000284610F0F1FB22466E21284610F00CFC26
:1014000000B23060FFF71DBA00287FF483AAC32220
:101410006F21284610F0E0FB01226E21284610F0D3
:10142000FBFB00B23060FFF70CBA00287FF472AA11
:10143000C4226F21284610F0CFFB22466E21284699
:1014400010F0EAFB3060FFF7FCB900287FF462AAD5
:10145000C4226F21284610F0BFFB01226E212846CE
:1014600010F0DAFB3060FFF7ECB900287FF452AAE5
:10147000C5226F21284610F0AFFB22466E21284678
:1014800010F0CAFB3060FFF7DCB900287FF442AAF5
:10149000C5226F21284610F09FFB01226E212846AD
:1014A00010F0BAFB3060FFF7CCB900287FF432AA05
:1014B000C6226F21284610F08FFB22466E21284657
:1014C00010F0AAFB3060FFF7BCB900287FF422AA15
:1014D000C6226F21284610F07FFB01226E2128468C
:1014E00010F09AFB3060FFF7ACB900287FF412AA25
:1014F000C7226F21284610F06FFB22466E21284636
:1015000010F08AFB3060FFF79CB900287FF402AA34
:10151000C7226F21284610F05FFB01226E2128466A
:1015200010F07AFB3060FFF78CB900287FF4F2A945
:10153000C8226F21284610F04FFB6E21284610F07C
:1015400029FB3060FFF77DB900287FF4E3A9C922A9
:101550006F21284610F040FB6E21284610F01AFB40
:101560003060FFF76EB900287FF4D4A9CA226F213A
:10157000284610F031FB6E21284610F00BFB30603E
:10158000FFF75FB900287FF4C5A9CB226F21284659
:1015900010F022FB6E21284610F0FCFA3060FFF7B5
:1015A00050B930B9344901EB05156B893360FFF749
:1015B00048B9012859D13049336801EB05156B81D1
:1015C0000024FFF73EB930B92B4901EB05156B7AC2
:1015D0003360FFF736B901284AD10D01264905F1DC
:1015E000080209350A443078294410F00FFD002420
:1015F000FFF727B900287FF48DA91F4901EB0515D6
:101600002B7A3360FFF71DB900287FF483A91A49AC
:1016100001EB0515EB883360FFF713B90424FFF7DE
:1016200010B90024FFF70DB90024FFF70AB9002410
:10163000FFF707B90024FFF704B90024FFF701B949
:101640000024FFF7FEB80024FFF7FBB80024FFF7E3
:10165000F8B80024FFF7F5B80024FFF7F2B800242B
:10166000FFF7EFB80024FFF7ECB80024FFF7E9B864
:101670000024FFF7E6B800BF0457002010B413465B
:101680000446084619B9224610BCFEF7CFBF082011
:1016900010BC70470120704707B5019239B9024666
:1016A00001AB0120FEF7C2FF03B05DF804FB082088
:1016B000FAE710B40C4630B9044B20461B681146BB
:1016C0009B6810BC1847002010BC704718570020BA
:1016D00070B52B4D2B4EEC6860682368C8303060C5
:1016E000DB689847236830685B6998472A69264B0E
:1016F00026491A606368012003F537735360244B51
:101700005A690A602349C2F804122349C2F8081230
:10171000002111705170214A18741A62204ADA614E
:10172000204A9A61204A5A62204ADA64204A9A631F
:10173000204A5A63204A9A62204ADA62204A9A640E
:10174000204A5A64204A5A65204A1A65204A1A6675
:10175000204ADA65204A9A653222DA6040F28A220B
:101760009A604FF47A721D4B9A8041F270721A603F
:101770004FF4807259725A81BDE87040FEF724BF61
:10178000649E020814570020185700201C570020A0
:10179000203E00209516010825050108AD05010829
:1017A000C7050108C3050108BF0501089705010821
:1017B0007D160108991601088505010871050108C3
:1017C0006B0501085D0501083505010821050108C3
:1017D000C905010829050108090601080457002068
:1017E00000207047012070470022014B5A6070476B
:1017F000203E0020002010F039BC7FB50646234B68
:10180000234C33F8060C5A780290981E019033F856
:10181000041C00200091314610F046FE23689E42D1
:1018200015D01C4B1B78032B28D0022B11D0012B79
:101830000CD16B21002010F0F7FB174D0246A86079
:101840006821002010F012FC0023EB61266004B038
:1018500070BD114D28460EF09BFB6B21002010F04F
:10186000E3FB68210246A860002010F0FFFB002087
:1018700066212A69E86110F0F9FBE7E7064D284682
:101880000EF0B8FBAA6868210020F4E70A57002090
:10189000141600204C5700202057002010B50020BF
:1018A000144610F0C1FB206010BD38B50D4604464B
:1018B00020B910F0E3FC2860204638BD082038BD70
:1018C000022804BF0B4B93F8D80030B90A4BDB68F1
:1018D0001B689B69094A10681847012809D1054B04
:1018E00093F8D830012B04D1034BDB681B685B698C
:1018F000F0E77047203E0020649E02081457002045
:1019000010B50020FFF7DCFFBDE81040034B044A90
:10191000DB6810681B689B69184700BF649E02085B
:101920001457002070B50E46A8B90C4C0C4D227807
:10193000012A02D110F0A2FC2861032100202170AD
:1019400010F0D8FB6B21002010F06EFB33681844B8
:101950006860002070BD082070BD00BF4C5700209B
:101960002057002070B50E4678B9094C094D2278F1
:10197000012A02D110F082FC28610321002021708D
:1019800010F0B8FB6E60002070BD082070BD00BF75
:101990004C5700202057002070B50E4678B9094CEE
:1019A000094D2278012A02D110F068FC2861022139
:1019B0000020217010F09EFBEE60002070BD08201A
:1019C00070BD00BF4C570020205700200021E3E7E6
:1019D0004942E1E7E0E7043A70B504460D461E4689
:1019E000FA2A01F21081DFE812F0FB000E090E095D
:1019F0000E090E090E090E091701320146010E09E2
:101A00000E090E090E090E090E090E090E090E091E
:101A10000E090E090E090E090E090E090E090E090E
:101A20000E090E090E090E090E090E090E090E09FE
:101A30000E090E090E090E090E090E090E090E09EE
:101A40000E090E090E094F0161010E09730186018D
:101A50000E090E090E090E090E090E090E090E09CE
:101A60000E090E090E090E090E090E090E090E09BE
:101A70000E090E090E090E090E090E090E090E09AE
:101A80000E090E090E090E090E090E090E090E099E
:101A90000E090E090E090E090E090E090E090E098E
:101AA0000E090E090E090E090E099A01AC01BA01C0
:101AB0000E090E090E090E090E090E090E090E096E
:101AC000C801D601E4010E090E09F201FC0106026B
:101AD0000E0910021A0224020E092E023D020E09FE
:101AE0004C0256020E090E090E0960026B027402C6
:101AF0007F028A020E090E090E0993029C02A502BA
:101B00000E090E090E090E090E090E090E09B00282
:101B1000BB02C602D102DC02F702120330034E03FD
:101B20006C03890394039F03AA03B5030E090E09EE
:101B30000E090E090E09C003CB03DF03F303FC03F8
:101B4000050410041D0428043004520460046E04CB
:101B50007C048A049804A604B4040E09C204D104C7
:101B6000EC04FA0409051805270536054505540552
:101B70006505760587059805AF05C005D105E20521
:101B8000F3050406150626063706480659066A06B2
:101B90007B068C069D06AD060E09BD06DA06F70625
:101BA00017073707570777070E090E090E0986072B
:101BB0009707A807B907CA07DB07EC07FD070E0858
:101BC0001E082E083E084E085E086E087E088E0825
:101BD0009D08AC08BB080E09CA08DF08F80803090D
:101BE00050B96021284610F01FFA24214D43B34B11
:101BF00030605851204670BD012801D00024F9E71B
:101C000032686021284610F031FA24214D433268B1
:101C1000AA4B00245A51EDE750B95F21284610F035
:101C200003FA2421A54B306001FB05356861E1E72B
:101C30000128E3D132685F21284610F017FA2421E9
:101C40009E4A336801FB052500246B61D2E738B951
:101C500024219A4B01FB053595F820303360C9E704
:101C60000128CBD12421954B002401FB0535336895
:101C700085F82030BEE70028C0D124218F4B01FB1E
:101C800005352B693360B5E730B90246082128468F
:101C900010F00CFA3060ADE70128AFD13388002294
:101CA0000821284610F00FFA0024A3E730B90246B5
:101CB0000921284610F0FAF930609BE701289DD1F0
:101CC000338800220921284610F0FDF9002491E70D
:101CD00038B901220821284610F0E8F900B2306036
:101CE00088E701288AD1024633880821284610F067
:101CF000EAF900247EE738B901220921284610F0CC
:101D0000D5F900B2306075E701287FF477AF02465D
:101D100033880921284610F0D6F900246AE758B91B
:101D200001220321284610F0A1F92246022128466B
:101D300010F0BCF930605DE7012C7FF45FAF042444
:101D400058E70028F8D101220321284610F08EF927
:101D500001220221284610F0A9F930604AE7002844
:101D6000EAD102220321284610F080F922460221FE
:101D7000284610F09BF930603CE70028DCD10222B5
:101D80000321284610F072F901220221284610F0A2
:101D90008DF930602EE70028CED103222846114667
:101DA00010F064F901220221284610F07FF930601A
:101DB00020E70028C0D103222846114610F056F92A
:101DC00022460221284610F071F9306012E70028FF
:101DD000B2D102461221284610F068F900B23060F4
:101DE00008E70028A8D101221221284610F05EF948
:101DF00000B23060FEE600289ED10246132128463C
:101E000010F054F900B23060F4E6002894D1024694
:101E10001521284610F04AF900B23060EAE60028A1
:101E20008AD101221521284610F040F900B2306015
:101E3000E0E6002880D102461621284610F036F947
:101E400000B23060D6E600287FF476AF0246032168
:101E5000284610F00BF922460221284610F026F9F8
:101E60003060C7E600287FF467AF024603212846AA
:101E700010F0FCF801220221284610F017F930601A
:101E8000B8E600287FF458AF02460B21284610F030
:101E90000DF93060AEE600287FF44EAF01220B2131
:101EA000284610F003F93060A4E600287FF444AF20
:101EB0004121284610F0B8F830609BE620570020FA
:101EC00000287FF439AF4221284610F0ADF8306089
:101ED00090E600287FF430AF01224621284610F01A
:101EE000E5F800B2306085E600287FF425AF0246B1
:101EF0004621284610F0DAF800B230607AE6002871
:101F00007FF41AAF4721284610F08EF8306071E652
:101F100000287FF411AF2121284610F085F83060A9
:101F200068E600287FF408AF2221284610F07CF8EC
:101F300030605FE600287FF4FFAE0246232128468A
:101F400010F0B4F800B2306054E600287FF4F4AE2C
:101F50002721284610F068F820F07F40306049E6DD
:101F600000287FF4E9AE2821284610F05DF820F023
:101F70007F4030603EE600287FF4DEAE01222A2159
:101F8000284610F093F800B2306033E600287FF462
:101F9000D3AE02462A21284610F088F800B23060FD
:101FA00028E650B9D4226F21284610F05FF86E2140
:101FB000284610F039F830601CE601287FF41EAE88
:101FC000D4226F21284610F051F832686E2128463D
:101FD00010F04CF800240DE650B9D5226F212846A8
:101FE00010F044F86E21284610F01EF8306001E62B
:101FF00001287FF403AED5226F21284610F036F871
:1020000032686E21284610F031F80024F2E560B9FC
:10201000D6226F21284610F029F822466E21284644
:1020200010F044F800B23060E4E501287FF4E6AD3A
:10203000D6226F21284610F019F8338800226E212D
:10204000284610F040F80024D4E560B9D6226F216C
:10205000284610F00BF801226E21284610F026F8D1
:1020600000B23060C6E501287FF4C8ADD6226F21EA
:1020700028460FF0FBFF224633886E21284610F0D9
:1020800022F80024B6E560B9D7226F2128460FF068
:10209000EDFF22466E21284610F008F800B23060AD
:1020A000A8E501287FF4AAADD7226F2128460FF0BA
:1020B000DDFF338800226E21284610F004F800244A
:1020C00098E558B9D7226F2128460FF0CFFF01229B
:1020D0006E2128460FF0EAFF30608BE501287FF47F
:1020E0008DADD7226F2128460FF0C0FF22463388DE
:1020F0006E2128460FF0E7FF00247BE500287FF4DF
:102100001BAE0246392128460FF0D0FF00B23060E6
:1021100070E500287FF410AE0122392128460FF027
:10212000C5FF00B2306065E500287FF405AE0246C9
:102130003D2128460FF0BAFF00B230605AE5002872
:102140007FF4FAAD02463F2128460FF0AFFF00B200
:1021500030604FE500287FF4EFAD02463A21284673
:102160000FF0A4FF00B2306044E500287FF4E4AD36
:102170000246532128460FF099FF00B2306039E53E
:1021800038B90122642128460FF090FF00B2306078
:1021900030E501287FF432AD0246338864212846B9
:1021A0000FF091FF002425E538B902466421284646
:1021B0000FF07CFF00B230601CE501287FF41EADFB
:1021C00033880022642128460FF07DFF002411E5AA
:1021D00000287FF4B1AD662128460FF025FF30605E
:1021E00008E500287FF4A8AD682128460FF01CFF01
:1021F0003060FFE400287FF49FAD0122692128466A
:102200000FF054FF00B23060F4E400287FF494AD86
:102210000C23CA4A284603FB012319890FF0C3FF88
:102220003060E7E400287FF487AD02466921284644
:102230000FF03CFF00B23060DCE400287FF47CAD9E
:10224000084610F01BF83060D4E420B9084610F0BE
:102250003FF83060CEE401287FF4D0AC32686B21C7
:1022600028460FF003FFB64B5B5D032B7FF4C6AC33
:102270002423B449326803FB05135A60326868218D
:102280009A60326828460FF0F1FE0024B2E400287C
:102290007FF452AD02466D2128460FF0E7FE6C2117
:1022A00028460FF0C1FE3060A4E400287FF444AD5E
:1022B00001226D2128460FF0D9FE6C2128460FF02F
:1022C000B3FE306096E400287FF436AD02226D2123
:1022D00028460FF0CBFE6C2128460FF0A5FE30609B
:1022E00088E400287FF428AD03226D2128460FF0F2
:1022F000BDFE6C2128460FF097FE30607AE400287E
:102300007FF41AAD04226D2128460FF0AFFE6C2138
:1023100028460FF089FE30606CE400287FF40CAD95
:1023200005226D2128460FF0A1FE6C2128460FF0F2
:102330007BFE30605EE400287FF4FEAC06226D2157
:1023400028460FF093FE6C2128460FF06DFE30609A
:1023500050E400287FF4F0AC07226D2128460FF0EE
:1023600085FE6C2128460FF05FFE306042E420B904
:1023700008460FF0DDFE30603CE401287FF43EACFF
:10238000316828460FF0C6FE002433E448B90C2318
:102390006A4A284603FB012319890FF0FAFE3060D0
:1023A00028E401287FF42AAC0C23644A284603FB66
:1023B0000123326819890FF0DAFE614B5C55002465
:1023C00018E400287FF4B8AC01226F2128460FF0F2
:1023D0004DFE6E2128460FF027FE30600AE40028EB
:1023E0007FF4AAAC02226F2128460FF03FFE6E2137
:1023F00028460FF019FE3060FFF7FCBB00287FF481
:102400009BAC03226F2128460FF030FE6E21284638
:102410000FF00AFE3060FFF7EDBB00287FF48CACB4
:1024200004226F2128460FF021FE6E2128460FF06E
:10243000FBFD3060FFF7DEBB00287FF47DAC05229A
:102440006F2128460FF012FE6E2128460FF0ECFD9A
:102450003060FFF7CFBB00287FF46EAC06226F21FF
:1024600028460FF003FE6E2128460FF0DDFD306098
:10247000FFF7C0BB00287FF45FAC07226F2128461E
:102480000FF0F4FD6E2128460FF0CEFD3060FFF70F
:10249000B1BB00287FF450AC08226F2128460FF012
:1024A000E5FD22466E2128460FF000FE00B23060A6
:1024B000FFF7A0BB00287FF43FAC08226F2128461D
:1024C0000FF0D4FD01226E2128460FF0EFFD00B27F
:1024D0003060FFF78FBB00287FF42EAC09226F21FC
:1024E00028460FF0C3FD22466E2128460FF0DEFD80
:1024F00000B23060FFF77EBB00287FF41DAC0A22DB
:102500006F2128460FF0B2FD22466E2128460FF0BB
:10251000CDFD00B23060FFF76DBB00287FF40CAC3E
:102520000A226F2128460FF0A1FD01226E212846C4
:102530000FF0BCFD00B23060FFF75CBB0457002019
:102540004C5700202057002000287FF4F5AB0B22C9
:102550006F2128460FF08AFD22466E2128460FF093
:10256000A5FD00B23060FFF745BB00287FF4E4AB67
:102570000B226F2128460FF079FD01226E2128469B
:102580000FF094FD00B23060FFF734BB00287FF4F9
:10259000D3AB0C226F2128460FF068FD22466E2136
:1025A00028460FF083FD00B23060FFF723BB002800
:1025B0007FF4C2AB0C226F2128460FF057FD012299
:1025C0006E2128460FF072FD00B23060FFF712BB9B
:1025D00000287FF4B1AB0D226F2128460FF046FD95
:1025E00022466E2128460FF061FD00B23060FFF7F1
:1025F00001BB00287FF4A0AB0D226F2128460FF00D
:1026000035FD01226E2128460FF050FD00B23060EA
:10261000FFF7F0BA00287FF48FAB0E226F21284617
:102620000FF024FD22466E2128460FF03FFD00B238
:102630003060FFF7DFBA00287FF47EAB0E226F21F7
:1026400028460FF013FD01226E2128460FF02EFDC3
:1026500000B23060FFF7CEBA00287FF46DAB0F22D6
:102660006F2128460FF002FD22466E2128460FF00A
:102670001DFD00B23060FFF7BDBA00287FF45CABEF
:102680000F226F2128460FF0F1FC01226E2128460F
:102690000FF00CFD00B23060FFF7ACBA00287FF4F9
:1026A0004BAB10226F2128460FF0E0FC22466E2132
:1026B00028460FF0FBFC00B23060FFF79BBA002801
:1026C0007FF43AAB11226F2128460FF0CFFC22464F
:1026D0006E2128460FF0EAFC00B23060FFF78ABA9C
:1026E00000287FF429AB11226F2128460FF0BEFC91
:1026F00001226E2128460FF0D9FC00B23060FFF7AE
:1027000079BA00287FF418AB12226F2128460FF007
:10271000ADFC22466E2128460FF0C8FC00B23060A6
:10272000FFF768BA00287FF407AB13226F21284611
:102730000FF09CFC22466E2128460FF0B7FC30605B
:10274000FFF758BA00287FF4F7AA13226F21284612
:102750000FF08CFC01226E2128460FF0A7FC3060A0
:10276000FFF748BA58B9D0226F2128460FF07EFCF7
:102770006E2128460FF058FC3060FFF73BBA012865
:102780007FF43CAAD0226F2128460FF06FFC3268FC
:102790006E2128460FF06AFC0024FFF72BBA58B9C7
:1027A000D1226F2128460FF061FC6E2128460FF0E0
:1027B0003BFC3060FFF71EBA01287FF41FAAD1222C
:1027C0006F2128460FF052FC32686E2128460FF028
:1027D0004DFC0024FFF70EBA68B9D2226F212846BB
:1027E0000FF044FC22466E2128460FF05FFC00B239
:1027F0003060FFF7FFB901287FF400AAD2226F21D1
:1028000028460FF033FC338800226E2128460FF053
:102810005AFC0024FFF7EEB968B9D2226F2128468E
:102820000FF024FC01226E2128460FF03FFC00B27D
:102830003060FFF7DFB901287FF4E0A9D2226F21D1
:1028400028460FF013FC224633886E2128460FF0ED
:102850003AFC0024FFF7CEB968B9D3226F2128468D
:102860000FF004FC22466E2128460FF01FFC00B238
:102870003060FFF7BFB901287FF4C0A9D3226F21D0
:1028800028460FF0F3FB338800226E2128460FF014
:102890001AFC0024FFF7AEB968B9D3226F2128468D
:1028A0000FF0E4FB01226E2128460FF0FFFB00B27F
:1028B0003060FFF79FB901287FF4A0A9D3226F21D0
:1028C00028460FF0D3FB224633886E2128460FF0AE
:1028D000FAFB0024FFF78EB900287FF42DAA1D22F1
:1028E0006F2128460FF0C2FB6E2128460FF09CFB9B
:1028F0003060FFF77FB900287FF41EAAC0226F2145
:1029000028460FF0B3FB22466E2128460FF0CEFB7F
:1029100000B23060FFF76EB900287FF40DAAC02224
:102920006F2128460FF0A2FB01226E2128460FF0EE
:10293000BDFB00B23060FFF75DB900287FF4FCA951
:10294000C1226F2128460FF091FB22466E212846B6
:102950000FF0ACFB00B23060FFF74CB900287FF4F9
:10296000EBA9C1226F2128460FF080FB01226E21C6
:1029700028460FF09BFB00B23060FFF73BB9002800
:102980007FF4DAA9C2226F2128460FF06FFB22469E
:102990006E2128460FF08AFB00B23060FFF72AB99B
:1029A00000287FF4C9A9C2226F2128460FF05EFBE0
:1029B00001226E2128460FF079FB00B23060FFF74C
:1029C00019B900287FF4B8A9C3226F2128460FF057
:1029D0004DFB22466E2128460FF068FB00B23060A6
:1029E000FFF708B900287FF4A7A9C3226F21284662
:1029F0000FF03CFB01226E2128460FF057FB00B27E
:102A00003060FFF7F7B800287FF496A9C4226F2141
:102A100028460FF02BFB22466E2128460FF046FB7E
:102A20003060FFF7E7B800287FF486A9C4226F2141
:102A300028460FF01BFB01226E2128460FF036FBC3
:102A40003060FFF7D7B800287FF476A9C5226F2140
:102A500028460FF00BFB22466E2128460FF026FB7E
:102A60003060FFF7C7B800287FF466A9C5226F2140
:102A700028460FF0FBFA01226E2128460FF016FBC4
:102A80003060FFF7B7B800287FF456A9C6226F213F
:102A900028460FF0EBFA22466E2128460FF006FB7F
:102AA0003060FFF7A7B800287FF446A9C6226F213F
:102AB00028460FF0DBFA01226E2128460FF0F6FAC5
:102AC0003060FFF797B800287FF436A9C7226F213E
:102AD00028460FF0CBFA22466E2128460FF0E6FA80
:102AE0003060FFF787B800287FF426A9C7226F213E
:102AF00028460FF0BBFA01226E2128460FF0D6FAC5
:102B00003060FFF777B800287FF416A9C8226F213C
:102B100028460FF0ABFA6E2128460FF085FA306098
:102B2000FFF768B800287FF407A9C9226F2128465B
:102B30000FF09CFA6E2128460FF076FA3060FFF70E
:102B400059B800287FF4F8A8CA226F2128460FF050
:102B50008DFA6E2128460FF067FA3060FFF74AB809
:102B600000287FF4E9A8CB226F2128460FF07EFAD7
:102B70006E2128460FF058FA3060FFF73BB838B99D
:102B80000C21224B01FB05352B893360FFF732B84E
:102B900001287FF433A80C211C4B002401FB0535D0
:102BA00033682B81FFF726B838B90C21174B01FB8E
:102BB0000535EB793360FFF71DB801287FF41EA8B7
:102BC0000C214D431149AA1D07350A443078294488
:102BD0000FF074FC0024FFF70DB800287FF4ACA8B8
:102BE0000C210A4B01FB0535AB793360FFF702B8C6
:102BF00000287FF4A1A80C23044903FB0515AB882A
:102C00003360FEF7F7BF0424FEF7F4BF045700203B
:102C100010B413460446084619B9224610BCFEF704
:102C2000DABE082010BC70470120704707B501923A
:102C300039B9024601AB0120FEF7CDFE03B05DF8C5
:102C400004FB0820FAE710B40C4630B9044B2046C8
:102C50001B6811469B6810BC1847002010BC7047C9
:102C60004857002070B52E4D2E4EEC6860682368E2
:102C7000C8303060DB689847236830685B699847E4
:102C80002A69294B00251A606368012403F537730C
:102C90005360264B26495A6926480A602649147013
:102CA000C2F8041225495570C2F80812244A1C744F
:102CB0001A62244ADA61244A9A61244A5A62244AEE
:102CC000DA64244A9A63244A5A63244A9A62244A58
:102CD000DA62244A9A64244A5A64244A5A65244A85
:102CE0001A65244A1A66244ADA65244A9A65322209
:102CF000DA6040F28A229A604FF47A72204B5A804E
:102D000041F270721A804FF48072DD711A810DF0F9
:102D100033F91C4B20461D70BDE87040FEF7D0BD56
:102D2000649E02081457002048570020203E0020CF
:102D30004457002020570020292C0108E5170108DE
:102D400099190108D5190108D1190108CD190108EF
:102D5000AB180108112C01082D2C01086519010878
:102D600025190108F51701089D180108FB1701082E
:102D7000E1170108C1180108E91701080119010844
:102D8000045700204C5700200022014B5A60704726
:102D9000203E002070B50446074E084D33682A4691
:102DA000014600200FF0E9FB33682A462146BDE8C2
:102DB000704001200FF0E1BBEC590020505700207B
:102DC000014B18680FF039BCEC59002001280CD8D1
:102DD000074B1A68202303FA00F040F0020002EBD0
:102DE0008000436800200B6070470820704700BFD8
:102DF000EC590020012810B5144611D003D3022845
:102E00001AD0042010BD14680F4A104BD268126803
:102E100024B15269D8689047002010BD9269F9E743
:102E2000094B0A4ADB6850681B681B6A98470030E8
:102E300018BF01202060EFE7034B044ADB6890686D
:102E40001B681B6AF2E700BF649E0208241600207C
:102E5000022804BF0B4B93F8D80030B90A4BDB684B
:102E60001B685B69094A10681847012809D1054B9E
:102E700093F8D830012B04D1034BDB681B689B69A6
:102E8000F0E77047203E0020649E020824160020D0
:102E900070B50020FFF7DCFF104B114CDD68206897
:102EA0002B689B6898472B6860689B6898472B68DD
:102EB000A0689B6898472B68A0699B6898472B6817
:102EC00020699B6898472B6860699B6898472B68C6
:102ED000E0689B68BDE87040184700BF649E020828
:102EE000241600202DE9F8430F4691469846174CCA
:102EF0000021236847F080009B689DF820609DF8C2
:102F000024509847236800219B68484698472368C7
:102F100000219B6840469847236800219B68304603
:102F20009847236828469B6801219847084B48EA40
:102F300009281B6846EA082607F07F0703EB870786
:102F400045EA06257D60BDE8F88300BFE85900200A
:102F5000EC59002007B5D3B20193C2F307230093C5
:102F6000C2F30743120EFFF7BDFF03B05DF804FB89
:102F70000020FFF7EFBF012873B505460C4624D8A3
:102F8000134E335C63B12021124B814003EB80036D
:102F900041F00701DA69C9B2FFF7DCFF002373557E
:102FA000202622460024AE4046F00D01C9B2284634
:102FB000FFF7D0FF28460194009423462246F1B241
:102FC000FFF790FF204602B070BD0820FBE700BF6E
:102FD0006C00002024160020012873B505460E461B
:102FE0001CD82024844044F0070186EAE672A2EB54
:102FF000E672C9B2FFF7AEFF0123094A002E53550E
:10300000E1B2B8BF0223002401932846009423466E
:103010002246FFF767FF204602B070BD0820FBE79D
:103020006C0000200021D7E74942D5E7D4E738B546
:10303000234B01F07F04234493F81432DB0705D4BB
:10304000204B1B6803EB8404606838BD1E4D0021D3
:103050002B6820469B68984700212B6808469B6890
:10306000984700212B6808469B68984700212B68E9
:1030700008469B6898472B6801219B680020984769
:103080002B6800219B682046984700212B68084642
:103090009B68984700212B6804029B680846984764
:1030A00000212B6804439B68084698472B6824023C
:1030B00004439B680121002098472402204338BD27
:1030C00050570020EC590020E859002010B500208E
:1030D0001446FFF7ACFF206010BD38B50D46202127
:1030E000814041F00101C9B20446FFF7A0FF296801
:1030F000014429602046BDE838403CE71C2A2DE900
:10310000F84304460D461E4600F0BA8300F2A6803E
:103110000C2A00F07B824AD8052A00F0008219D8D8
:10312000022A00F0AB8107D8002A00F07081012A42
:1031300000F08981042474E1032A00F0BC81042A90
:10314000F8D1002840F0CC81CB4800EB8100C36966
:10315000336066E1082A00F0398213D8062A00F0AD
:10316000F781072AE6D1002840F018822021A940E3
:1031700041F01001C9B22846FFF759FF00F01F00C7
:1031800030604EE10A2A00F02F820B2AD2D10028AB
:1031900040F0A2812021A94041F01501C9B2284682
:1031A000FFF745FFC04300F00100306039E1122A0B
:1031B00000F0C88227D80F2A00F0848211D80D2A87
:1031C00000F04B820E2AB5D1002840F06D822021FC
:1031D000A94041F01401C9B22846FFF728FF30602A
:1031E0001FE1102A00F08782112AA3D1002840F0A5
:1031F0009B822021A94041F00801C9B22846FFF76F
:1032000016FF30600DE1152A00F0E08211D8132A74
:1032100000F0B182142A8DD1002840F0C98220210B
:10322000A94041F00B01C9B22846FFF700FF30600A
:10323000F7E0172A00F0FD82C0F0E182182A7FF43F
:1032400079AF002840F00E832021A94041F01301FE
:10325000C9B22846FFF7EBFE3060E2E0AC2A00F08E
:10326000268562D8A52A00F0F78331D8A22A00F07B
:10327000918318D81D2A00F028838C2A7FF45AAF36
:10328000002840F03083090141F06C0101F0FC019D
:103290002846FFF7CCFE4FF48073C0F3036043FA77
:1032A00000F03060BDE0A32A00F09983A42A7FF4E7
:1032B00041AF002840F0B883090141F06C0101F0F2
:1032C000FC012846FFF7B3FEC0F300303060A8E0F1
:1032D000A82A00F0608414D8A62A00F00584A72A42
:1032E0007FF428AF002840F03F84090141F06C01D1
:1032F00001F0FC012846FFF79AFE00F00F00306055
:103300008FE0AA2A00F0938440F26984002840F0FC
:10331000B584090141F06D0101F0FD012846FFF778
:1033200086FEC0F3411030607BE0B62A00F0678271
:103330003ED8B32A00F021851BD8AD2A00F0DD84E9
:10334000AE2A7FF4F7AE002840F0FE84090141F078
:103350006D0101F0FD012846FFF769FE001400F041
:103360007F0310F0400018BF6FF07F0018433060FB
:1033700057E0B42A00F02885B52A7FF4DBAE202779
:103380008F407FB247F014085FFA88F8414628461C
:10339000FFF74DFE002C40F02985410540F12385C3
:1033A00047F01101C9B22846FFF741FE306038E00E
:1033B000CE2A00F0798514D8B82A00F03585B92ACC
:1033C0007FF4B8AE002840F05685090141F06C0149
:1033D00001F0FC012846FFF72AFEC0F303503060DD
:1033E0001FE0D22A00F07E85D32A00F09685D12AEC
:1033F0007FF4A0AE002840F066852021A94041F06E
:103400001901C9B22846FFF712FE306009E058B929
:103410002021A94041F00D01C9B22846FFF707FE5F
:1034200030602046BDE8F883012801D00024F8E789
:103430002021A94041F00D011A68C9B22846FFF7C2
:1034400089FD0024EDE748B92021A94041F00101A0
:10345000C9B22846FFF7EBFD3060E2E70128E5D16D
:103460002021A94041F001011A68C9B22846FFF79E
:1034700071FD0024D5E700BF2416002048B92021A3
:10348000A94041F00701C9B22846FFF7D0FD3060DE
:10349000C7E70128CAD120213268BC4BA940002AC5
:1034A00041F007015855B8BF5242C9B22846FFF74C
:1034B00051FD0024B5E778B92021A94041F002016F
:1034C000C9B22846FFF7B3FD10F4000318BF4FF050
:1034D0007F4318433060A4E7012CA7D10424A0E760
:1034E0000128A3D120273268A94B002A07FA01F747
:1034F00003EB8103B8BF5242F9B22846DA61FFF705
:1035000096FD0446002891D1326847F00701002A51
:10351000B8BF5242C9B22846FFF71CFD81E748B93F
:103520002021A94041F00601C9B22846FFF77FFDDE
:10353000306076E701287FF479AF2021A94041F07F
:1035400006011A68C9B22846FFF704FD002468E79F
:1035500058B92021A94041F01001C9B22846FFF70F
:1035600066FDC0F3042030605BE701287FF45EAFA6
:1035700020248C4044F01004E4B221462846FFF792
:1035800056FD336820F4F8521B0203F4F853214629
:103590001A432846FFF7DEFC002442E701287FF4A7
:1035A00045AF20248C4044F01004E4B22146284664
:1035B000FFF73DFD336820F01F0203F01F03214693
:1035C0001A432846FFF7C6FC00242AE7002883D1C7
:1035D0002021A94041F01501C9B22846FFF727FD77
:1035E000C0F3402030601CE700287FF475AF202135
:1035F000A94041F01501C9B22846FFF718FD10F0A7
:10360000020F0CBF0123002333600AE758B92021C1
:10361000A94041F01401C9B22846FFF708FDC0F3E4
:1036200040003060FDE601287FF400AF20248C408C
:1036300044F01404E4B221462846FFF7F8FC33684E
:1036400020F00202002B14BF0023022321461A435C
:103650002846FFF77FFC0024E3E658B92021A94063
:1036600041F01401C9B22846FFF7E1FC00F0010067
:103670003060D6E601287FF4D9AE20248C4044F097
:103680001404E4B221462846FFF7D1FC326820F04A
:103690000100002A14BF024640F0010221462846DC
:1036A000FFF758FC0024BCE601287FF4BFAE2021C0
:1036B000A94041F014011A68C9B22846FFF74AFC34
:1036C0000024AEE648B92021A94041F00401C9B266
:1036D0002846FFF7ACFC3060A3E601287FF4A6AED5
:1036E0002021A94041F004011A68C9B22846FFF719
:1036F00031FC002495E648B92021A94041F005019C
:10370000C9B22846FFF793FC30608AE601287FF4AF
:103710008DAE2021A94041F005011A68C9B22846A2
:10372000FFF718FC00247CE601287FF47FAE2021FF
:10373000A94041F008011A68C9B22846FFF70AFCFF
:1037400000246EE648B92021A94041F00A01C9B21F
:103750002846FFF76CFC306063E601287FF466AE14
:103760002021A94041F00A011A68C9B22846FFF792
:10377000F1FB002455E668B92021A94041F003017E
:10378000C9B22846FFF753FC30604AE66C000020BF
:103790002416002001287FF449AE2021A94041F0E1
:1037A00003011A68C9B22846FFF7D4FB002438E6A3
:1037B00001287FF43BAE2021A94041F00B011A689B
:1037C000C9B22846FFF7C6FB00242AE648B92021E3
:1037D000A94041F00C01C9B22846FFF728FC30602F
:1037E0001FE601287FF422AE2021A94041F00C0100
:1037F0001A68C9B22846FFF7ADFB002411E654B998
:103800002021A94041F01101C9B22846FFF70FFC61
:103810000024306005E6012C7FF408AE2021A94089
:1038200041F011013268C9B22846FFF793FB00242A
:10383000F7E548B92021A94041F01201C9B2284654
:10384000FFF7F5FB3060ECE501287FF4EFAD2021B8
:10385000A94041F012011A68C9B22846FFF77AFB65
:103860000024DEE501287FF4E1AD2021A94041F0EC
:1038700013011A68C9B22846FFF76CFB0024D0E593
:1038800058B9090141F06C0101F0FC012846FFF72D
:10389000CEFBC0F380403060C3E501287FF4C6ADA5
:1038A0000C0144F06C04E4B221462846FFF7BFFB4C
:1038B000336820F480229B0403F4802321461A43BA
:1038C0002846FFF747FB0024ABE500287FF404AE51
:1038D0002020C94B88401B6840F0020003EB8000A9
:1038E000436833609DE501287FF4A0AD1B68102B71
:1038F00023D00DDC022B1CD004DC012B16D04FF0A2
:10390000FF3314E0042B16D0082BF8D105230EE06A
:10391000402B14D003DC202BF1D1032307E0802BB4
:103920000FD0B3F5807FEAD1002300E00823336095
:1039300008E00723FBE70623F9E70423F7E7022360
:10394000F5E73060336801333FF470AD2C0144F08B
:103950006C04E4B221462846FFF769FB336820F087
:1039600070621B0603F070631A4321462846FFF776
:10397000F1FA21462846FFF75AFB336820F07062BF
:103980001B0603F0706321461A432846FFF7E2FA4C
:10399000002446E558B9090141F06C0101F0FC0131
:1039A0002846FFF744FBC0F3C130306039E50128F9
:1039B0007FF43CAD0C0144F06C04E4B2214628468F
:1039C000FFF735FB336820F4C032DB0303F4C03368
:1039D00021461A432846FFF7BDFA002421E558B9CD
:1039E000090141F06C0101F0FC012846FFF71FFBC3
:1039F000C0F38030306014E501287FF417AD0C016E
:103A000044F06C04E4B221462846FFF710FB33680B
:103A100020F480429B0303F4804321461A43284646
:103A2000FFF798FA0024FCE401287FF4FFAC0C01B6
:103A300044F06C04E4B221462846FFF7F8FA3368F4
:103A400020F480521B0303F4805321461A43284676
:103A5000FFF780FA0024E4E40F0147F06C07FFB29F
:103A600039462846FFF7E3FA8046C4B918F480497E
:103A70003946284605D0FFF7DAFAC0F3C3103060A4
:103A8000CFE4FFF7D4FA18F4006FC0F3021001D1AD
:103A90003060CBE440F0080030604C46C1E4012CBB
:103AA0007FF4C4AC18F48044394628460ED0FFF7A2
:103AB000BEFA336820F4F062DB0103F4F0631A43CA
:103AC00039462846FFF746FA0024AAE4FFF7AFFA82
:103AD000336820F070021B0103F070031A4339466B
:103AE0002846FFF737FA9CE40F0147F06C07FFB256
:103AF00039462846FFF79BFA8CB910F480443946C2
:103B0000284606D0FFF793FAC0F302103060002475
:103B100087E4FFF78CFAC0F3C310306081E4012C16
:103B20007FF484AC10F48044394628460ED0FFF769
:103B30007EFA336820F070021B0103F070031A4311
:103B400039462846FFF706FA00246AE4FFF76FFAC1
:103B5000336820F4F062DB0103F4F0631A43394662
:103B60002846FFF7F7F95CE401287FF45FAC0C010D
:103B700044F06C04E4B221462846FFF758FA336853
:103B800020F00F0203F00F0321461A432846FFF7E7
:103B9000E1F9002445E458B9090141F06D0101F053
:103BA000FD012846FFF743FAC0F3C030306038E427
:103BB00001287FF43BAC0C0144F06D04E4B22146D3
:103BC0002846FFF734FA336820F40042DB039BB247
:103BD00021461A432846FFF7BDF9002421E468B9BD
:103BE000090141F06D0101F0FD012846FFF71FFAC0
:103BF000C0F34130306014E4EC59002001287FF418
:103C000015AC0C0144F06D04E4B221462846FFF7E0
:103C10000EFA336820F4C0425B0303F4C04321462C
:103C20001A432846FFF796F90024FFF7FABB60B95C
:103C3000090141F06D0101F0FD012846FFF7F7F998
:103C4000C0F303203060FFF7ECBB01287FF4EEAB3C
:103C50000C0144F06D04E4B221462846FFF7E7F971
:103C6000336820F470621B0203F4706321461A4328
:103C70002846FFF76FF90024FFF7D3BB01287FF434
:103C8000D5AB0C0144F06D04E4B221462846FFF7A1
:103C9000CEF9336820F060025B0103F06003214637
:103CA0001A432846FFF756F90024FFF7BABB60B95C
:103CB000090141F06D0101F0FD012846FFF7B7F958
:103CC00000F00F003060FFF7ACBB01287FF4AEAB13
:103CD0000C0144F06D04E4B221462846FFF7A7F931
:103CE000336820F00F0203F00F0321461A432846E1
:103CF000FFF730F90024FFF794BB60B9090141F0E8
:103D00006D0101F0FD012846FFF791F9C0F3006055
:103D10003060FFF786BB01287FF488AB0C0144F0CC
:103D20006D04E4B221462846FFF781F9336820F09C
:103D300080721B0603F0807321461A432846FFF762
:103D400009F90024FFF76DBB01287FF46FAB0C016C
:103D500044F06D04E4B221462846FFF768F9336861
:103D600020F4FE021B0403F4FE0321461A432846F6
:103D7000FFF7F0F80024FFF754BB60B9090141F0E8
:103D80006C0101F0FC012846FFF751F9C0F34040F7
:103D90003060FFF746BB01287FF448AB0C0144F0CC
:103DA0006C04E4B221462846FFF741F9336820F459
:103DB00000325B0403F4003321461A432846FFF720
:103DC000C9F80024FFF72DBB00287FF485AB09015B
:103DD00041F06F01C9B22846FFF729F9C0F304404A
:103DE0003060FFF71EBB3460FFF71BBB012C7FF474
:103DF0001DAB47F011013268C9B22846FFF7AAF897
:103E000041462846FFF713F9336820F48062002BFF
:103E10000CBF00234FF4806341461A432846FFF746
:103E200099F80024FFF7FDBA60B9090141F06C016F
:103E300001F0FC012846FFF7FAF8C0F3403030608B
:103E4000FFF7EFBA01287FF4F1AA0C0144F06C04EB
:103E5000E4B221462846FFF7EAF8336820F400521E
:103E60005B0303F4005321461A432846FFF772F818
:103E70000024FFF7D6BA01287FF4D8AA0C0144F039
:103E80006C04E4B221462846FFF7D1F8336820F4E9
:103E900070021B0503F4700321461A432846FFF7FE
:103EA00059F80024FFF7BDBA00287FF415AB0901CB
:103EB00041F06F01C9B22846FFF7B9F8C0F3090015
:103EC0003060FFF7AEBA01287FF4B0AA2021A940E4
:103ED00041F019011A68C9B22846FFF73BF80024DF
:103EE000FFF79FBA50B92021A94041F01A01C9B289
:103EF0002846FFF79CF83060FFF793BA01287FF45B
:103F000095AA2021A94041F01A011A68C9B2284691
:103F1000FFF720F80024FFF784BAE8B979B1012946
:103F20007FF47FAA01462846FFF781F800F0600081
:103F3000A0F12003584258413060FFF772BA08469A
:103F4000FFF775F800F01800A0F110025042504140
:103F500030602C46FFF765BA01287FF467AA21B1CB
:103F6000012917D00024FFF75CBA0846FFF75FF875
:103F7000336853B120F0080242F0100200210846D5
:103F8000FEF7E8FF0024FFF74CBA20F0100242F0E1
:103F90000802F3E700212846FFF749F8336853B1D8
:103FA00020F0400242F0200200210120FEF7D2FF63
:103FB0000024FFF736BA20F0200242F04002F3E777
:103FC00007B50129019207D8024601AB0120FFF78E
:103FD00095F803B05DF804FB0820FAE701291346C1
:103FE00003D802460020FFF789B80820704708B5BB
:103FF00022210020FFF71BF850B942210120FFF7D2
:1040000016F828B9034B1868BDE808400EF00EBB3F
:10401000002008BDEC59002070B53D4E3D480EF023
:104020006FFAF5683C4C6B6803F5AA72626003F5A1
:10403000B872A26003F56F72E26003F5767203F165
:10404000C800226103F57D7203F58263A3612B68CA
:104050006261DB68206098472B68E068DB689847FE
:104060002B68E0689B6998472B6860681B699847D4
:104070002B68A0681B6998472B68A0691B69984743
:104080002B6820691B6998472B6860691B699847F2
:104090003269224B22491A606B68012003F537739D
:1040A0005360204B5A690A601F491070C2F804120D
:1040B0001E49C2F80812002151701D4A1A621D4A99
:1040C000DA611D4A9A611D4A5A621D4A9A631D4A65
:1040D0005A631D4A9A621D4ADA621D4A9A641D4A51
:1040E0005A641D4A5A651D4A1A651D4ADA641D4AFA
:1040F0001A661D4ADA6502221A743222DA60B62282
:104100009A601A4A9A65BDE87040FEF7A1BE00BFEA
:10411000649E02085057002024160020E859002011
:10412000EC590020203E0020EF3F0108C12D01087E
:10413000D92F01082D300108293001082530010848
:10414000DD3F0108C13F0108772F0108DB3001087E
:10415000712F0108CD300108952D0108F52D0108BA
:10416000CD2D0108512E0108892D0108912E01083D
:1041700001289FBF034B53F8203000200B6088BFFD
:1041800008207047F85900200022014B5A60704700
:10419000203E002070B50446074E084D33682A467D
:1041A000014600200EF08FFA33682A462146BDE80A
:1041B000704001200EF087BAF0590020F859002015
:1041C000014B18680EF0C9BAF0590020012810B54B
:1041D000144603D002280ED0042010BD094B0A4A11
:1041E000DB6850681B681B6A9847003018BF0120C5
:1041F0002060002010BD034B034ADB6890681B68F9
:104200001B6AF1E7649E020854160020022804BFCE
:104210000B4B93F8D80030B90A4BDB681B685B691D
:10422000094A10681847012809D1054B93F8D8307E
:10423000012B04D1034BDB681B689B69F0E77047D7
:10424000203E0020649E02085416002070B5002015
:10425000FFF7DCFF084B094CDD6820682B689B6882
:1042600098472B6860689B6898472B68A0689B6894
:10427000BDE87040184700BF649E02085416002035
:104280002DE9F8430F4691469846174C00212368C4
:1042900047F080009B689DF820609DF82450984767
:1042A000236800219B6848469847236800219B6843
:1042B00040469847236800219B683046984723680A
:1042C00028469B6801219847084B48EA09281B6843
:1042D00046EA082607F07F0703EB870745EA06252D
:1042E0007D60BDE8F88300BFF4590020F05900203C
:1042F00007B5D3B20193C2F307230093C2F3074378
:10430000120EFFF7BDFF03B05DF804FB0020FFF7BE
:10431000EFBF0128F7B505460F4628D8154C0444D1
:1043200094F8943273B12021134B81401B6841F003
:10433000070103EB81035A68C9B2FFF7D9FF0023D5
:1043400084F8943220260024AE4046F00D013A460F
:10435000C9B22846FFF7CCFF2846019400942346B3
:104360002246F1B2FFF78CFF204603B0F0BD0820D3
:10437000FBE700BFF8590020F0590020012873B571
:1043800005460C4620D82026864084EAE47246F092
:104390000701A2EBE472C9B2FFF7AAFF01220B4B9F
:1043A000002C2B4483F894224FF00004ACBF13463A
:1043B000022328460193009423462246F1B2FFF7D8
:1043C0005FFF204602B070BD0820FBE7F8590020CF
:1043D0000021D3E74942D1E7D0E738B5234B01F0BC
:1043E0007F04234493F81432DB0705D4204B1B6869
:1043F00003EB8404606838BD1E4D00212B68204605
:104400009B68984700212B6808469B6898470021C5
:104410002B6808469B68984700212B6808469B68D4
:1044200098472B6801219B68002098472B68002142
:104430009B682046984700212B6808469B68984750
:1044400000212B6804029B680846984700212B68CE
:1044500004439B68084698472B68240204439B68E2
:104460000121002098472402204338BDF85900203C
:10447000F0590020F459002010B500201446FFF731
:10448000ACFF206010BD38B50D462021814041F0C1
:104490000101C9B20446FFF7A0FF29680144296061
:1044A0002046BDE8384034E71C2A2DE9F041044697
:1044B0000D461E4600F0108300F294800C2A00F096
:1044C00026824DD8052A00F0C6811ED8022A00F0A7
:1044D000728107D8002A00F04A81012A00F05E812B
:1044E00004244EE1032A00F07F81042AF8D1002839
:1044F00040F092812020C64B88401B6840F00700A6
:1045000003EB8000436833603BE1082A00F0E2815E
:1045100012D8062A00F0AC81072AE1D1002840F029
:10452000C7812021A94041F01001C9B22846FFF7F8
:1045300054FF00F01F0023E10A2A00F0D8810B2A63
:10454000CED1002840F060812021A94041F0150122
:10455000C9B22846FFF741FFC04300F001000FE158
:10456000122A00F05E821DD80F2A00F036820CD885
:104570000D2A00F0FC810E2AB2D1002840F02582DD
:104580002021A94041F01401F6E0102A00F0338206
:10459000112AA5D1002840F03C822021A94041F0F9
:1045A0000801E9E0152A00F060820CD8132A00F017
:1045B0004682142A94D1002840F04F822021A9403D
:1045C00041F00B01D8E0172A00F07082C0F05B8246
:1045D000182A85D1002840F077822021A94041F097
:1045E0001301C9E0AB2A00F00C845ED8A52A00F0C4
:1045F0002D832FD8A22A00F0DB8217D81D2A00F0C5
:1046000089828C2A7FF46CAF002840F08F820901E8
:1046100041F06C0101F0FC012846FFF7DEFE4FF48B
:104620008073C0F3036043FA00F0A9E0A32A00F00E
:10463000DD82A42A7FF454AF002840F0F5820901FE
:1046400041F06C0101F0FC012846FFF7C6FEC0F303
:10465000003095E0A82A00F0878312D8A62A00F03F
:104660003E83A72A7FF43CAF002840F06E83090107
:1046700041F06C0101F0FC012846FFF7AEFE34600A
:104680007FE0A92A00F08D83AA2A7FF429AF0028B1
:1046900040F0A583090141F06D0101F0FD012846BC
:1046A000FFF79BFEC0F303206AE0B52A00F03884D0
:1046B0002AD8AE2A00F0F28313D8AC2A00F0BF83C8
:1046C000AD2A7FF40DAF002840F0D683090141F0F8
:1046D0006D0101F0FD012846FFF77FFEC0F3006089
:1046E0004EE0B32A00F0FE83B42A7FF4F9AE00282E
:1046F00040F08A80090141F06F01C9B22846FFF7F6
:104700006CFEC0F304403BE0CE2A00F03B8413D89B
:10471000B62A00F0B881B82A7FF4E2AE002840F053
:104720001F84090141F06C0101F0FC012846FFF7EC
:1047300054FEC0F3403023E0D12AFFF4D1AED22A98
:1047400024D9D32A7FF4CCAE002840F0338400294A
:1047500000F02684012914D101462846FFF73DFECA
:1047600000F06000A0F120035842584108E058B919
:104770002021A94041F00D01C9B22846FFF72DFEC6
:1047800030602046BDE8F081012801D00024F8E720
:104790002021A94041F00D01326820E020B92021FC
:1047A000A94041F00101E7E70128EFD12021A9400C
:1047B00041F00101F0E720B92021A94041F00701B3
:1047C000DAE70128E2D1134B0B44202183F894024D
:1047D0003268A940002A41F00701B8BF5242C9B26D
:1047E0002846FFF785FDD1E770B92021A94041F0A7
:1047F0000201C9B22846FFF7F0FD10F4000318BF0C
:104800004FF07F431843BBE7012C3FF469AEBDE78F
:10481000F0590020F85900200128B7D12021C14BC0
:104820003268A9401B6841F00707002A03EB8703A1
:10483000B8BF52425A60C9B22846FFF7CEFD0446BF
:104840000028A3D13268F9B2002AB8BF52422846E4
:10485000FFF74EFD95E720B92021A94041F0060160
:104860008AE7012892D12021A94041F0060193E76F
:1048700050B92021A94041F01001C9B22846FFF7E4
:10488000ACFDC0F304207BE701287FF47FAF202438
:104890008C4044F01004E4B221462846FFF79DFD09
:1048A000336820F4F8521B0203F4F8531A4359E218
:1048B00001287FF46BAF20248C4044F01004E4B254
:1048C00021462846FFF789FD336820F01F0203F0D8
:1048D0001F03EBE7002897D12021A94041F01501E3
:1048E000C9B22846FFF779FDC0F3402048E7002809
:1048F0008AD12021A94041F01501C9B22846FFF70D
:104900006CFD10F0020F0CBF01230023FBE550B932
:104910002021A94041F01401C9B22846FFF75DFDEE
:10492000C0F340002CE701287FF430AF20248C40F6
:1049300044F01404E4B221462846FFF74EFD3368E4
:1049400020F00202002B0CBF0023022321461A4351
:104950002846FFF7CDFC21462846FFF73EFD336889
:1049600020F00802022B14BF002308239EE740B961
:104970002021A94041F01401C9B22846FFF72DFDBE
:10498000EBE501287FF402AF20248C4044F01404AE
:10499000E4B221462846FFF720FD326820F00100EE
:1049A000002A0CBF024640F0010221462846FFF7CC
:1049B0009FFC21462846FFF710FD336820F00402D3
:1049C000022B14BF0023042370E701287FF4DEAE1E
:1049D0002021A94041F01401DEE620B92021A940A0
:1049E00041F00401C8E601287FF4D0AE2021A9409F
:1049F00041F00401D0E620B92021A94041F0050191
:104A0000BAE601287FF4C2AE2021A94041F0050199
:104A1000C2E601287FF4BAAE2021A94041F0080186
:104A2000BAE620B92021A94041F00A01A4E60128F4
:104A30007FF4ACAE2021A94041F00A01ACE620B9D8
:104A40002021A94041F0030196E601287FF49EAEA3
:104A50002021A94041F003019EE601287FF496AE93
:104A60002021A94041F00B0196E620B92021A94060
:104A700041F00C0180E601287FF488AE2021A94096
:104A800041F00C0188E64CB92021A94041F0110108
:104A9000C9B22846FFF7A1FC306077E6012C7FF40D
:104AA00075AE2021A94041F0110175E620B9202101
:104AB000A94041F012015FE601287FF467AE202192
:104AC000A94041F0120167E601287FF45FAE202182
:104AD000A94041F013015FE650B9090141F06C01B2
:104AE00001F0FC012846FFF778FCC0F3804047E660
:104AF00001287FF44BAE0C0144F06C04E4B2214673
:104B00002846FFF76AFC336820F480229B0403F4F4
:104B10008023CBE600287FF477AE034B53F8213097
:104B2000F1E400BFF0590020F859002001287FF47B
:104B30002DAE1B68102B23D00DDC022B1CD004DC07
:104B4000012B16D04FF0FF3314E0042B16D0082BA6
:104B5000F8D105230EE0402B14D003DC202BF1D13B
:104B6000032307E0802B0FD0B3F5807FEAD1002329
:104B700000E00823336008E00723FBE70623F9E79A
:104B80000423F7E70223F5E73060336801333FF48D
:104B9000FDAD2C0144F06C04E4B221462846FFF739
:104BA0001CFC336820F070621B0603F070637DE626
:104BB00050B9090141F06C0101F0FC012846FFF7F2
:104BC0000CFCC0F3C130DBE501287FF4DFAD0C0144
:104BD00044F06C04E4B221462846FFF7FEFB33683C
:104BE00020F4C032DB0303F4C0335FE650B909019F
:104BF00041F06C0101F0FC012846FFF7EEFBC0F329
:104C00008030BDE501287FF4C1AD0C0144F06C0497
:104C1000E4B221462846FFF7E0FB336820F48042E7
:104C20009B0303F4804341E601287FF4AFAD0C0100
:104C300044F06C04E4B221462846FFF7CEFB33680B
:104C400020F480521B0303F480532FE60F0147F03A
:104C50006C07FFB239462846FFF7BFFB94B910F442
:104C6000804206D039462846FFF7B7FBC0F3C31091
:104C700086E5031103F07003010548BF43F0080304
:104C8000336083E5012C7FF481AD10F48044394614
:104C900028460AD0FFF7A1FB336820F4F062DB015D
:104CA00003F4F0631A4339469AE5FFF796FB33683D
:104CB00020F4006213F0080F18BF4FF40064394667
:104CC00028462243FFF714FB39462846FFF785FBA9
:104CD000336820F070021B0103F07003E2E70F015C
:104CE00047F06C07FFB239462846FFF776FB80464F
:104CF000A4B918F480443946284604D0FFF76DFB68
:104D0000C0F30210C8E6FFF768FB18F4006FC0F3A9
:104D1000C3103FF4C1AE40F0080031E5012C7FF430
:104D200035AD39462846FFF758FB10F48044394624
:104D30002846CBD1FFF751FB336820F4F062DB014A
:104D400003F4F0631A43394681E501287FF41EAD70
:104D50000C0144F06C04E4B221462846FFF73DFB09
:104D600020F00F0221463BE550B9090141F06D01E9
:104D700001F0FD012846FFF730FBC0F3C030FFE42F
:104D800001287FF403AD0C0144F06D04E4B2214628
:104D90002846FFF722FB336820F40042DB039BB276
:104DA00084E550B9090141F06D0101F0FD0128468B
:104DB000FFF713FBC0F34130E2E401287FF4E6ACD7
:104DC0000C0144F06D04E4B221462846FFF705FBD0
:104DD000336820F4C0425B0303F4C04366E5012856
:104DE0007FF4D4AC0C0144F06D04E4B221462846B3
:104DF000FFF7F3FA336820F470621B0203F4706368
:104E000054E550B9090141F06D0101F0FD0128465A
:104E1000FFF7E3FAC0F34110B2E401287FF4B6AC27
:104E20000C0144F06D04E4B221462846FFF7D5FAA0
:104E3000336820F060025B0103F0600336E550B98F
:104E4000090141F06D0101F0FD012846FFF7C5FAA7
:104E500000F00F0094E401287FF498AC0C0144F0BA
:104E60006D04E4B221462846FFF7B7FA336820F014
:104E70000F0203F00F0319E501287FF487AC0C0142
:104E800044F06D04E4B221462846FFF7A6FA3368E1
:104E900020F080721B0603F0807307E580B90901DA
:104EA00041F06D0101F0FD012846FFF796FA00146C
:104EB00000F07F0310F0400018BF6FF07F00A1E406
:104EC00001287FF463AC0C0144F06D04E4B2214688
:104ED0002846FFF782FA336820F4FE021B0403F42D
:104EE000FE03E3E450B9090141F06C0101F0FC015B
:104EF0002846FFF772FAC0F3404041E401287FF4EE
:104F000045AC0C0144F06C04E4B221462846FFF79E
:104F100064FA336820F400325B0403F40033C5E420
:104F200000283FF4B1AD01287FF430AC20248C4040
:104F300064B244F0110144F014041A68C9B228465E
:104F4000E4B2FFF7D5F921462846FFF746FA336861
:104F500020F48062002B0CBF00234FF48063A5E493
:104F600001287FF413AC0C0144F06C04E4B2214638
:104F70002846FFF732FA336820F400525B0303F44B
:104F8000005393E400287FF43FAC090141F06F0126
:104F9000C9B22846FFF721FAC0F30900FFF7F0BBBA
:104FA0000846FFF71AFA00F01800A0F1100250426C
:104FB000504171E501287FF4E9AB79B101297FF413
:104FC000E5AB00212846FFF708FA336820F06002BD
:104FD000A3B142F020020021012002E40846FFF7BD
:104FE000FCF9336820F018022BB142F010020021C6
:104FF0000846FFF7F6BB42F00802F8E742F040022D
:10500000E9E707B50129019207D8024601AB012063
:10501000FFF74AFA03B05DF804FB0820FAE701291C
:10502000134603D802460020FFF73EBA0820704717
:1050300008B522210020FFF7D0F950B94221012004
:10504000FFF7CBF928B9044B1868BDE808400DF00C
:105050007BBB002008BD00BFF059002070B52D4E6D
:105060002D480DF0F3FAF4682C4D636803F5AA722D
:1050700003F1C80003F5B873AB6023686A60DB68AE
:1050800028609847236868681B6998472368A86860
:105090001B6998473269224B22491A6063680220D3
:1050A00003F537735360204B5A690A601F49C2F8F1
:1050B00004121F49C2F80812012111700021517019
:1050C0001C4A18741A621C4ADA611C4A9A611C4A0A
:1050D0005A621C4A9A631C4A5A631C4A9A621C4AC6
:1050E000DA621C4A9A641C4A5A641C4A5A651C4A71
:1050F0001A651C4ADA641C4A1A661C4ADA653222AE
:10510000DA604FF48C729A60194A9A65BDE8704073
:10511000FFF77CB8649E0208F8590020541600205E
:10512000F4590020F0590020203E002031500108A1
:10513000C14101087D430108D9430108D543010855
:10514000D14301081F50010803500108134301080F
:10515000874401080D43010879440108954101087D
:10516000CD410108714101080D4201088941010842
:105170004D42010801289FBF044B03EB8000C36927
:10518000002094BF0B600820704700BF945C002093
:105190000022014B5A607047203E0020024B02461D
:1051A000196802480DF0DABB905C0020945C002086
:1051B0000A46014601480DF003BB00BF945C002085
:1051C00010B500201446FFF7F3FF206010BD38B57E
:1051D00014460A46014603481D460DF0F1FA2040E8
:1051E000E84038BD945C002013460A460146014859
:1051F0000DF0E2BA945C00200020F5E72DE9F047BD
:105200000C4D994606460F4690460A4601462846EA
:10521000089C0DF0D5FA04FA09F2424002EA0802AD
:1052200082EA000331463A462846BDE8F0470DF0D1
:10523000C3BA00BF945C0020014B18680DF050BB4E
:10524000905C002008B522210020FFF7B1FF50B983
:1052500042210120FFF7ACFF28B9044B1868BDE8D4
:1052600008400DF034BB002008BD00BF905C00205A
:10527000012810B5144611D003D302281AD00420F7
:1052800010BD14680F4A104BD268126824B15269DD
:10529000D8689047002010BD9269F9E7094B0A4A87
:1052A000DB6850681B681B6A9847003018BF0120F4
:1052B0002060EFE7034B044ADB6890681B681B6AB9
:1052C000F2E700BF649E02086C160020022804BFAB
:1052D0000B4B93F8D80030B90A4BDB681B685B694D
:1052E000094A10681847012809D1054B93F8D830AE
:1052F000012B04D1034BDB681B689B69F0E7704707
:10530000203E0020649E02086C16002070B500202C
:10531000FFF7DCFF104B114CDD6820682B689B68A1
:1053200098472B6860689B6898472B68A0689B68C3
:1053300098472B68A0699B6898472B6820699B68F1
:1053400098472B6860699B6898472B68E0689B6862
:10535000BDE87040184700BF649E02086C1600202C
:10536000012870B504460E461DD8104D05EB80058A
:10537000EA6942B12021814041F00701C9B2FFF73B
:1053800033FF0023EB612025A54045F00D01324697
:105390002046C9B2FFF728FF20460022E9B2FFF7F6
:1053A00023FF002070BD082070BD00BF6C160020D8
:1053B00038B50D462021814041F00101C9B20446B3
:1053C000FFF7F6FE2968014429602046BDE8384011
:1053D000C6E7012870B504460E4622D8124D05EBEB
:1053E0008005EB693BB92021814041F00701C9B23A
:1053F000FFF7DEFEE8612025A54045F0070186EABB
:10540000E672A2EBE6722046C9B2FFF7EDFE002E6F
:105410002046ACBF01220222E9B2FFF7E5FE0020E0
:1054200070BD082070BD00BF6C1600200021D0E7C1
:105430004942CEE7CDE71C2A2DE9F34104460D464B
:105440001E4600F0A08300F2AD800C2A00F07482AA
:1054500051D8052A00F006821ED8022A00F0B38136
:1054600007D8002A00F07781012A00F091810424F6
:105470007BE1032A00F0C281042AF8D1002840F021
:10548000D2812020C84B88401B6840F0070003EB06
:1054900080004368336068E1082A00F02D8213D849
:1054A000062A00F0F881072AE1D1002840F0138293
:1054B0002021A94041F0100103461F22C9B228460D
:1054C000FFF785FE306050E10A2A00F024820B2AA3
:1054D000CDD1002840F0A3812021A94041F0150141
:1054E00003460122C9B22846FFF771FEB0FA80F0E8
:1054F0004009306039E1122A00F0A88227D80F2A2B
:1055000000F0648211D80D2A00F034820E2AAED148
:10551000002840F04D822021A94041F01401C9B279
:105520002846FFF745FE30601FE1102A00F0678231
:10553000112A9CD1002840F07B822021A94041F013
:105540000801C9B22846FFF733FE30600DE1152A85
:1055500000F0BC8211D8132A00F09182142A86D15F
:10556000002840F0A5822021A94041F00B01C9B2DA
:105570002846FFF71DFE3060F7E0172A00F0DC82B6
:10558000C0F0BD82182A7FF472AF002840F0ED828F
:105590002021A94041F01301C9B22846FFF708FEB7
:1055A0003060E2E0AC2A00F0D48464D8A52A00F090
:1055B000A68333D8A22A00F0508319D81D2A00F000
:1055C00002838C2A7FF453AF002840F00583090141
:1055D00041F06C0118234FF0706201F0FC01284685
:1055E000FFF7F5FD4FF4807343FA00F03060BCE044
:1055F000A32A00F05283A42A7FF439AF002840F098
:105600006C83090141F06C010C234FF4805201F0CE
:10561000FC012846FFF7DBFD3060A6E0A82A00F079
:10562000258414D8A62A00F0C483A72A7FF41FAFCC
:10563000002840F00A84090141F06C0103460F2262
:1056400001F0FC012846FFF7C2FD30608DE0AA2A78
:1056500000F04E8440F22A84002840F06984090159
:1056600041F06D010523602201F0FD012846FFF79E
:10567000AEFD306079E0B62A00F041823BD8B32A13
:1056800000F0BC841BD8AD2A00F08384AE2A7FF4DE
:10569000EEAE002840F09F84090141F06D01102317
:1056A0004FF4FE0201F0FD012846FFF790FD10F0D7
:1056B000400318BF6FF07F031843306055E0B42AF1
:1056C00000F0BE84B52A7FF4D2AE002840F0C88432
:1056D00020278F407FB247F01401C9B22846FFF758
:1056E00067FD410547D547F01101C9B22846FFF7CC
:1056F0005FFD306039E0CE2A00F0058515D8B82A64
:1057000000F0CC84B92A7FF4B2AE002840F0E884DF
:10571000090141F06C0114234FF4700201F0FC0107
:105720002846FFF754FD30601FE0D22A00F00A85BA
:10573000D32A00F02285D12A7FF499AE002840F0C8
:10574000F2842021A94041F01901C9B22846FFF78F
:105750002FFD306009E060B92021A94041F00D0122
:10576000C9B22846FFF724FD3060204602B0BDE8EC
:10577000F081012801D00024F7E72021A94041F061
:105780000D011A68C9B22846FFF72EFD0024ECE788
:1057900060B92021A94041F00101C9B22846FFF7B4
:1057A00007FD3060E1E700BF905C00200128E2D1F6
:1057B0002021A94041F001011A68C9B22846FFF72B
:1057C00013FD0024D1E748B92021A94041F0070189
:1057D000C9B22846FFF7ECFC3060C6E70128CAD101
:1057E00020211A68A940002A41F00701B8BF52429F
:1057F000C9B22846FFF7F8FC0024B6E778B92021A3
:10580000A94041F00201C9B22846FFF7D1FC10F4CB
:10581000000318BF4FF07F4318433060A5E7012C09
:10582000A9D10424A1E70128A5D12021BA4B3268CF
:10583000A9401B6841F00707002A03EB8703B8BFA4
:1058400052425A60C9B22846FFF7B2FC044600280B
:1058500091D13268F9B2002AB8BF52422846FFF708
:10586000C3FC82E748B92021A94041F00601C9B232
:105870002846FFF79DFC306077E701287FF47BAF77
:105880002021A94041F006011A68C9B22846FFF755
:10589000ABFC002469E760B92021A94041F0100168
:1058A00008234FF4F852C9B22846FFF790FC306045
:1058B0005BE701287FF45FAF20211B68A94041F01E
:1058C000100100934FF4F8520823C9B22846FFF79D
:1058D00095FC002449E701287FF44DAF20211B6887
:1058E000A94041F0100100931F220023C9B22846AD
:1058F000FFF784FC002438E7002890D12021A9403C
:1059000041F0150109234FF40072C9B22846FFF790
:105910005EFC306029E7002881D12021A94041F0B8
:10592000150101230222C9B22846FFF750FCB0FA44
:1059300080F04009306018E758B92021A94041F0B3
:10594000140101230222C9B22846FFF740FC30604F
:105950000BE701287FF40FAF20211B68A94041F01D
:105960001401009302220346C9B22846FFF746FC01
:105970000024FAE658B92021A94041F0140100237F
:105980000122C9B22846FFF722FC3060EDE601286B
:105990007FF4F1AE20211B68A94041F0140100936F
:1059A00002460023C9B22846FFF728FC0024DCE6A3
:1059B00001287FF4E0AE2021A94041F014011A68CB
:1059C000C9B22846FFF710FC0024CEE648B92021D2
:1059D000A94041F00401C9B22846FFF7E9FB306055
:1059E000C3E601287FF4C7AE2021A94041F004019D
:1059F0001A68C9B22846FFF7F7FB0024B5E648B994
:105A00002021A94041F00501C9B22846FFF7D0FB8B
:105A10003060AAE601287FF4AEAE2021A94041F013
:105A200005011A68C9B22846FFF7DEFB00249CE690
:105A300001287FF4A0AE2021A94041F008011A6896
:105A4000C9B22846FFF7D0FB00248EE648B92021D2
:105A5000A94041F00A01C9B22846FFF7A9FB30600E
:105A600083E601287FF487AE2021A94041F00A0196
:105A70001A68C9B22846FFF7B7FB002475E648B993
:105A80002021A94041F00301C9B22846FFF790FB4D
:105A900030606AE601287FF46EAE2021A94041F013
:105AA00003011A68C9B22846FFF79EFB00245CE692
:105AB00001287FF460AE2021A94041F00B011A6853
:105AC000C9B22846FFF790FB00244EE648B92021D2
:105AD000A94041F00C01C9B22846FFF769FB3060CC
:105AE00043E601287FF447AE2021A94041F00C0194
:105AF0001A68C9B22846FFF777FB002435E66CB96F
:105B00002021A94041F01101C9B22846FFF750FBFE
:105B10000024306029E600BF905C0020012C7FF457
:105B20002AAE2021A94041F011013268C9B22846AD
:105B3000FFF75AFB002418E648B92021A94041F09C
:105B40001201C9B22846FFF733FB30600DE6012889
:105B50007FF411AE2021A94041F012011A68C9B2A8
:105B60002846FFF741FB0024FFE501287FF403AE40
:105B70002021A94041F013011A68C9B22846FFF755
:105B800033FB0024F1E560B9090141F06C011223F7
:105B90004FF4802201F0FC012846FFF718FB30602B
:105BA000E3E501287FF4E7AD1B68090141F06C01D2
:105BB00000934FF48022122301F0FC012846FFF7E6
:105BC0001DFB0024D1E500287FF429AEBE4800EB80
:105BD0008100C3693360C8E501287FF4CCAD1B6840
:105BE000102B23D00DDC022B1CD004DC012B16D093
:105BF0004FF0FF3314E0042B16D0082BF8D1052307
:105C00000EE0402B14D003DC202BF1D1032307E05E
:105C1000802B0FD0B3F5807FEAD1002300E008236A
:105C2000336008E00723FBE70623F9E70423F7E7DF
:105C30000223F5E730603368581C3FF49CAD29011E
:105C400041F06C0100934FF07062182301F0FC01E9
:105C50002846FFF7D3FA002487E560B9090141F02F
:105C60006C010F234FF4C03201F0FC012846FFF70E
:105C7000AEFA306079E501287FF47DAD1B6809013B
:105C800041F06C0100934FF4C0320F2301F0FC018E
:105C90002846FFF7B3FA002467E560B9090141F02F
:105CA0006C010E234FF4804201F0FC012846FFF7FF
:105CB0008EFA306059E501287FF45DAD1B6809015B
:105CC00041F06C0100934FF480420E2301F0FC017F
:105CD0002846FFF793FA002447E501287FF44BADEF
:105CE0001B68090141F06C0100934FF480520C23B2
:105CF00001F0FC012846FFF781FA002435E560BB7E
:105D00000F0147F06C07FFB20E234FF48042394673
:105D10002846FFF75CFA804640B107234FF4F06253
:105D200039462846FFF753FA30601EE504237022F7
:105D300039462846FFF74BFA0B2330604FF40062D8
:105D400039462846FFF743FA00283FF414AD33687C
:105D5000444643F00803336007E501287FF40BADA8
:105D60000F0147F06C07FFB239462846FFF720FACB
:105D700010F48044336809D000934FF4F062072395
:105D800039462846FFF73AFA0024EEE4C3F3C0038D
:105D90000093394628460B234FF40062FFF72EFA92
:105DA000336870220093394604232846FFF726FA09
:105DB000DBE450BB0F0147F06C07FFB239462846C1
:105DC000FFF7F6F910F4804408D004237022394616
:105DD0002846FFF7FCF900243060C6E407234FF49F
:105DE000F06239462846FFF7F2F90B2330604FF492
:105DF000006239462846FFF7EAF900283FF4BBACB9
:105E0000336843F008033360AFE401287FF4B3AC98
:105E10000F0147F06C07FFB239462846FFF7C8F973
:105E2000336810F48044009307D00423702239466D
:105E30002846FFF7E3F9002497E407234FF4F062C4
:105E400039462846FFF7DAF98FE401287FF493AC4E
:105E50001B68090141F06C0100930F22002301F03F
:105E6000FC012846FFF7CAF900247EE460B9090165
:105E700041F06D010F234FF4004201F0FD0128466F
:105E8000FFF7A5F9306070E401287FF474AC1B685B
:105E9000090141F06D0100934FF400420F2301F01E
:105EA000FD012846FFF7AAF900245EE470B9090154
:105EB00041F06D010D234FF4C04201F0FD01284671
:105EC000FFF785F9306050E4945C002001287FF4EE
:105ED00052AC1B68090141F06D0100934FF4C042C0
:105EE0000D2301F0FD012846FFF788F900243CE46A
:105EF00060B9090141F06D0108234FF4706201F0AF
:105F0000FD012846FFF763F930602EE401287FF495
:105F100032AC1B68090141F06D0100934FF47062CF
:105F2000082301F0FD012846FFF768F900241CE46E
:105F300001287FF420AC1B68090141F06D0100933A
:105F40006022052301F0FD012846FFF757F90024E0
:105F50000BE460B9090141F06D0103460F2201F025
:105F6000FD012846FFF733F93060FFF7FEBB01283B
:105F70007FF401AC1B68090141F06D0100930F2211
:105F8000002301F0FD012846FFF738F90024FFF750
:105F9000ECBB68B9090141F06D0118234FF0807224
:105FA00001F0FD012846FFF712F93060FFF7DDBB75
:105FB00001287FF4E0AB1B68090141F06D010093FB
:105FC0004FF08072182301F0FD012846FFF716F903
:105FD0000024FFF7CABB01287FF4CDAB1B68090181
:105FE00041F06D0100934FF4FE02102301F0FD011A
:105FF0002846FFF703F90024FFF7B7BB68B909018A
:1060000041F06C0111234FF4003201F0FC012846ED
:10601000FFF7DDF83060FFF7A8BB01287FF4ABABDA
:106020001B68090141F06C0100934FF40032112309
:1060300001F0FC012846FFF7E1F80024FFF795BBCB
:1060400000287FF4ECAB090141F06F0110234FF4FD
:10605000F812C9B22846FFF7BAF83060FFF785BBDF
:1060600001287FF488AB20248C4064B244F01101F5
:106070001A68C9B22846FFF7B7F8336844F014012C
:10608000003318BF01234FF480620093C9B20A2382
:106090002846FFF7B3F80024FFF767BB68B909018A
:1060A00041F06C010D234FF4005201F0FC01284631
:1060B000FFF78DF83060FFF758BB01287FF45BAB2A
:1060C0001B68090141F06C0100934FF400520D234D
:1060D00001F0FC012846FFF791F80024FFF745BBCB
:1060E00001287FF448AB1B68090141F06C01009363
:1060F0004FF47002142301F0FC012846FFF77EF8EC
:106100000024FFF732BB00287FF489AB090141F07E
:106110006F01034640F2FF32C9B22846FFF757F835
:106120003060FFF722BB01287FF425AB2021A94076
:1061300041F019011A68C9B22846FFF755F8002442
:10614000FFF713BB50B92021A94041F01A01C9B291
:106150002846FFF72DF83060FFF707BB01287FF4D2
:106160000AAB2021A94041F01A011A68C9B2284699
:10617000FFF73AF80024FFF7F8BAE8B979B1012936
:106180007FF4F3AA01462846FFF712F800F06000FA
:10619000A0F12003584258413060FFF7E6BA0846A4
:1061A000FFF706F800F01800A0F11002504250412D
:1061B00030602C46FFF7D9BA01287FF4DCAA21B160
:1061C000012915D00024FFF7D0BA0846FEF7F0FFEA
:1061D000336820F0180243B142F010020021084653
:1061E000FFF702F80024FFF7C0BA42F00802F5E713
:1061F00000212846FEF7DCFF336820F0600243B13F
:1062000042F0200200210120FEF7EEFF0024FFF7FC
:10621000ACBA42F04002F5E707B50129019207D870
:10622000024601AB0120FFF706F903B05DF804FB5D
:106230000820FAE70129134603D802460020FFF799
:10624000FAB808207047012810B40C4606D8054B50
:1062500020461B6811469B6810BC1847002010BCE4
:10626000704700BFBC5E00202DE9F041614E624FD7
:106270008AB000213046614B01220CF0EDFAFD6836
:106280005F4C6B684FF0000803F5AA72626003F57B
:10629000B872A26003F56F72E26003F5767203F1E3
:1062A000C800226103F57D7203F58263A3612B6848
:1062B0006261DB68206098472B68E068DB6898477C
:1062C0002B68E0689B6998472B6860681B69984752
:1062D0002B68A0681B6998472B68A0691B699847C1
:1062E0002B6820691B6998472B6860691B69984770
:1062F0003A69444B444C1A606B68022703F53773C4
:1063000053606369414A0125136004333360404B95
:106310006A46009303F19F2303F56A035633019302
:106320003C4B414602933C4B304603936FF08063F5
:1063300004933A4B8DF824800593A3F1D943A3F538
:106340009113A3F227230693354B079380238DF8EF
:106350002030FF238DF821308DF822309DF8233036
:1063600067F3010365F3830365F3051365F387138F
:106370008DF82330F7238DF825300CF049FB6A4661
:10638000294630460CF044FB6369264A1D70C3F869
:106390000422254A83F80180C3F80822234B2846AB
:1063A0002362234B2774E361224BA361224B636278
:1063B000224BA363224B6363224BA362224BE36213
:1063C000224BA364224B6364224B6365224B2365FB
:1063D000224BE364224B2366224BE3653223E360C6
:1063E000DE23A360204BA365FEF770FF0AB0BDE873
:1063F000F08100BF945C0020649E02080024F40039
:106400006C160020BC5E0020203E0020905C002026
:1064100054B5AAAA29294924224210107D77BBB578
:10642000224240004552010839520108D353010865
:1064300035540108315401082D5401083562010812
:106440001962010861530108B1530108F9510108AB
:10645000C15101089D51010871520108755101088F
:10646000CD520108915101080D53010801289FBF29
:10647000034B53F8203000200B6088BF0820704782
:10648000C45E00200022014B5A607047203E00206D
:1064900070B50446074E084D33682A460146002071
:1064A0000CF074FC33682A462146BDE87040012098
:1064B0000CF06CBCC05E0020C45E002010B5034828
:1064C00014460CF0D2FB206010BD00BFC45E00205B
:1064D00001480CF0BCBB00BFC45E00200A46014668
:1064E00001480CF0D4BC00BFC45E00200968F5E789
:1064F0000A46014601480CF09BBC00BFC45E002068
:106500000021F5E74942F3E7F2E7024B18680CF087
:1065100086BC00BFC05E002008B5222108480CF0F0
:10652000A4FB50B9422106480CF09FFB28B9054B4B
:106530001868BDE808400CF069BC002008BD00BF29
:10654000C45E0020C05E0020012810B5144611D0A2
:1065500003D302281AD0042010BD14680F4A104B30
:10656000D268126824B15269D8689047002010BDE3
:106570009269F9E7094B0A4ADB6850681B681B6A95
:106580009847003018BF01202060EFE7034B044A12
:10659000DB6890681B681B6AF2E700BF649E020814
:1065A0009C160020022804BF0B4B93F8D80030B98A
:1065B0000A4BDB681B685B69094A106818470128A9
:1065C00009D1054B93F8D830012B04D1034BDB687C
:1065D0001B689B69F0E77047203E0020649E02081C
:1065E0009C16002070B50020FFF7DCFF104B114C0B
:1065F000DD6820682B689B6898472B6860689B68FB
:1066000098472B68A0689B6898472B68A0699B688F
:1066100098472B6820699B6898472B6860699B683E
:1066200098472B68E0689B68BDE87040184700BF3A
:10663000649E02089C1600201C2AF7B506460C46EC
:106640001F4600F0FB8200F292800C2A00F01982B3
:106650004BD8052A00F0B9811ED8022A00F06681C5
:1066600007D8002A00F03D81012A00F0528104265B
:1066700041E1032A00F07281042AF8D1002840F099
:1066800085812021BF4BA1401B6841F0070403EB2B
:10669000840463683B602EE1082A00F0D88111D899
:1066A000062A00F09F81072AE1D1002840F0BE8130
:1066B0002021A14041F01001C9B2B3480CF0D5FA35
:1066C000C0B217E10A2A00F0CF810B2ACFD10028EF
:1066D00040F054812021A14041F01501C9B2AA48DF
:1066E0000CF0C3FA00F0010004E1122A00F04B8222
:1066F0001DD80F2A00F023820CD80D2A00F0EE815D
:106700000E2AB4D1002840F012822021A14041F08D
:106710001401EBE0102A00F02082112AA7D10028F2
:1067200040F029822021A14041F00801DEE0152A35
:1067300000F04D820CD8132A00F03382142A96D12F
:10674000002840F03C822021A14041F00B01CDE027
:10675000172A00F05D82C0F04882182A87D10028ED
:1067600040F064822021A14041F01301BEE0AB2A39
:1067700000F0DE835ED8A52A00F00D832ED8A22A71
:1067800000F0C78217D81D2A00F07A828C2A7FF485
:106790006EAF002840F07B82090141F06C0101F0EE
:1067A000FC0179480CF061FA4FF4807300F00F009F
:1067B00043FA00F09EE0A32A74D0A42A7FF457AFD6
:1067C000002840F0D682090141F06C0101F0FC0183
:1067D0006D480CF04AFAC0F300308BE0A82A00F0B4
:1067E0005A8313D8A62A00F01A83A72A7FF43FAF52
:1067F000002840F03F83090141F06C0101F0FC01E9
:1068000061480CF032FA00F00F0073E0A92A00F0A2
:106810005F83AA2A7FF42BAF002840F07783090119
:1068200041F06D0101F0FD0157480CF01EFAC0F374
:1068300003205FE0B52A00F0FD8329D8AE2A00F0DE
:10684000B78313D8AC2A00F09383AD2A7FF40FAF3F
:10685000002840F09B83090141F06D0101F0FD012A
:1068600049480CF002FAC0F3006043E0B32A00F09C
:10687000C383B42A7FF4FBAE00287FD1090141F025
:106880006F01C9B240480CF0F0F9C0F3044031E0A8
:10689000CE2A00F0FD8313D8B62A00F0A681B82ACC
:1068A0007FF4E5AE002E40F05282210141F06C01F0
:1068B00001F0FC0134480CF0D8F9C0F340309DE100
:1068C000D22A00F0FA83D32A00F00584D12A7FF47B
:1068D000CEAE002840F0E9832021A14041F019010B
:1068E00004E058B92021A14041F00D01C9B2264869
:1068F0000CF0BBF93860304603B0F0BD012801D080
:106900000026F8E72021A14041F00D013A68C9B204
:1069100083E220B92021A14041F00101E6E70128EE
:10692000EED12021A14041F00101EFE720B9202163
:10693000A14041F00701D9E70128E1D112484318ED
:10694000202183F894623A68A14041F00701002AAF
:10695000B8BF5242C9B20CF07AF9D1E770B9202120
:10696000A14041F00201C9B207480CF07EF910F4D1
:10697000000318BF4FF07F431843BBE7012E3FF4DD
:1069800076AEBDE7C05E0020C45E00200128B7D10E
:106990002021B94B3A68A1401B6841F00705002A45
:1069A00003EB8503B8BF52425A60C9B2B3480CF03A
:1069B0005CF906460028A3D13A68E9B2002AB8BFBC
:1069C0005242AE480CF043F995E720B92021A1408E
:1069D00041F006018AE7012892D12021A14041F02F
:1069E000060193E750B92021A14041F01001C9B23E
:1069F000A2480CF03AF9C0F307207BE701287FF4A6
:106A00007FAF2021A14041F01004E4B221469B4811
:106A10000CF02BF9C3B201933B7800930022C0F332
:106A20000743214695480CF0DBF869E701287FF41D
:106A300067AF2021A14041F01004E4B221468F4805
:106A40000CF013F93B780193C0F30723E5E7002826
:106A500094D12021A14041F01501C9B287480CF022
:106A600004F9C0F3402045E7002887D12021A14048
:106A700041F01501C9B281480CF0F7F8C0F34000AD
:106A800038E720B92021A14041F01401F2E70128A4
:106A90007FF436AF2021A14041F01404E4B2214636
:106AA00076480CF0E2F83B6820F00202002BCCBFE5
:106AB0000223002321461A4370480CF0C8F82146EF
:106AC0006E480CF0D2F83B6820F00802022B08BF99
:106AD000082318BF00231A4321469EE120B9202134
:106AE000A14041F01401F9E501287FF409AF20210C
:106AF000A14041F01404E4B2214660480CF0B5F81E
:106B00003A6820F00100002AD4BF024640F001029A
:106B100021465A480CF09BF8214658480CF0A5F83D
:106B20003B6820F00402022B08BF0423D1E70128B0
:106B30007FF4E6AE2021A14041F01401E6E620B941
:106B40002021A14041F00401D0E601287FF4D8AE15
:106B50002021A14041F00401D8E620B92021A14024
:106B600041F00501C2E601287FF4CAAE2021A14010
:106B700041F00501CAE601287FF4C2AE2021A14000
:106B800041F00801C2E620B92021A14041F00A01EC
:106B9000ACE601287FF4B4AE2021A14041F00A0107
:106BA000B4E620B92021A14041F003019EE601286E
:106BB0007FF4A6AE2021A14041F00301A6E6012802
:106BC0007FF49EAE2021A14041F00B019EE620B94A
:106BD0002021A14041F00C0188E601287FF490AE0D
:106BE0002021A14041F00C0190E64EB92021A140A6
:106BF00041F01101C9B221480CF037F838607FE646
:106C0000012E7FF47DAE2021A14041F011017DE6EF
:106C100020B92021A14041F0120167E601287FF44C
:106C20006FAE2021A14041F012016FE601287FF4F0
:106C300067AE2021A14041F0130167E650B9090178
:106C400041F06C0101F0FC010C480CF00EF8C0F3AF
:106C500080404FE601287FF453AE090141F06C04F7
:106C6000E4B2214605480CF000F83B6820F480228D
:106C70009B0403F480232EE7C05E0020C45E002046
:106C800000287FF47BAEB94B53F8213002E5012890
:106C90007FF436AE1B68102B23D00DDC022B1CD0EA
:106CA00004DC012B16D04FF0FF3314E0042B16D078
:106CB000082BF8D105230EE0402B14D003DC202B49
:106CC000F1D1032307E0802B0FD0B3F5807FEAD109
:106CD000002300E008233B6008E00723FBE70623CE
:106CE000F9E70423F7E70223F5E738603B6801334F
:106CF0003FF406AE210141F06C04E4B221469B480A
:106D00000BF0B3FF3B6820F070621B0603F070636A
:106D1000E1E650B9090141F06C0101F0FC01934832
:106D20000BF0A3FFC0F3C130E4E501287FF4E8AD28
:106D3000090141F06C04E4B221468C480BF095FF48
:106D40003B6820F4C032DB0303F4C033C3E6012EFA
:106D50007FF4D6AD210141F06C04E4B221468348B2
:106D60000BF083FF3B6820F400525B0303F40053F5
:106D7000B1E601287FF4C4AD090141F06C04E4B22E
:106D800021467A480BF071FF3B6820F480521B03C8
:106D900003F480539FE6090141F06C05EDB22946EA
:106DA00072480BF062FFC0F3803466B929466F4821
:106DB00024B10BF05AFFC0F3C3109BE50BF055FF55
:106DC000C0F302101AE7012E7FF49AAD29466748F6
:106DD00044B10BF04AFF3B6820F4F062DB0103F49E
:106DE000F06318E00BF041FF3B6820F4006213F001
:106DF000080F18BF4FF4006429465C4822430BF08B
:106E000026FF294659480BF030FF3B6820F07002FE
:106E10001B0103F0700329461A4354489BE50901FE
:106E200041F06C05EDB2294650480BF01EFFC0F34F
:106E30008034BEB929464D4824B10BF016FFC0F38B
:106E4000021057E50BF011FFC0F3C310386029465C
:106E500046480BF00AFF3B68000A00F008000343B5
:106E60003B604DE5012E7FF44BAD29463F48002C99
:106E7000AFD0C8E701287FF443AD090141F06C04AD
:106E8000E4B2214639480BF0F0FE3B6820F00F02D7
:106E900003F00F031FE650B9090141F06D0101F045
:106EA000FD0132480BF0E1FEC0F3C03022E50128BD
:106EB0007FF426AD090141F06D04E4B221462B4870
:106EC0000BF0D3FE3B6820F40042DB039BB202E6EA
:106ED00050B9090141F06D0101F0FD0123480BF0AB
:106EE000C4FEC0F3413005E501287FF409AD090176
:106EF00041F06D04E4B221461C480BF0B6FE3B683D
:106F000020F4C0425B0303F4C043E4E501287FF4AE
:106F1000F7AC090141F06D04E4B2214613480BF0CF
:106F2000A4FE3B6820F470621B0203F47063D2E598
:106F300050B9090141F06D0101F0FD010B480BF062
:106F400094FEC0F34110D5E401287FF4D9AC0901C7
:106F500041F06D04E4B2214604480BF086FE3B6824
:106F600020F060025B0103F06003B4E5C45E002022
:106F700028B9090141F06D0101F0FD0140E401284B
:106F80007FF4BEAC090141F06D0479E701287FF47C
:106F9000B7AC090141F06D04E4B221467B480BF027
:106FA00064FE3B6820F080721B0603F0807392E55C
:106FB00080B9090141F06D0101F0FD0173480BF04A
:106FC00054FE001400F07F0310F0400018BF6FF073
:106FD0007F00D1E401287FF493AC090141F06D04F6
:106FE000E4B2214669480BF040FE3B6820F4FE0203
:106FF0001B0403F4FE036EE550B9090141F06C0176
:1070000001F0FC0161480BF030FEC0F3404071E438
:1070100001287FF475AC090141F06C04E4B221460B
:107020005A480BF022FE3B6820F400325B0403F464
:10703000003350E578B92021A1404DB245F014014C
:10704000C9B252480BF011FE10F480603FF4D6AD87
:1070500045F011014AE401287FF452AC2021A140FF
:107060004CB244F0110144F014041A68C9B2474804
:10707000E4B20BF0ECFD214644480BF0F6FD3B6812
:1070800020F48062002B14BF4FF48063002322E5BC
:1070900000287FF473AC090141F06F01C9B23B488D
:1070A0000BF0E3FDC0F3090024E401287FF428ACD1
:1070B0002021A14041F0190128E420B92021A1405C
:1070C00041F01A0112E401287FF41AAC2021A140FA
:1070D00041F01A011AE4C8B971B101297FF40BAC6F
:1070E00001462A480BF0C1FD00F06000A0F120032A
:1070F00058425841FFF7FEBB24480BF0B6FD00F0A4
:107100001800A0F110025042504177E501287FF4A9
:10711000F7ABF1B101297FF4F3AB00211B480BF071
:10712000A4FD3B6820F02002002B14BF2023002385
:1071300000211A4315480BF08AFD002113480BF07B
:1071400094FD3B6820F04002002B0CBF402300233D
:1071500019E00E480BF089FD3B6820F00802002B77
:107160000CBF0823002321461A4308480BF06FFD8B
:10717000214606480BF079FD3B6820F01002002BF9
:1071800014BF102300231A43002146E6C45E0020EA
:1071900007B50129019207D8024601AB0120FFF78C
:1071A0004BFA03B05DF804FB0820FAE70129134607
:1071B00003D802460020FFF73FBA08207047034B70
:1071C00008461B6811469B68184700BF6061002095
:1071D000F8B500263E4C3F4F20460BF097FDFD686A
:1071E00084F896626B683C4C03F5AA72626003F502
:1071F000B872A26003F56F72E26003F5767203F174
:10720000C800226103F57D7203F58263A3612B68D8
:107210006261DB68206098472B68E068DB6898470C
:107220002B68E0689B6998472B6860681B699847E2
:107230002B68A0681B6998472B68A0691B69984751
:107240002B6820691B6998472B6860691B69984700
:107250003A69224B22491A606B68022003F53773A2
:107260005360204B5A690A601F495670C2F80412D5
:107270001E49C2F80812012111701D4A18741A62C1
:107280001C4ADA611C4A9A611C4A5A621C4A9A6377
:107290001C4A5A631C4A9A621C4ADA621C4A9A6463
:1072A0001C4A5A641C4A5A651C4A1A651C4ADA640C
:1072B0001C4A1A661C4ADA653222DA604FF48C7274
:1072C0009A601A4A9A65BDE8F840FFF76BB900BFAB
:1072D000C45E0020649E02089C16002060610020AD
:1072E000C05E0020203E0020196501080B650108E2
:1072F000F1640108096501080565010801650108D7
:10730000AD71010891710108DD640108ED640108A7
:10731000D1640108BD640108916401084965010850
:107320006D640108A565010885640108E56501082B
:1073300018B9034B5B680B6070470820704700BFAB
:10734000646100200022014B5A607047203E0020FB
:107350000428F8B5144600F0848009D801284BD0E1
:107360001FD3022866D0032862D004242046F8BD2B
:10737000062800F0A580C0F09880072800F0A780BC
:10738000FC28F2D114685B4D5B4B002C00F0AB8005
:10739000DC6828692368DB689847236828699B694B
:1073A00016E0136833F0030240F0A28013F0010FDF
:1073B000504D514E0ED0F3681B681B6968689847A2
:1073C000246814F002040DD0F36828681B681B6958
:1073D00098472DE0F76868683B68DB6898473B682A
:1073E0009B69EBE7F66828683368DB689847336881
:1073F00028689B699847B9E7136844F6206293426E
:1074000076DC42F2107293423B4A3A4BD268586A99
:107410001268CCBF52699269904742F21173226898
:1074200092FBF3F003FB1020344B80B29B6898472B
:1074300000249BE71468304B64B1DC686068236803
:1074400000F50670DB6898476068236800F50670F1
:107450009B69BDE7DB6858681B6800F506709B6890
:10746000C8E71568234E244B5DB1012D15D0DD68AA
:1074700030692B681B6998472B6830691B6A9847ED
:1074800009E0DF6830693B68DB6898473B689B69C7
:107490003069984728462060CAE7DF6830693B6852
:1074A000DB6898473B685B69F2E7134B114ADB687E
:1074B000D0691B681B6A9847003018BF0120EAE7B3
:1074C0000D4B0C4ADB68106A1B681B6AF3E71368F4
:1074D000094A012BD268074B126898690CBF5269A0
:1074E00092699047A4E7DB6828691B681B6981E7FC
:1074F00010243BE7C4160020649E02087009002097
:107500001C4B70B5DD681C4C2B68A0689B699847C4
:107510002B68A06A9B6898472B68606A9B689847AD
:107520002B68E0689B6898472B6820699B689847A0
:107530002B6860699B6898472B6820689B68984710
:107540002B6860689B6898472B68E0699B68984740
:107550002B68206A9B6898472B68A0699B689847AE
:107560002B68A0689B689847BDE87040034B5B6838
:10757000184700BF649E0208C4160020700900204E
:1075800001480BF0FABC00BF6461002001460148CD
:107590000BF080BD6461002010B5034814460BF069
:1075A000FAFC206010BD00BF6461002008B5034BE9
:1075B00003481A680BF000FE002008BDF8630020A5
:1075C0006461002008B5034B03481A680BF0E0FD26
:1075D000002008BDF86300206461002008B502485F
:1075E0000BF0D3FD002008BD6461002008B50248FF
:1075F0000BF0C8FD002008BD6461002008B50248FA
:107600000BF0BEFD002008BD6461002008B50248F3
:107610000BF0A2FD002008BD6461002001480BF0C2
:1076200020BD00BF6461002038B522210B480BF05B
:10763000B2FC10B909480BF0FFFC094B094CDD689E
:10764000606A2B689B6998472B6820681B6998477C
:107650002B6860681B699847012038BD6461002071
:10766000649E0208C4160020022804BF0B4B93F846
:10767000D80030B90A4BDB681B685B69094A90681F
:107680001847012809D1054B93F8D830012B04D1B4
:10769000034BDB681B689B69F0E77047203E0020C6
:1076A000649E0208C4160020012903D1024A7021F9
:1076B0000BF063BC704700BFC80405008C2970B58F
:1076C0000446154600F06A8300F298800E2900F007
:1076D0004B8241D8062900F0BE8119D8022900F05A
:1076E000718107D8002900F04A81012900F05A81F0
:1076F00004244AE1042900F08B8140F273810028C0
:1077000040F0A0812621BE480BF045FC28603CE1FA
:107710000A2900F0D8810FD8072900F0B88108297C
:10772000E6D1002840F070813521B5480BF033FCDC
:10773000C0F34020286028E10C2900F0DC8140F2F1
:10774000CF81002840F0F8813421AD480BF023FCB4
:1077500000F00100286018E1152900F06E821FD8A2
:10776000112900F02D820DD80F2900F00E8210296A
:10777000BED1002840F01A822521A1480BF00BFC55
:10778000286002E1132900F03D8240F22A8200289D
:1077900040F049822B219A480BF0FDFB2860F4E071
:1077A0001C2900F0A5821AD8182900F06D821B2927
:1077B00000F07B8217299BD1002840F04F821521D1
:1077C0008F480BF0E8FB8F4B30B14FF08072B2FB6B
:1077D000F0F0834228BF03462B600024D5E0212926
:1077E00000F0A382222900F0BC821D2980D100284C
:1077F00040F00A81824B5B681360C6E0B32900F059
:10780000BF8457D8A82900F0048424D8A42900F004
:10781000478310D8A22900F01283A3297FF468AF10
:10782000002840F029836C2175480BF0B4FBC0F3AD
:1078300080302860A9E0A62900F0908340F24D83B3
:10784000002840F0D3836C216D480BF0A4FB00F0BE
:107850000F00286099E0AB2900F0288410D8A929EE
:1078600000F0F383AA297FF443AF002840F00A8494
:107870006D2163480BF08FFBC0F30320286084E088
:10788000AD2900F04C84C0F02E84AE297FF430AFD7
:10789000002840F061846D2159480BF07CFB0014F6
:1078A00000F07F0310F0400018BF6FF07F00184316
:1078B00028606AE0BB2900F0438536D8B62900F07D
:1078C000B5841FD8B42900F07A84B5297FF410AFAD
:1078D000002840F08384342149480BF05CFB4305C9
:1078E00040F17984142146480BF055FB454B30B1EB
:1078F0004FF08072B2FBF0F0834228BF03462B604A
:10790000002442E0B92900F0D38400F2F084B829C1
:107910007FF4EEAE002840F0B1846C2138480BF0C3
:107920003AFBC0F3403028602FE0CC2900F08C8572
:1079300012D8BF2900F04485C02900F06385BC2916
:107940007FF4D6AE002840F0298570212C480BF03A
:1079500022FBC0B2286018E0D12900F09485D2291A
:1079600000F0A485CE297FF4C3AE00284CD16F214E
:1079700023480BF010FBC0F30900286005E030B984
:107980002D211F480BF007FB2860204670BD012801
:1079900001D00024F9E712682D2119480BF0EDFA07
:1079A0000024F2E728B9212115480BF0F4FA2860E9
:1079B000EBE70128EDD11268212111480BF0DDFA27
:1079C0000024E2E728B927210D480BF0E4FA2860EB
:1079D000DBE70128DDD11268272109480BF0CDFA39
:1079E0000024D2E780B9222105480BF0D4FA10F424
:1079F000000318BF4FF07F4318432860C5E700BF5E
:107A000064610020FFFF0F00012CC2D10424BCE7F9
:107A100018B9AA4B1B681360B7E70128B9D11368DE
:107A2000A64E002BB8BF5B422021A54833600BF067
:107A3000B2FA04460028ACD132682721A0480BF0E6
:107A40009CFAA2E70128A4D1126826219C480BF0D9
:107A500094FA002499E738B9102199480BF09BFA61
:107A6000C0F30420286090E7012892D110219448A7
:107A70000BF091FA2B6820F4F8521B0203F4F85330
:107A80001A4310218E480BF078FA00247DE738B9AC
:107A900010218B480BF07FFA00F01F00286074E77C
:107AA00001287FF476AF102185480BF074FA2B681B
:107AB00020F01F0203F01F031A43102180480BF02F
:107AC0005CFA002461E700289ED135217C480BF048
:107AD00062FA10F0020F0CBF012300232B6054E761
:107AE000002891D1352176480BF055FAC04300F0BB
:107AF0000100286049E738B9342171480BF04BFA8E
:107B0000C0F34000286040E701287FF442AF3421F1
:107B10006B480BF040FA2C6834B940F00202342173
:107B200067480BF02AFA30E720F00202342164485B
:107B30000BF023FA002428E701287FF42AAF342130
:107B40005F480BF028FA2C6834B940F00102342168
:107B50005B480BF012FA18E720F001023421584874
:107B60000BF00BFA002410E728B9342154480BF02D
:107B700012FA286009E701287FF40BAF126834215C
:107B80004F480BF0FAF90024FFE628B924214C48AD
:107B90000BF001FA2860F8E601287FF4FAAE1268CB
:107BA000242147480BF0E9F90024EEE601287FF490
:107BB000F0AE1268252142480BF0DFF90024E4E61C
:107BC00028B928213E480BF0E6F92860DDE60128B7
:107BD0007FF4DFAE1268282139480BF0CEF900247B
:107BE000D3E628B92A2136480BF0D5F92860CCE62F
:107BF00001287FF4CEAE12682A2131480BF0BDF97E
:107C00000024C2E628B923212D480BF0C4F92860CE
:107C1000BBE601287FF4BDAE1268232128480BF093
:107C2000ACF90024B1E601287FF4B3AE12682B2131
:107C300023480BF0A2F90024A7E628B92C212048FC
:107C40000BF0A9F92860A0E601287FF4A2AE126823
:107C50002C211B480BF091F9002496E601287FF4B3
:107C600098AE1168174B69B14FF0807292FBF1F238
:107C70009A42A8BF1A462A60152111480BF07DF9D7
:107C8000002482E61A46F6E728B933210C480BF0A7
:107C900082F9286079E601287FF47BAE12683321EF
:107CA00007480BF06AF900246FE668B96C210448B4
:107CB0000BF071F9C0F3C040286066E6F86300205D
:107CC00064610020FFFF0F0001287FF462AE6C2189
:107CD000B0480BF060F92B6820F40022DB0403F4B9
:107CE00000231A436C21AB480BF047F900244CE603
:107CF00038B96C21A7480BF04EF9C0F380402860DA
:107D000043E601287FF445AE6C21A2480BF043F90D
:107D10002B6820F480229B0403F480231A436C21F7
:107D20009C480BF02AF900242FE638B90021994825
:107D30000BF031F900F00100286026E601287FF4FD
:107D400028AE002193480BF026F92B6820F00102A1
:107D500003F001031A4300218E480BF00EF90024B2
:107D600013E638B901468B480BF015F9C0F3400013
:107D700028600AE601287FF40CAE002185480BF04C
:107D80000AF92B6820F002025B0003F002031A4399
:107D9000002180480BF0F1F80024F6E558B96C2179
:107DA0007C480BF0F8F84FF48073C0F3036043FA9B
:107DB00000F02860E9E501287FF4EBAD1368102B93
:107DC00023D00DDC022B1CD004DC012B16D04FF08D
:107DD000FF3314E0042B16D0082BF8D105230EE056
:107DE000402B14D003DC202BF1D1032307E0802BA0
:107DF0000FD0B3F5807FEAD1002300E008232B6089
:107E000008E00723FBE70623F9E70423F7E702234B
:107E1000F5E728602B68013300F05B836C215D4837
:107E20000BF0B9F82B6820F070621B0603F070634A
:107E30001A436C2157480BF0A0F80024A5E538B987
:107E40006C2154480BF0A7F8C0F3C13028609CE5C2
:107E500001287FF49EAD6C214E480BF09CF82B68F6
:107E600020F4C032DB0303F4C0331A436C214948C9
:107E70000BF083F8002488E501287FF48AAD6C219B
:107E800044480BF088F82B6820F480429B0303F4ED
:107E900080431A436C213F480BF06FF8002474E5CF
:107EA00038B96C213B480BF076F8C0F300302860FD
:107EB0006BE501287FF46DAD6C2136480BF06BF853
:107EC0002B6820F480521B0303F480531A436C2167
:107ED00030480BF052F8002457E56C212D480BF088
:107EE0005AF89CB9460407D56C212A480BF053F880
:107EF000C0F3C310286048E5C0F3021300F400602B
:107F000003430CBF002308232B603EE5012C7FF4C4
:107F100040AD440410D56C211E480BF03CF82B6892
:107F200020F4F062DB0103F4F0631A436C2119487A
:107F30000BF023F8002428E52A68002411074CBF21
:107F400040F4006020F40060120120F07000D2B212
:107F500002436C210F480BF010F816E56C210D4818
:107F60000BF019F8C4B910F4804408D06C2109480A
:107F70000BF011F8C0F302102860002405E5C0F3EF
:107F8000C31300F4006003430CBF002308232B60DD
:107F9000FBE400BF64610020012C7FF4FAAC6C218B
:107FA000C1480AF0F8FF10F480444FF06C01BE485D
:107FB0000ED00AF0F0FF2B6820F070021B0103F0D6
:107FC00070031A436C21B8480AF0D7FF0024DCE4A0
:107FD0000AF0E1FF2B6820F4F062DB0103F4F063A8
:107FE0001A436C21B0480AF0C8FFCEE401287FF4A0
:107FF000D0AC6C21AC480AF0CEFF2B6820F00F0209
:1080000003F00F031A436C21A7480AF0B6FF0024BF
:10801000BBE438B96D21A4480AF0BDFFC0F3C030FD
:108020002860B2E401287FF4B4AC6D219E480AF0C8
:10803000B2FF2B6820F40042DB039BB21A436D2190
:1080400099480AF09AFF00249FE438B96D219648B8
:108050000AF0A1FFC0F34130286096E401287FF4C4
:1080600098AC6D2190480AF096FF2B6820F4C0422E
:108070005B0303F4C0431A436D218B480AF07DFF74
:10808000002482E401287FF484AC6D2186480AF044
:1080900082FF2B6820F470621B0203F470631A43A2
:1080A0006D2181480AF069FF00246EE438B96D2122
:1080B0007D480AF070FFC0F34110286065E4012894
:1080C0007FF467AC6D2178480AF065FF2B6820F0DB
:1080D00060025B0103F060031A436D2172480AF0ED
:1080E0004CFF002451E438B96D216F480AF053FF6A
:1080F00000F00F00286048E401287FF44AAC6D21AD
:1081000069480AF048FF2B6820F00F0203F00F03C4
:108110001A436D2164480AF030FF002435E438B971
:108120006D2161480AF037FFC0F3006028602CE43D
:1081300001287FF42EAC6D215B480AF02CFF2B68E0
:1081400020F080721B0603F080731A436D2156489D
:108150000AF013FF002418E401287FF41AAC6D2103
:1081600051480AF018FF2B6820F4FE021B0403F4A8
:10817000FE031A436D214C480AF0FFFE002404E47C
:1081800040B96C2148480AF006FFC0F3404028601F
:10819000FFF7FBBB01287FF4FCAB6C2142480AF0DF
:1081A000FAFE2B6820F400325B0403F400331A4318
:1081B0006C213D480AF0E1FE0024FFF7E6BB0028F1
:1081C0007FF422AC6F2138480AF0E5FEC0F304408A
:1081D0002860FFF7DABB2C60FFF7D7BB01287FF4DC
:1081E000D8AB342130480AF0D6FE2B6820F48062E8
:1081F000002B0CBF00234FF4806334211A432A481C
:108200000AF0BBFE2968294B71B14FF0807292FBD6
:10821000F1F29A42A8BF1A462A60142122480AF0B5
:10822000ACFE0024FFF7B1BB1A46F5E780B9142174
:108230001D480AF0B0FE1D4B30B14FF08072B2FB0A
:10824000F0F0834228BF03462B600024FFF79DBB5C
:1082500001287FF49EAB136873B14FF0807292FBDC
:10826000F3F2124B9A42C8BF1A4614210E480AF084
:1082700084FE0024FFF789BB0C4AF6E701287FF44F
:1082800088AB6C2108480AF086FE2B6820F4005267
:108290005B0303F400531A436C2103480AF06DFE9C
:1082A0000024FFF772BB00BF64610020FFFF0F00D6
:1082B00040B96C218B480AF06EFEC0F30350286071
:1082C000FFF763BB01287FF464AB6C2185480AF09B
:1082D00062FE2B6820F470021B0503F470031A433E
:1082E0006C2180480AF049FE0024FFF74EBB80B99C
:1082F00013217C480AF04FFE7B4B30B14FF0807267
:10830000B2FBF0F0834228BF03462B600024FFF746
:108310003CBB01287FF43DAB1168734B71B14FF04A
:10832000807292FBF1F29A42A8BF1A462A6013218A
:108330006C480AF022FE0024FFF727BB1A46F5E737
:1083400040B9702167480AF026FEC0F30720286074
:10835000FFF71BBB01287FF41CAB702161480AF0BA
:108360001AFE2A6820F47F40120292B20243702162
:108370005C480AF002FE00215A480AF00CFE2B6805
:1083800020F00402002B0CBF0023042300211A4319
:1083900054480AF0F2FD0024FFF7F7BA01287FF4F1
:1083A000F8AA70214F480AF0F6FD2A7820F0FF0065
:1083B000024370214B480AF0E0FD0024FFF7E5BAC4
:1083C00040B9702147480AF0E6FDC0F3014028603B
:1083D000FFF7DBBA01287FF4DCAA1368032B7BD8F4
:1083E000702140480AF0D7FD2B6820F440321B046E
:1083F00003F440331A4370213A480AF0BEFD0024CA
:10840000FFF7C3BA40B9702136480AF0C4FDC0F383
:1084100080402860FFF7B9BA01287FF4BAAA136830
:10842000012B5CD870212F480AF0B5FD2B6820F491
:1084300080229B0403F480231A43702129480AF008
:108440009CFD0024FFF7A1BA40B9702125480AF02D
:10845000A2FDC0F301502860FFF797BA01287FF40E
:1084600098AA70211F480AF096FD2B6820F440124C
:108470001B0503F440131A4370211A480AF07DFDCE
:108480000024FFF782BA30B9392116480AF083FD7B
:108490002860FFF77ABA01287FF47BAA1268392195
:1084A00010480AF06AFD0024FFF76FBA30B93A218C
:1084B0000C480AF070FD2860FFF767BA01287FF4C6
:1084C00068AA12683A2107480AF057FD0024FFF70E
:1084D0005CBA1024FFF759BA1024FFF756BA1024DB
:1084E000FFF753BA64610020FFFF0F0007B5019248
:1084F00039B9014601AA0120FFF7E0F803B05DF8A1
:1085000004FB0820FAE70B4619B901461846FFF7A5
:10851000D5B808207047034B08461B681146DB6836
:10852000184700BFF46300202DE9F0415A4E5B4C20
:10853000F56801276B68DFF8C88103F1C802A26003
:1085400003F58072E26003F58E72226103F5B87262
:10855000226003F5C672626003F5F072626203F591
:10856000FE72A26203F5617203F1E400A26103F5F9
:10857000687203F56F73E3612B6822621B696061A7
:1085800098472B6820691B6998472B68E0681B692E
:1085900098472B68E0691B6998472B68206A1B691C
:1085A00098472B68A069DB6898472B6820681B698F
:1085B00098472B6860681B6998472B68A068DB6840
:1085C00098472B68606ADB6898472B68A06ADB686D
:1085D00098472B68A0699B69984732690026304B01
:1085E00030491A606B68404603F5377353602E4B71
:1085F0005A69C2F804122D491770C2F808122C49A2
:10860000567019622B491F74D9612B4999612B4906
:1086100059622B4999632B4959632B4999622B491C
:10862000D9622B4999642B4959642B4959652B49C7
:1086300019652B49D9642B4919662B49D965322113
:10864000D9604FF4F071996028499965284B3146FB
:108650000AF0D5FC274940460AF018FDD8F800304A
:108660000220D3F8A020244B1A60FEF7FDFF02225F
:10867000A36A197C5A7418683A460CF04DF92B68B5
:10868000A06A1E4C1B68984723689847A368304629
:10869000BDE8F041184700BF649E0208C4160020E0
:1086A000F463002029760108203E00201D76010891
:1086B0000D760108FD750108ED750108DD750108ED
:1086C00007850108ED840108C5750108AD7501082D
:1086D00081750108997501088D75010851730108AC
:1086E00031730108697601084573010801750108B5
:1086F0005C9A0208A9760108F8630020700900203E
:108700006461002018B9034B1B680B607047082098
:10871000704700BF046400200022014B5A6070477C
:10872000203E00200428F8B50C4615467BD005D81D
:10873000022846D05CD8B8B104242EE0062800F008
:10874000A180C0F09480FC28F6D11468544D554B9C
:10875000002C00F09E80DC6828692368DB6898475D
:10876000236828699B6916E0136833F0030240F020
:10877000958013F0010F4A4E4A4F10D0FB681B68DA
:108780001B69706898472C6814F002040FD0FB68CE
:1087900030681B681B69984700242046F8BDFC68B8
:1087A00070682368DB68984723689B69E9E7FD6880
:1087B00030682B68DB6898472B6830689B6998475E
:1087C000EBE71468374B64B1DC686068236800F538
:1087D0000670DB6898476068236800F506709B693F
:1087E000D9E7DB6858681B6800F506709B68E6E708
:1087F0002B4B2C4A69B12C68D26814F00104126822
:1088000003D0526998699047C6E792699869904782
:10881000C3E7D26898691268126A9047003018BF9F
:1088200001202860B9E714681D4E1E4B5CB1012C75
:1088300015D0DC68306923681B6998472368306964
:108840001B6A984709E0DF6830693B68DB68984736
:108850003B689B6930699847204628609CE7DF6841
:1088600030693B68DB6898473B685B69F2E70D4B12
:108870000B4ADB68106A1B681B6A9847003018BFF8
:108880000120EAE7074B064ADB68506A1B681B6A4F
:10889000F3E7DB6828691B681B6990E710247CE715
:1088A000FC160020649E02081C4B70B5DD681C4C51
:1088B0002B68A0689B6998472B68A0699B699847BB
:1088C0002B68E0699B6998472B68E0689B6898472C
:1088D0002B6820699B6898472B6860699B6898475C
:1088E0002B6820689B6898472B6860689B6898474E
:1088F0002B68206A9B6898472B68606A9B6898473A
:108900002B68A0689B6898472B68A0699B6898476C
:108910002B68E0699B68BDE870401847649E0208B8
:10892000FC160020034B01461B68034A00200AF096
:108930008ABC00BF0064002004640020014B18685A
:108940000AF0B9BC00640020022804BF0B4B93F866
:10895000D80030B90A4BDB681B685B69094A90682C
:108960001847012809D1054B93F8D830012B04D1C1
:10897000034BDB681B689B69F0E77047203E0020D3
:10898000649E0208FC1600202DE9F0478846044644
:10899000924699461A4D002155F8203048F0800043
:1089A0009B689DF820709DF82460984755F8243006
:1089B00000219B685046984755F8243000219B6859
:1089C0004846984755F8243000219B683846984718
:1089D00055F8243030469B6801219847094B49EAF5
:1089E0000A2953F8243047EA092708F07F0803EBE7
:1089F000880846EA0726C8F80460BDE8F08700BF8B
:108A0000FC6300200064002007B5D3B20193C2F3D9
:108A100007230093C2F30743120EFFF7B5FF03B01D
:108A20005DF804FB0020FFF7EFBF73B50D46064667
:108A3000E8B9104C94F8283043B10F4B27211B683C
:108A4000D3F8A020FFF7E0FF84F8286000242A462E
:108A50002D210020FFF7D8FF2046019400942346E3
:108A600022462021FFF790FF204602B070BD08206B
:108A7000FBE700BFFC1600200064002037B50D4660
:108A80000446C8B901220D4B83F8282081EAE1721F
:108A9000A2EBE1722721FFF7B7FF002DACBF012346
:108AA0000223204601930094234622462021FFF70B
:108AB0006BFF204603B030BD0820FBE7FC1600200A
:108AC0000021DBE74942D9E7D8E74FF424732B4A6A
:108AD00070B503FB002301F07F04234493F80C32AC
:108AE0000546DB0706D4264B53F8203003EB8404FD
:108AF000606870BD234E002156F8203020469B68E8
:108B00009847002156F8253008469B689847002171
:108B100056F8253008469B689847002156F82530BE
:108B200008469B68984756F8253001219B6800202D
:108B3000984756F8253000219B6820469847002129
:108B400056F8253008469B689847002156F825308E
:108B500004029B6808469847002156F825300443D4
:108B60009B680846984756F82530240204439B68C2
:108B70000121002098472402204370BD0464002096
:108B800000640020FC63002010B500201446FFF7AD
:108B90009CFF206010BD38B50C4621210546FFF72B
:108BA00094FF2168014421602846BDE838403CE735
:108BB000222AF8B504460D461E4600F0478300F20F
:108BC0008E800E2A00F03C8241D8062A00F0B8813F
:108BD00019D8022A00F0618107D8002A00F03A81F2
:108BE000012A00F04A8104243AE1042A00F07C8141
:108BF00040F26981002840F09A8126212846FFF73B
:108C000064FF30602CE10A2A00F0D2810FD8072AD5
:108C100000F0B281082AE6D1002840F061813521B8
:108C20002846FFF752FFC0F34020306018E10C2ABD
:108C300000F0D68140F2C981002840F0EE81342155
:108C40002846FFF742FF00F00100306008E1152AD6
:108C500000F066821FD8112A00F01E820DD80F2A5C
:108C600000F0FF81102ABED1002840F00B822521A0
:108C70002846FFF72AFF3060F2E0132A00F0358221
:108C800040F22282002840F041822B212846FFF743
:108C90001CFF3060E4E01B2A00F084820DD8172A04
:108CA00000F04F82182A9ED1002840F071823321B3
:108CB0002846FFF70AFF3060D2E01D2A00F0AC82A0
:108CC000C0F08D82212A8ED1002840F0AC8201466E
:108CD0002846FFF7FAFE00F001003060C0E0AE2A3F
:108CE00000F0AF8451D8A72A00F0F58328D8A32A32
:108CF00000F02E8310D88C2A00F0C582A22A7FF4BF
:108D000072AF002840F010836C212846FFF7DDFE8B
:108D1000C0F3C1303060A3E0A52A00F0538340F2D5
:108D200034836C212846FFF7D0FE002C40F0AD8341
:108D3000410440F19F83000900F0700030608FE033
:108D4000AA2A00F0148410D8A82A00F0E083A92AE7
:108D50007FF449AF002840F0F6836D212846FFF7E5
:108D6000B4FEC0F3413030607AE0AC2A00F03984C0
:108D700040F21A84002840F050846D212846FFF705
:108D8000A4FEC0F3006030606AE0BB2A00F03C85BE
:108D900036D8B62A00F0B2841FD8B42A00F07784FF
:108DA000B52A7FF420AF002840F080843421284683
:108DB000FFF78BFE430540F1768414212846FFF728
:108DC00084FEBE4B30B14FF08072B2FBF0F08342B4
:108DD00028BF03463360002442E0B92A00F0CC8467
:108DE00000F2E984B82A7FF4FEAE002840F0AF8498
:108DF0006C212846FFF769FEC0F3403030602FE059
:108E0000CC2A00F0848512D8BF2A00F03C85C02A05
:108E100000F05B85BC2A7FF4E6AE002840F0218597
:108E200070212846FFF751FEC0B2306018E0D12A09
:108E300000F08C85D22A00F09C85CE2A7FF4D3AE38
:108E400000284DD16F212846FFF73FFEC0F30900EF
:108E5000306005E030B92D212846FFF736FE30603E
:108E60002046F8BD012801D00024F9E71A682D2119
:108E70002846FFF7C9FD0024F2E728B9212128463A
:108E8000FFF723FE3060EBE70128EDD11A682121BE
:108E90002846FFF7B9FD0024E2E728B92721284634
:108EA000FFF713FE3060DBE70128DDD11A682721C8
:108EB000002AB8BF52422846FFF7A6FD804B83F830
:108EC00028400024CCE758B922212846FFF7FDFDB1
:108ED00010F4000318BF4FF07F4318433060BFE722
:108EE000012CC1D10424BBE730B9764B53F82130B3
:108EF000D3F8A0303360B3E70128B5D1714B2846D1
:108F000053F8212033682021002BB8BF5B42C2F800
:108F1000A030FFF7DAFD04460028A5D132682721EA
:108F2000002AB8BF52422846FFF76EFD98E7012895
:108F30009AD11A6826212846FFF766FD00248FE79C
:108F400038B910212846FFF7C0FDC0F30420306077
:108F500086E7012888D110212846FFF7B6FD33683F
:108F600020F4F8521B0203F4F8531A431021284648
:108F7000FFF74AFD002473E738B910212846FFF7B0
:108F8000A4FD00F01F0030606AE701287FF46CAF99
:108F900010212846FFF799FD336820F01F0203F0E7
:108FA0001F031A4310212846FFF72EFD002457E720
:108FB000002895D135212846FFF787FD10F0020FD4
:108FC0000CBF0123002333604AE7002888D13521F4
:108FD0002846FFF77AFDC04300F0010030603FE70C
:108FE00038B934212846FFF770FDC0F340003060E7
:108FF00036E701287FF438AF34212846FFF765FDB6
:10900000336820F002025B0003F002031A433421AC
:109010002846FFF7F9FC002422E701287FF424AF5B
:1090200034212846FFF751FD336820F0010203F098
:1090300001031A4334212846FFF7E6FC00240FE71A
:1090400028B934212846FFF740FD306008E70128A1
:109050007FF40AAF1A6834212846FFF7D5FC0024B4
:10906000FEE628B924212846FFF72FFD3060F7E6F9
:1090700001287FF4F9AE1A6824212846FFF7C4FCC2
:109080000024EDE601287FF4EFAE1A68252128467A
:10909000FFF7BAFC0024E3E628B928212846FFF7A9
:1090A00014FD3060DCE601287FF4DEAE1A6828216A
:1090B0002846FFF7A9FC0024D2E600BFFFFF0F00FF
:1090C000FC1600200064002028B92A212846FFF75A
:1090D000FCFC3060C4E601287FF4C6AE1A682A2181
:1090E0002846FFF791FC0024BAE628B92321284638
:1090F000FFF7EBFC3060B3E601287FF4B5AE1A68E9
:1091000023212846FFF780FC0024A9E601287FF4EC
:10911000ABAE1A682B212846FFF776FC00249FE6A9
:1091200028B92C212846FFF7D0FC306098E60128AA
:109130007FF49AAE1A682C212846FFF765FC0024BC
:109140008EE678B915212846FFF7BFFCBB4B30B13E
:109150004FF08072B2FBF0F0834228BF03463360C9
:1091600000247DE601287FF47FAE1968B34B69B116
:109170004FF0807292FBF1F29A42A8BF1A46326019
:1091800015212846FFF740FC002469E61A46F6E759
:1091900001287FF469AE1A6833212846FFF734FCB2
:1091A00000245DE638B96C212846FFF78EFCC0F339
:1091B000C040306054E601287FF456AE6C2128464A
:1091C000FFF783FC336820F40022DB0403F4002360
:1091D0001A436C212846FFF717FC002440E638B9F3
:1091E0006C212846FFF771FCC0F38040306037E601
:1091F00001287FF439AE6C212846FFF766FC3368FE
:1092000020F480229B0403F480231A436C21284617
:10921000FFF7FAFB002423E600287FF461AE884BB9
:109220001B6833601CE601287FF41EAE002128462F
:10923000FFF74BFC336820F0010203F001031A43EF
:1092400000212846FFF7E0FB002409E638B9014673
:109250002846FFF73AFCC0F34000306000E60128E2
:109260007FF402AE00212846FFF72FFC336820F080
:1092700002025B0003F002031A4300212846FFF7B5
:10928000C3FB0024ECE558B96C212846FFF71DFC10
:109290004FF48073C0F3036043FA00F03060DFE501
:1092A00001287FF4E1AD1B68102B23D00DDC022BCD
:1092B0001CD004DC012B16D04FF0FF3314E0042B3C
:1092C00016D0082BF8D105230EE0402B14D003DC78
:1092D000202BF1D1032307E0802B0FD0B3F5807F43
:1092E000EAD1002300E00823336008E00723FBE70E
:1092F0000623F9E70423F7E70223F5E73060336834
:10930000013300F049836C212846FFF7DEFB336808
:1093100020F070621B0603F070631A436C2128462C
:10932000FFF772FB00249BE501287FF49DAD6C21C3
:109330002846FFF7CAFB336820F4C032DB0303F48E
:10934000C0331A436C212846FFF75EFB002487E5F3
:1093500038B96C212846FFF7B8FBC0F38030306085
:109360007EE501287FF480AD6C212846FFF7ADFB38
:10937000336820F480429B0303F480431A436C213A
:109380002846FFF741FB00246AE538B96C212846DE
:10939000FFF79BFBC0F30030306061E501287FF4EC
:1093A00063AD6C212846FFF790FB336820F48052B0
:1093B0001B0303F480531A436C212846FFF724FB58
:1093C00000244DE56C212846FFF77FFB0746CCB90A
:1093D00010F4804405D0C70907F4F0673760002413
:1093E0003EE56C212846FFF770FB17F00B0F4FEAA4
:1093F000201000F0700001D1306035E540F0080029
:1094000030602DE5012C7FF42FAD6C212846FFF74D
:109410005CFB10F480444FF06C01284612D0FFF73B
:1094200054FB336820F4F062DB0103F4F0631A4369
:109430006C212846FFF7E8FA002411E5FFFF0F0032
:1094400004640020FFF741FB6C2120F400622846F1
:10945000FFF7DAFA6C212846FFF737FB336820F074
:1094600070021B0103F070031A436C212846FFF7BA
:10947000CBFAF5E4C309020503F4F06301D43360C9
:10948000F2E443F008033360EAE4012C7FF4ECAC2F
:1094900010F480444FF06C0128460ED0FFF715FB06
:1094A000336820F070021B0103F070031A436C2133
:1094B0002846FFF7A9FA0024D2E4FFF706FB336839
:1094C00020F4F062DB0103F4F0631A436C212846B8
:1094D000FFF79AFAC4E438B96C212846FFF7F5FA89
:1094E00000F00F003060BBE401287FF4BDAC6C21BC
:1094F0002846FFF7EAFA336820F00F0203F00F0363
:109500001A436C212846FFF77FFA0024A8E438B9F3
:109510006D212846FFF7D9FAC0F3C03030609FE4D0
:1095200001287FF4A1AC6D212846FFF7CEFA3368FD
:1095300020F40042DB039BB21A436D212846FFF75B
:1095400063FA00248CE401287FF48EAC6D21284658
:10955000FFF7BBFA336820F4C0425B0303F4C04357
:109560001A436D212846FFF74FFA002478E438B9F2
:109570006D212846FFF7A9FAC0F3032030606FE49D
:1095800001287FF471AC6D212846FFF79EFA3368FD
:1095900020F470621B0203F470631A436D212846A5
:1095A000FFF732FA00245BE438B96D212846FFF753
:1095B0008CFAC0F34110306052E401287FF454ACBF
:1095C0006D212846FFF781FA336820F060025B01C5
:1095D00003F060031A436D212846FFF715FA0024B3
:1095E0003EE438B96D212846FFF76FFA00F00F000E
:1095F000306035E401287FF437AC6D212846FFF751
:1096000064FA336820F00F0203F00F031A436D2150
:109610002846FFF7F9F9002422E401287FF424AC5E
:109620006D212846FFF751FA336820F080721B063F
:1096300003F080731A436D212846FFF7E5F90024F3
:109640000EE478B96D212846FFF73FFA001400F0C8
:109650007F0310F0400018BF6FF07F0018433060A8
:10966000FFF7FEBB01287FF4FFAB6D212846FFF713
:109670002CFA336820F4FE021B0403F4FE031A43A1
:109680006D212846FFF7C0F90024FFF7E9BB002849
:109690007FF426AC6F212846FFF717FAC0F3044089
:1096A0003060FFF7DDBB3460FFF7DABB01287FF4E1
:1096B000DBAB34212846FFF708FA336820F48062D8
:1096C000002B0CBF00234FF4806334211A4328463B
:1096D000FFF79AF93168B54B71B14FF0807292FB88
:1096E000F1F29A42A8BF1A46326014212846FFF7C9
:1096F0008BF90024FFF7B4BB1A46F5E780B91421B3
:109700002846FFF7E2F9A94B30B14FF08072B2FB67
:10971000F0F0834228BF034633600024FFF7A0BB6C
:1097200001287FF4A1AB1B687BB14FF0807292FBE4
:10973000F3F29E4B9A42A8BF1A4632601421284683
:10974000FFF762F90024FFF78BBB984AF5E7012881
:109750007FF48AAB6C212846FFF7B7F9336820F411
:1097600000525B0303F400531A436C212846FFF7B1
:109770004BF90024FFF774BB40B96C212846FFF772
:10978000A4F9C0F303503060FFF76ABB01287FF4EF
:109790006BAB6C212846FFF798F9336820F4700210
:1097A0001B0503F470031A436C212846FFF72CF9BC
:1097B0000024FFF755BB80B913212846FFF785F930
:1097C0007A4B30B14FF08072B2FBF0F0834228BF89
:1097D000034633600024FFF743BB01287FF444AB0A
:1097E0001968724B71B14FF0807292FBF1F29A429C
:1097F000A8BF1A46326013212846FFF705F9002456
:10980000FFF72EBB1A46F5E740B970212846FFF74F
:109810005CF9C0F307203060FFF722BB01287FF41A
:1098200023AB70212846FFF750F9326820F47F40BF
:10983000120292B2024370212846FFF7E5F8002198
:109840002846FFF742F9336820F004029B0003F03A
:1098500004031A4300212846FFF7D6F80024FFF737
:10986000FFBA01287FF400AB70212846FFF72DF9DD
:10987000327820F0FF00024370212846FFF7C4F839
:109880000024FFF7EDBA40B970212846FFF71DF913
:10989000C0F301403060FFF7E3BA01287FF4E4AA87
:1098A0001B68032B7BD870212846FFF70EF933681D
:1098B00020F440321B0403F440331A43702128463D
:1098C000FFF7A2F80024FFF7CBBA40B97021284671
:1098D000FFF7FBF8C0F380403060FFF7C1BA012802
:1098E0007FF4C2AA1B68012B5CD870212846FFF7C1
:1098F000ECF8336820F480229B0403F480231A439D
:1099000070212846FFF780F80024FFF7A9BA40B974
:1099100070212846FFF7D9F8C0F301503060FFF7F7
:109920009FBA01287FF4A0AA70212846FFF7CDF83E
:10993000336820F440121B0503F440131A437021CE
:109940002846FFF761F80024FFF78ABA30B93921B9
:109950002846FFF7BAF83060FFF782BA01287FF493
:1099600083AA1A6839212846FFF74EF80024FFF72A
:1099700077BA30B93A212846FFF7A7F83060FFF7E9
:109980006FBA01287FF470AA1A683A212846FFF7B7
:109990003BF80024FFF764BA1024FFF761BA1024E3
:1099A000FFF75EBA1024FFF75BBA00BFFFFF0F009E
:1099B00007B5019239B9024601AB0120FFF7F8F86B
:1099C00003B05DF804FB0820FAE710B41346044620
:1099D000084619B9224610BCFFF7EAB8082010BCA7
:1099E000704738B522210020FFF76FF818B9084BEF
:1099F000186809F057FC074B074CDD6820682B6896
:109A00001B6998472B6860681B699847012038BD1F
:109A100000640020649E0208FC16002070B5524EBF
:109A2000524809F0D9FBF568514C6B6803F1E40228
:109A3000626103F58072E26003F58E72226103F5C4
:109A4000B872226003F5C672626003F5E272A26129
:109A500003F5FE7203F1C800E26103F5687203F5D5
:109A60006F7323622B686262DB68A06098472B6883
:109A7000A069DB6898472B68E069DB6898472B682A
:109A8000A0685B6998472B68A0699B6998472B6819
:109A9000E0695B6998472B6860691B6998472B6888
:109AA00020691B6998472B68E0681B6998472B68F9
:109AB000206A1B6998472B68606A1B6998472B6866
:109AC00020681B6998472B6860681B69984768681D
:109AD0002B6800F50670DB68984768682B6800F50E
:109AE00006709B6998473269224B23491A606B685C
:109AF000002003F537735360204B5A690A602049F0
:109B00005070C2F804121F490220C2F80812012145
:109B100011701D4A19741A621C4ADA611C4A9A6152
:109B20001C4A5A621C4A9A631C4A5A631C4A9A622B
:109B30001C4ADA621C4A9A641C4A5A641C4A5A65D6
:109B40001C4A1A651C4ADA641C4A1A661C4ADA6501
:109B50003222DA604FF425729A601A4A9A65BDE89B
:109B60007040FEF7F1BE00BF649E0208046400204E
:109B7000FC160020FC63002000640020203E002032
:109B8000E39901083D8901087D8A0108C98A010815
:109B9000C58A0108C18A0108CB990108B199010859
:109BA0002B8A0108978B0108258A0108898B0108F7
:109BB00025890108258701080587010849890108C9
:109BC00019870108A988010818B9034B5B680B6065
:109BD00070470820704700BF341700200022014B57
:109BE0005A607047203E00200428F8B50C46154600
:109BF00000F0868005D802284DD063D8C8B104246F
